:1000000000800020BD010000EDA90000A5A90000AE
:10001000A5A90000A5A90000A5A90000A5A90000A8
:10002000A5A90000A5A90000A5A90000EDA9000050
:10003000EDA90000A5A900006DA0000071A10000BD
:10004000EDA90000EDA90000EDA90000EDA9000058
:10005000EDA90000EDA90000EDA90000EDA9000048
:10006000EDA90000EDA90000EDA90000EDA9000038
:10007000EDA90000EDA90000EDA90000EDA9000028
:10008000EDA90000EDA90000EDA90000EDA9000018
:10009000EDA90000EDA90000EDA90000EDA9000008
:1000A000A9850000B5850000EDA90000EDA90000BC
:1000B000EDA90000EDA90000EDA90000EDA90000E8
:1000C000EDA90000EDA90000EDA90000EDA90000D8
:1000D000EDA90000EDA90000EDA90000EDA90000C8
:1000E000EDA90000EDA90000EDA90000EDA90000B8
:1000F000EDA9000059CA0000EDA9000085CB000061
:10010000EDA90000C5B30000EDA90000EDA90000B5
:10011000EDA90000EDA90000EDA90000EDA9000087
:10012000EDA90000EDA90000EDA90000EDA9000077
:10013000EDA90000EDA90000EDA90000EDA9000067
:10014000EDA90000EDA90000EDA90000EDA9000057
:100150005DA2000071A2000085A2000099A200002B
:10016000EDA90000E1B60000EDA90000EDA9000036
:10017000EDA90000EDA90000EDA90000EDA9000027
:10018000EDA90000EDA90000EDA90000EDA9000017
:10019000EDA90000EDA90000EDA90000EDA9000007
:1001A000EDA90000EDA90000EDA90000EDA90000F7
:1001B000EDA90000EDA90000EDA90000564B4CF29E
:1001C000205210B51A804DF628121A8000BF00BFC9
:1001D0000AF010FC514B4FF010621A60504A9A60BE
:1001E000504ADA60504A136813F4807304D14F49BF
:1001F0000B604FF4A85313604D4B1A78110703D5C9
:100200001A7842F008021A704A4B4B492A221A7097
:100210004A4A4B4B8B4204D252F8040F43F8040B6A
:10022000F8E7484B484900228B4202D243F8042B9E
:10023000FAE74649464A002352F8230041F82300D2
:1002400001336F2BF8D1434B434A802103F8011B44
:100250009342FBD1414B3D4A1A60414B8A221A70AE
:10026000A3F5805324225A70A0221A709A7992071B
:10027000FCD59A79D406FCD43A4A937903F00C035E
:10028000082B384BF9D103221A7140225A719A79FE
:100290009006FCD5334A9179324B4906FBD5324A58
:1002A000324911600221516020221A709A7902F0BD
:1002B0000C020C2AFAD12E4B2E4A1A602E4B2F4AD2
:1002C0001A6000225A60072243F8042C2C4AC3F813
:1002D0000C2D62B60AF03EFF144B1B68DA0705D5F9
:1002E00028480AF00BFD284B284A1A60284B1B7837
:1002F0005B0609D5244C254B22689A4204D121483B
:100300000AF0FCFC002323600DF0F6FE0AF078FBF7
:100310000AF0A6FAFEE700BF0E2005403080044038
:10032000823F04000100002B10D0034014D0034092
:1003300002D0074000E00740549BFF1FCC0F010094
:100340004088FF1F549BFF1F40A3FF1F0082FF1F19
:100350000000000000E400E05FE400E008ED00E0E1
:100360000050064000400640448004400000030165
:1003700004800440C010050014E000E0FF76010096
:1003800000002020F7C8D75E1CE00340A5C3945AA4
:1003900000F00740FFFFFFFFFFFFFFFFFFFFFFFF32
:1003A000FFFFFFFFFFFFFFFFFFFFFFFFFFFFFFFF5D
:1003B000FFFFFFFFFFFFFFFFFFFFFFFFFFFFFFFF4D
:1003C000FFFFFFFFFFFFFFFFFFFFFFFFFFFFFFFF3D
:1003D000FFFFFFFFFFFFFFFFFFFFFFFFFFFFFFFF2D
:1003E000FFFFFFFFFFFFFFFFFFFFFFFFFFFFFFFF1D
:1003F000FFFFFFFFFFFFFFFFFFFFFFFFFFFFFFFF0D
:10040000FFFFFFFFFFFFFFFFFFFFFFFFDEF9FFFF23
:1004100010B5054C237833B9044B13B10448AFF33E
:1004200000800123237010BD549BFF1F00000000BB
:10043000D00F0100084B10B51BB108490848AFF3B5
:1004400000800848036803B910BD074B002BFBD0A0
:10045000BDE81040184700BF00000000589BFF1F78
:10046000D00F0100549BFF1F0000000038B5044668
:10047000104621700A491D460DF020FC01464FF040
:100480007E500DF0CFFC07490DF018FCE560606070
:10049000256165610AF0EEFDE061204638BD00BFD0
:1004A000DB0FC9400024744938B50446104621705A
:1004B00009491D460DF002FC01464FF07E500DF03B
:1004C000B1FC06490DF0FAFBE560606025616561ED
:1004D0000AF0D0FDE06138BDDB0FC940002474494B
:1004E00038B503780446032B20D8DFE803F01A1848
:1004F0001002C16840690DF0D7FA0D4905466068E1
:100500000DF090FC014628460DF08CFC38BD0849E2
:1005100040680DF087FCE1680DF0D0FB38BDC06885
:1005200038BDC16840690DF0BFFA38BD002038BD44
:100530000024744970B504460E460AF09BFD05463A
:10054000E069281A0DF066FBE3682361E5616661E6
:10055000A061014660680DF065FC0146A06010488E
:100560000DF060FC0CF036FF0CF0D6FB0DF048FAF5
:10057000054601464FF07E500DF096FA61690DF088
:100580009DFB2169064628460DF098FB0146304642
:100590000DF08CFAE0602046BDE87040FFF7A0BF88
:1005A000000080BF38B50E201C4C0AF033F82188BB
:1005B0001B4B884205461A881DDA0023511AB1F5F3
:1005C000805FAABF1B03C3EB03330131142093FBED
:1005D000F1F10AF0A5FB134B1988F1B923889D426C
:1005E00010DAC3F57F630F33282091FBF3F1BDE8E8
:1005F00038400AF095BB9042D4BFC1EB0003C1EB79
:100600000203DBE740F6FF718D42D4BFC3EB050167
:10061000C3EB0101C1EB0131E3E738BD329CFF1FA1
:10062000DC9DFF1F849DFF1F10B5044609F0F4FDFB
:10063000204610BD70B44C88A04220D9012301335C
:10064000DBB21CB2660031F8144084421D46F6D37A
:10065000A04211D005F10045013D965B31F815101F
:1006600032F81530401AF21A00FB02F0641A90FBBF
:10067000F4F4E01870BC7047905B70BC70470226C1
:100680000125E5E700280CDA064A434282FB0320F5
:10069000DA17C2EB600000EB4000A3EB8000C0F172
:1006A0000C007047ABAAAA2A2DE9F0470C2009F0EC
:1006B0007DFF0C200AF032FCBB4914200AF03EFCFE
:1006C000BA49BB4807F076FC022103200AF0CCFCB3
:1006D000022104200AF0C8FC022105200AF0C4FC13
:1006E000022106200AF0C0FC01210A200AF0BCFC0D
:1006F000012109200AF0B8FC01210D200AF0B4FC08
:10070000012128200AF0B0FC012114200AF0ACFCE1
:10071000012116200AF0A8FC172001210AF0A4FCF0
:1007200004200AF093FC00283BD005200AF08EFC40
:10073000054600283CD0002528469E4C207005F038
:1007400003F824784CBB284606F014FC9A4B9B49CE
:100750001B889B4D098829709A4A9B4EA3F5AF715F
:1007600040F23A7303FB01F382FB0312DB17A3EBA6
:100770006213323301210D2033600AF061FC6420E2
:100780000AF09AFC4FF416710A200AF0C9FA5D21AA
:100790008E4807F0B9FF90B9FEE7BDE8F04707F0D3
:1007A00019BB06200AF052FC0028BED10125C4E77F
:1007B00003200AF04BFCB0FA80F04009BDE764204A
:1007C0000AF07AFC21460A200AF0AAFA4FF4967140
:1007D00009200AF0A5FA5C217D4807F095FF00B9D1
:1007E000FEE764200AF068FC214609200AF098FA26
:1007F0004FF4967116200AF093FA5B21754807F0C2
:1008000083FF00B9FEE764200AF056FC214616205B
:100810000AF086FA4FF4967117200AF081FA6420E4
:100820000AF04AFC214617200AF07AFA64200AF0FE
:1008300043FC21460D200AF003FC674A6748126812
:10084000DFF8E8A1DFF8A091654EDFF8E481654F9D
:1008500000230121FFF728FE0123C9F8004034607E
:10086000C8F800408AF8003004240F200AF016FE71
:10087000D8F8003003440E20C8F8003009F0CAFE52
:10088000D9F800309AF800200344C9F80030152048
:10089000002A78D009F0BEFE33681844306004F0B6
:1008A000010080F0010003F047FE3B88002B14BFDD
:1008B0004B20DC200AF000FC013CD6D1D8F80030F7
:1008C000D9F80020484930683C88DFF868E1474F94
:1008D000002BB8BF0333002AB8BF033292100A605E
:1008E0004349444A098812880028B8BF03309B1046
:1008F000801030605E1A19443E60CEF800103E4F02
:100900003E4E3F49C8F80030C2EB000E0244C7F823
:1009100000E032600B605CB94FF4FA7003F01CFE2B
:1009200003F006FE05F004FA4FF4AF600AF0C4FBD2
:10093000344B012404201C600AF088FB10B9324BB0
:1009400028701C70314B1B881C2B23D0304C04F1B9
:10095000C805232009F05EFE44F8040F01200AF0C8
:10096000ABFBA542F5D12B4A2B4B1078187006F043
:100970000BFA03F0D9FD45F6BF5228492848BDE8D7
:10098000F04709F0FFBB11200AF088FD33681844D6
:10099000306084E7234B18880028D7D0224BC0B2A0
:1009A000197806F039F9D1E7001B3746801A06009E
:1009B0006090FF1FA99BFF1FD89DFF1F489DFF1F31
:1009C000FC9BFF1FB5814E1B008AFF1FA89BFF1FCA
:1009D000309CFF1FD49BFF1F2489FF1F4C9DFF1FCE
:1009E000709BFF1F7A9DFF1F889BFF1FA49DFF1F09
:1009F000128AFF1F2C89FF1FC89BFF1F009CFF1F2F
:100A0000EC9DFF1FAC9DFF1F979BFF1FB29DFF1F1B
:100A10003C9CFF1F349DFF1F199DFF1FA505000073
:100A2000D09DFF1F049CFF1FC09BFF1F949DFF1FB5
:100A3000A09DFF1F1C9DFF1FF0B40E8886420DD2A3
:100A400003F10043013B31F81350854202D9F0BC59
:100A5000FFF7F0BD32F81300F0BC70471088F0BC0F
:100A6000704700BF094B1B880C2B09D8084A80B27D
:100A700052F8232028B143F6FE73984203D9108C14
:100A80007047108870470349FFF7D4BDA49BFF1F30
:100A9000E0F10000C8F20000374A38491088384AAF
:100AA000F8B5384B12881B68834248DB9342A8BFD5
:100AB000134698420B60C8BF002342DD101AB0F500
:100AC000804FAABF9B03C3EB8333013093FBF0F04D
:100AD000FFF7C8FF2C4B2D4F1C883B68C0F3C61591
:100AE00005FB04F47F2CA8BF7F249D42064608D056
:100AF000274B1B88002B38D1264B1B88002B30D16D
:100B00003D60254D2B689E4205D0214B1B885A1F06
:100B1000032A1DD92E60214D2B689C420ED0204BFC
:100B2000188848B11A4B1F4A1B88D35C834203D0F4
:100B3000C0B2E1B206F070F82C60F8BDF8BD034613
:100B400008609A42D4BFC0EB0203C0EB0303B5E7D1
:100B5000144AD05C2030C0B206F07F0106F05CF889
:100B6000D8E7284606F0CCF8CAE70E4A2946D05CFA
:100B700006F052F8C0E700BF329CFF1F789BFF1FB2
:100B8000DC9DFF1F809DFF1F8C9BFF1FDC9BFF1FB9
:100B9000709DFF1F2A9CFF1FE49DFF1F2C9CFF1FC1
:100BA000B69DFF1F048AFF1F2DE9F04F012089B079
:100BB0000AF074FCAF4B186000200AF06FFCAE4BDB
:100BC000AE4A1B8810600C2B00F03B81AC4BAD4A49
:100BD00019880093AC4B52F8214000221A70AB4B9D
:100BE000AB4D1B88AB4A2E88013B32F91370002EA7
:100BF0005CD0A94BA94A1B88A9491278013B31F95D
:100C00001380002A40F0DF8011200AF047FCA54B3A
:100C10000193D3F800A00646B24540F3DF80A24B13
:100C2000DFF8A4921B88A14A012BD9F80030B2F852
:100C300000B09F4A02922046C8EB030800F09A8257
:100C40000CF0E8FF029A52F82B100DF037F801462D
:100C500000200CF029FF0DF0F7F9CAEB0802B045AF
:100C6000B8BFB0469042CAEB080880F2968200FBFB
:100C70000888013298FBF2F08E4BDFF85082029325
:100C8000D8F80030034403EBD3735B10C8F800308E
:100C90002B88012B12D1884BDFF834B20393874B9A
:100CA000DBF8005004934FF0000A47E07D4B0193BE
:100CB000DFF814927F4BDFF8148202937E4B03938C
:100CC0001D460F200AF0EAFB2B689842824641DA63
:100CD000754A1288012A00F01D82744A0593128811
:100CE000734D049220460CF095FF049ADFF8E0B1B2
:100CF00055F82210DBF800500CF0E0FF0146002010
:100D00000CF0D2FE0DF0A0F9EF1B059B5745A7EBA9
:100D10000302B8BF5746FF1A9042BABF013200FB28
:100D20000777474397FBF2F7D8F80020634B04930B
:100D3000BB1803EBD3735B10C8F80030604B1B8803
:100D4000013B032B00F2B082DFE813F06301A9013D
:100D5000C4008601594B04931B68984240F3C2813A
:100D6000514A1288012A00F0A682504A079311883E
:100D70004F4A0691204605920CF04CFF059A0699C1
:100D8000DFF84CB152F82110DBF800500CF096FF60
:100D90000DF05AF9079B2F445745A7EB0302A8BF54
:100DA0005746FF1AD8F800309042BABF00FB0777C9
:100DB0000132474397FBF2F73B4403EBD3735B10DD
:100DC000C8F80030BAE7152009F024FC354B019330
:100DD000D3F800A00646B2453FF721AF354B02934A
:100DE000D3F800A0B24580F289812F4BDFF8D8906C
:100DF0001B882E4A012BD9F80030B2F800B02C4ADB
:100E000003922046984400F070820CF003FF039A8E
:100E100052F82B100CF052FF0DF016F9B045CAEB4A
:100E20000802A8BFB046CAEB08089042B6BF00FB54
:100E3000088800FB08F8013298FBF2F0DFF88C809C
:100E40001EE7204B1B78002B3FF4C0AE0C4B0D4A25
:100E5000198800930C4B52F8210001221A700CF0F3
:100E6000D9FE4FF07C510CF029FF0DF0EDF804464F
:100E7000B5E600BFD09BFF1FB29DFF1FF89DFF1F6F
:100E8000D69BFF1F8C89FF1F7E9BFF1F108AFF1FB1
:100E9000229DFF1FF0F30000608AFF1F949DFF1F3B
:100EA000A4F20000C89BFF1F169CFF1FA09BFF1F02
:100EB00008F40000009CFF1FA49DFF1F1C9DFF1F46
:100EC0006089FF1F969BFF1F709BFF1FBC9DFF1F2C
:100ED000A09DFF1F28460CF09DFEB2490CF0EEFECF
:100EE000054650460CF096FEAF490CF0E7FE014671
:100EF00028460CF0DBFD0DF0A7F80546CBF80050B6
:100F0000D9F800000CF086FEA6490CF0D7FE074683
:100F100030460CF07FFEA4490CF0D0FE0146384666
:100F20000CF0C4FD0DF090F8C9F800009F4AA04BEA
:100F3000168819889F4AA04B12681B889F4FC6EBE2
:100F4000050E3544039EC6F800E0461A084404998D
:100F50000D6001990E6002993E8808609A4280F205
:100F600089810025C3EB060E954974450F6880F210
:100F70007681611C9F4205FB01F50EF1010E95FB88
:100F8000FEF5C0F2BE81BE42A8BF3E46F61A01FB86
:100F900006F494FBFEF49A4200F33681BB42C0F2A1
:100FA0003381884C20680CF035FE87490CF086FEB2
:100FB00086490CF07BFD0DF047F8A0F5FF531C3B74
:100FC000082B98BF4FF40050D8F800301844002880
:100FD0002060C0F24281B0F5804F80F252817C4B9C
:100FE0001B781BB1B0F5005F40F05381794D2B7831
:100FF000002B40F05481784D20682B68714C98424A
:1010000004D080B205F0E6FE23682B6009B0BDE88D
:10101000F08F28460CF0FEFD70490CF04FFE05469F
:1010200050460CF0F7FD6E490CF048FE014628468C
:101030000CF03CFD0DF008F80546CBF80050D9F84F
:1010400000000CF0E7FD65490CF038FE074630461D
:101050000CF0E0FD62495FE728460CF0DBFD5A49E1
:101060000CF02CFE054650460CF0D4FD5D490CF00A
:1010700025FE014628460CF019FD0CF0E5FF05465B
:10108000CBF80050D9F800000CF0C4FD4E490CF02C
:1010900015FE074630460CF0BDFD52493CE7284698
:1010A0000CF0B8FD50490CF009FE054650460CF016
:1010B000B1FD4E490CF002FE014628460CF0F6FC4C
:1010C0000CF0C2FF0546CBF80050D9F800000CF038
:1010D000A1FD45490CF0F2FD074630460CF09AFDA3
:1010E000424919E7D8F80030DFF810B103EBD373A9
:1010F0005B10DBF80050C8F800301FE6DFF8008115
:10110000DFF80091D8F8003003EBD3735B10C8F818
:101110000030BDE5364A06931188364A05912046CF
:101120000492DFF8D8B00CF075FD049A0599DBF84D
:10113000005052F821100CF0C1FD0CF085FFEF1BA0
:10114000069B5745A7EB0302B8BF5746FF1AD8F8CE
:1011500000309042BABF013200FB0777474397FB4C
:10116000F2F73B4403EBD373234A04925B10C8F8B5
:101170000030E3E50CF04EFD029A52F82B100CF013
:101180009DFD0CF061FFCAEB0802B045B8BFB04648
:101190008242CAEB08083FF76AAD00FB08F898FBEB
:1011A000F2F069E5CDCC4C3FCDCC4C3E128AFF1F0E
:1011B0002C89FF1FD09BFF1F7E9DFF1FB89BFF1F29
:1011C000F89DFF1FC089FF1F9A99193FCDCC4C4550
:1011D000AF9EFF1F289CFF1F2089FF1F3333733FE3
:1011E000CDCC4C3DCDCCCC3E6666663FCDCCCC3D27
:1011F000A09BFF1F08F400001C9DFF1FA09DFF1F68
:10120000BC9DFF1F709BFF1F009B1B88002B3FF4A2
:10121000C8AE2B1B002BB8BF5B42092B47DD05F581
:1012200000500130001B0CF0F5FC3B493B4C0CF02E
:1012300045FD054620680CF0EDFC39490CF03EFDFB
:10124000014628460CF032FC0CF0FEFED8F80030C7
:10125000184400282060BFF6BEAE002213E09F4273
:1012600005FB04F5B8BF002195FBFEF54BDA91FBB9
:10127000FEF490E6B242D4BFC3EB0205C3EB060511
:1012800070E643F6FF72274B22601B78002B3FF479
:10129000ADAE03F04DF9244B01221A70ABE603F01A
:1012A00043F900232B70A6E6D9F800003EE64FF480
:1012B00000501A4C88E61D491D4A069320460D88A9
:1012C00005920CF0A7FC059ADFF868B052F82510DB
:1012D000DBF800500CF0F2FC014600200CF0E4FBBF
:1012E0000CF0B2FE2F44069B56E50CF093FC039ADB
:1012F00052F82B100CF0E2FC014600200CF0D4FB5D
:101300008AE51E4642E6B742D4BFC3EB0701C3EBF2
:10131000060104FB01F1AAE7CDCCCC3EC089FF1F3A
:101320009A99193FAF9EFF1F289CFF1FA09BFF1F8C
:1013300008F40000A09DFF1F38B5114C232025782C
:1013400009F068F90F4A42F82500131F02F1C400A2
:10135000002253F8041F83420A44FAD123780A4931
:1013600007480A4C0133DBB2322B81FB025108BF24
:101370000023D217C2EB21120370226038BD00BFD8
:101380008E9BFF1F409CFF1F1F85EB519C9DFF1FE5
:101390002DE9F04FB84CB94D2068B94F83B00CF02F
:1013A00039FCB8490CF08AFC064610200AF076F8A1
:1013B0000CF030FCB4490CF081FC31460CF076FBAB
:1013C0000CF042FE2988206088423B8843DA9E4622
:1013D0005B1A7F2B4FF0000247DDD2015E1C92FBAF
:1013E000F6F2AA4EDFF8C882B6F800C0C8F80020AE
:1013F000BCF1190F00F0DF80BCF11A0F00F017816B
:10140000BCF11E0F00F020810126B146A04A1288CF
:10141000002A00F09D808842C0F207817045D4BF49
:10142000C1EB0000C1EB0E009A42BABF02FB000004
:101430000133504390FBF3F3964A1360964B1888A0
:10144000C0B9964A1288AAB9954B197801B11A7099
:1014500003B0BDE8F08F9842D4BFC1EB0002C1EBEE
:1014600003029E465B1A7F2BB7DCC2EBC21292FBD3
:10147000F3F2B6E72988D4F800E0DFF80082DFF85D
:10148000F8A171456CDCDFF818C29CF80020002A36
:101490002ED14FF0010B04288CF800B028D1002E7B
:1014A00040F094817D4B18880028D1D0B9F1000F0D
:1014B000CED023682C883A88A34280F2658100232D
:1014C000141B7E2C774DD5BFC3EB8313C3EBC31323
:1014D0005B00013493FBF4F42B680134A34203D086
:1014E000C0B2E1B205F098FB2C6003B0BDE8F08F0C
:1014F000012800F0F680022800F0EB800328D1D10B
:10150000694B1B88092BCDD0002ECBD023682E88A9
:101510003A88B34280F27B810023961B7E2EDFF84F
:101520008CA1D5BFC3EB8313C3EBC3135B000136A0
:1015300093FBF6F6DAF800300136B34203D0F1B28D
:101540004A2005F069FBCAF80060ABE716469146F1
:10155000BCF11E0F7FF472AF0022DFF858817EE0ED
:101560004F4B1A78002A3FF473AF002401281C70F7
:1015700000F0A480022840F00E81002E00F0A3802D
:101580004A4D2B68002B00F09E800420214605F078
:1015900043FB424B2C60188800283FF459AFB9F147
:1015A000000F3FF455AFC0B2002105F035FB3D4BB5
:1015B00000221A604CE7DFF8FC8098F80020C2B1E6
:1015C000DFF8D890B9F800A0BAF1000F11D0DFF819
:1015D000E89099F800B0934578D05FFA8AF07F21BF
:1015E00005F01AFB98F80030B6F800C089F8003012
:1015F00010E0DFF8C49099F800A0924566D0274B20
:101600000021187805F008FB98F80030B6F800C003
:1016100089F800301E4B1A88002A97D0BCF11E0FA3
:1016200040F006810026B14619E00020FCE6DFF814
:10163000848098F80020002A0BBF012600264FF076
:1016400000094FF00109E1E6DFF86880104B98F8D7
:1016500000601A88B6FA86F676094FF0000998F805
:101660000030002B3FF4E8AE2988B7F800E020688E
:10167000C1EB0E03CFE600BFC49BFF1F2C9DFF1FD5
:10168000269DFF1F9A99193FCDCCCC3EB29DFF1FDE
:10169000E09DFF1F389CFF1FCE9BFF1FC49DFF1FB7
:1016A000B99DFF1FAC9BFF1F709DFF1F3C9CFF1F40
:1016B000989DFF1F969BFF1F929BFF1F1EB1614DC0
:1016C0002B68002B7BD1604B188865E70026B1465C
:1016D0009CE6002E3FF4E6AEDFF868A1DAF80020C1
:1016E0002EE0002E3FF4DEAEB7F80080F045D4BF08
:1016F000C1EB0802C1EB0E02C1EB0808B8F17E0F86
:10170000DFF840A1D5BFC2EB8212C2EBC212520079
:1017100008F1010892FBF8F8DAF8002008F1010856
:10172000424506D05FFA88F10120009305F074FA73
:10173000009B1888CAF8008002287FF4DFAE42467A
:101740002168B5F800803888414559DA0021C8EB96
:101750000008B8F17E0FD3BFC1EB8111C1EBC111FD
:1017600008F10108490091FBF8F808F101089045DB
:1017700006D05FFA88F10420009305F04DFA009B33
:101780001888CAF80080B9E69342D4BFC4EB0303BB
:10179000C4EB020394E6032827D12C4B1B88092BAA
:1017A00091D0002E8FD0274D2B68002B8BD04A2054
:1017B000214605F031FA244B2C601888ECE62146CE
:1017C00005F02AFA204B2C601888E5E640207F219E
:1017D0008DE80C0005F020FA019B009A1888584506
:1017E0001CD002287FF48AAE76E704287FF46BAF22
:1017F000002E3FF468AF2146402005F00DFA62E765
:101800008142D4BFC8EB0101C8EB00019FE79342BE
:10181000D4BFC6EB0303C6EB02037EE6B8F80010A4
:10182000DAF800E0B7F800808E45FFF665AF5DE7B7
:101830002988B7F800E020680026C1EB0E03B14606
:10184000E9E500BF3C9CFF1FC49DFF1F709DFF1F6B
:1018500008B50F4B1B88022B0FD0032B12D0042B83
:1018600003D00C4B01221A7008BD7F21092005F01E
:10187000D3F9084B01221A7008BD7F21412005F0E1
:10188000CBF9EEE74021092005F0C6F9E9E700BFF2
:10189000369CFF1FEF9BFF1F38B51C4B1B881D2B71
:1018A00026D01B4B1B88012B25D01A4A1A4B1488B3
:1018B0001B681A4AA342128818DB9342D4BFC4EBB8
:1018C0000303C4EB0203141B7F2CC6BFDB010134EE
:1018D000C3EBC31393FBF4F4114D2B689C4203D06C
:1018E000E1B2052005F098F92C6038BD0023EAE745
:1018F0000C4B1C88F0E70C4B0C4A0D491B68126816
:101900000C689B1A1C1B84F30704E5E7B29DFF1FBC
:10191000229DFF1FEA9BFF1F849BFF1FB09DFF1F9F
:10192000CC9DFF1FC09BFF1FEC9DFF1F2889FF1F41
:10193000309DFF1F10B50F4C23685BB90E4B1B8801
:10194000022B11D0033B012B09D90C4A0023137041
:10195000236010BD0021052005F05EF9EEE70021AF
:10196000092005F059F9F0E70021412005F054F96C
:10197000EBE700BFCC9DFF1F369CFF1FEF9BFF1FB7
:1019800008B5274B1B78ABB1152008F043FE254A5C
:10199000254B128818601D2A15D0244A1288EAB1F6
:1019A000012A25D0224B1B78002B34D0BDE80840FB
:1019B000FFF7C0BF112009F071FD1A4A1A4B1288B7
:1019C00018601D2AE9D11B4B1B78002BEAD0184B5D
:1019D0001B780BB3BDE80840FFF75EBF164A1288BC
:1019E000002ADFD0154A1B6812889A42DADCEEE73B
:1019F0000F2009F053FD104B114A1B88106033B1C2
:101A0000104B114A1B6812689B1A9842DFDD084B85
:101A10001B78002BCAD108BDFFF71AFFDAE700BF19
:101A2000949DFF1FB29DFF1F849BFF1F229DFF1FE0
:101A3000EF9BFF1F969BFF1F369CFF1FEA9BFF1F1C
:101A4000309DFF1FEC9DFF1F2889FF1F2DE9F04FE0
:101A5000A64C2278012A95B000F02082C0F0ED81DA
:101A6000022A00F0C980A248DFF81CE390F8008049
:101A7000A048A14DA14FA24EA24BA3490390A34859
:101A80000290A3489EF800B000902D78A1483F78BE
:101A900096F800E01B780978DFF8F4C2DFF8F492DA
:101AA000DFF8F4A20190012A94BF013200222270D3
:101AB000994A9A4813709A4A80F800B0157099486C
:101AC000994A077082F800809848994A037011700B
:101AD000BEF1000F40F0FF80964A10880D2800F0FC
:101AE0009D81954C00202070024604462DB19148FE
:101AF0000088002840F09E810546904806882544CD
:101B0000002E40F04B818E488E4C009E0078367837
:101B100024780130A0EB4600002C40F02782019C85
:101B200094F800E0CEEB0004BEF1000F40F04A82D2
:101B30000026DFF850E202989EF800E00078A41B2F
:101B4000A4EB4E043C44CBEB040410B1B7FA87F08D
:101B500040099CF800602718BC1B1EB11EF100064E
:101B600018BF012699F800009AF80090039FC6EB71
:101B7000040EC0EB0E00A0EB4900804497F800C0B3
:101B8000714FC3EB0803A3EB41010C2313FB0C11B2
:101B900039606E4B6E4C6F4E1B886F4824883768D7
:101BA00000886E4E033B03EB4303C4EBC40401EB1C
:101BB00083033C4403440C3B56F824001D44054475
:101BC0000AB1674B1960674B1A68954200F0228191
:101BD000654A664811680791079901601268089282
:101BE0006348089A00881D60521A824284BF614A85
:101BF000156015B0BDE8F08F5F4F08AE0025E9B263
:101C00005E4806F045FD57F8043B0135C01A0C2D1F
:101C100046F8040BF3D15A4B3D4D00953D4DB3F8BA
:101C200000C00195109D09980F99464EDFF8D0A08D
:101C3000DFF8C490DFF8CC80654511AA8CCAAE46A7
:101C4000ACBF4FF0000E4FF0010E8445D4BF002012
:101C5000012030708C452E480B9D254E8AF800E0FF
:101C6000D4BF00210121017094452A4921480390E5
:101C7000D4BF002201220A709C45424A23480290A8
:101C8000D4BF00230123BC45AB46D4BF00270127A6
:101C90001370AC45194B0C9D1F70D4BF4FF0000B57
:101CA0004FF0010B384B227883F800B0AC45DFF8D9
:101CB00058C098F800309CF8001096F80080DFF8C3
:101CC000D0C0DFF8D4A0D4BF0025012589F800508A
:101CD000DFF8C090E7E62D4A174814880122182C37
:101CE000027040F24B81002400E700BF189DFF1FE7
:101CF0006C9DFF1F219DFF1FEE9BFF1FEC9BFF1F95
:101D0000039EFF1F6D9DFF1F6E9DFF1FDA9DFF1F2E
:101D1000C79DFF1FC09DFF1FFD9DFF1FFE9DFF1F55
:101D2000FF9DFF1F009EFF1F019EFF1F029EFF1FC2
:101D3000B89DFF1F049EFF1F969BFF1F7C9BFF1FEC
:101D4000148AFF1FF09DFF1F749DFF1F889DFF1FBA
:101D5000A89DFF1F389CFF1F909BFF1F30F40000C1
:101D6000BC9BFF1FE49BFF1FEC9EFF1F089CFF1FF7
:101D7000C29DFF1FF49DFF1F3089FF1F309CFF1F76
:101D8000D89DFF1FC89DFF1FED9BFF1FB29DFF1F2A
:101D9000FC9DFF1FB49DFF1FB59DFF1F012E00F08E
:101DA0007981022E00F0D581032E9F4B00F00F8128
:101DB0001E78009B9CF800E01878029B99F800C000
:101DC00093F80080019B9AF800401F78A6EB4E0321
:101DD000A4EB8404CCEB030CC0EB80760CEB040387
:101DE000C0EB8600034403EB480303EB810327B1F8
:101DF0008E490978002940F04782012603998C48D2
:101E00000978C1F1060101EB4101334403EB810183
:101E10000160BEE68749884A0968DFE6002D3FF485
:101E200060AE864A864E14880122182C327040F229
:101E3000A5807446A0F10D055FE6824F08AE00252F
:101E4000E9B2814806F024FC57F8043B0135C01A7A
:101E5000062D46F8040BF3D17C4A7D4B03921646BF
:101E60001B880D9A00219A423170C0F294800C9A1E
:101E7000934240F3D8817749774A91F80080774BB5
:101E800011780398764A029205221B78DFF8F8C190
:101E9000DFF8F891DFF8F8A1027057E0714F08AE53
:101EA0000025E9B2704806F0F3FB57F8043B013512
:101EB000C01A0C2D46F8040BF3D1654B0C9D1F88FE
:101EC000674B02930B9B0A98099A089EDFF8C0A102
:101ED000DFF8B8910F99DFF8B0C1BB42ACBF4FF04B
:101EE000000E4FF0010EAF42D4BF002501258742FE
:101EF000109B8CF80050D4BF002001209742D4BF23
:101F000000220122B742D4BF4FF000084FF0010871
:101F10008AF800209F42514A89F80000D4BF00236C
:101F200001234C481370129A80F800808F424C4E67
:101F3000494886F800E0D4BF002101219742017092
:101F40003ADC00224948414D039502704848494A0D
:101F5000494E4A4D07784A4800904A4892F800E0B6
:101F600096F800B02D78227801909CE5019C46B14E
:101F70002678002E40F07081441EDAE50C3C0122E8
:101F8000B4E594F800E00138CEEB0004BEF1000F98
:101F90007FF4CFADCCE52F492F4A304B91F800802C
:101FA00011782F4A35701B780292DFF8DCC0DFF819
:101FB000DC90DFF8DCA0C9E7119A9742D4BF002279
:101FC0000122BFE7002E3FF4B3AD0126B1E51C7836
:101FD0000298009B9CF800601B7890F800C099F86C
:101FE000007001989AF8008090F800E0A4EB460495
:101FF000E71BA8EB8800C3EB83743844C3EB84036E
:10200000034403EB4C0303EB8103BEF1000F40F0EC
:102010004081012603990648097833440C2414FBB7
:1020200001310160B5E500BF148AFF1FC89DFF1F85
:10203000749DFF1F089CFF1FEC9EFF1FB29DFF1F9A
:10204000969BFF1F488AFF1FA89BFF1F219DFF1F14
:10205000D89DFF1F6C9DFF1F6E9DFF1F6D9DFF1F75
:10206000DA9DFF1F188AFF1FD49BFF1FBA9BFF1F1B
:10207000EC9BFF1F039EFF1FED9BFF1FEE9BFF1FAF
:10208000C79DFF1FC09DFF1FFC9DFF1FB49DFF1F2D
:10209000B59DFF1FAA4CDFF8B4E2207805909EF8AA
:1020A000004000980494059C007800900134A4EB53
:1020B00040040498002840F0A780019890F800E0C0
:1020C0000498261ACEEB0606BEF1000F40F096806B
:1020D000CDF810E09B4C029824780194049C007881
:1020E000341B019EA4EB46043C44CBEB040410B12A
:1020F000B7FA87F040099CF800602044871B1EB1A6
:102100000198061C18BF012699F800009AF80040B3
:10211000BE1B301AA0EB440080440098C3EB0803B8
:10212000A3EB4103002864D1BEF1000F40F0BB8057
:102130007344002C75D100290CBF00206FF00900FA
:102140000399814C097803440C2010FB0131216074
:102150001FE5009C019E247800947C4C3678019603
:102160009AF8006094F800A0764C794899F800E05D
:1021700094F800909DF80440847080F806E080F8A0
:1021800003909CF800C09DF80040DFF8DC91DDF87A
:1021900000E080F808800470077180F805C0C671FF
:1021A000417280F801A04FF0000801200021684C26
:1021B0000E465FFA88FA4F46F44607E0022809D037
:1021C0000A290BD014F801CF17F8010F844501F14B
:1021D0000101F3D101360A29F6B2F3D1092E00F23A
:1021E000828008F10108B8F10F0F38D019F80A0FF2
:1021F000DCE74FF0000E9BE7CEEB040600980030C2
:1022000018BF0120049065E70098002853D001987A
:1022100090F800E0BEF1000FEED1661ECDF810E0A0
:1022200058E700208CE70B9A934249DC0A9A9342C4
:102230006FDD4849484A91F80080484B117803986F
:10224000474A029203221B78DFF820C1DFF8209171
:10225000DFF820A1027079E6841B012669E4384882
:1022600040490478886B0299013409782044CBEB0B
:102270000000084400230399334C0E78C31A0C2144
:1022800011FB0631216084E41BF1000618BF012612
:10229000B4E52C49097800293FF4BBAE1BF10006D8
:1022A00018BF0126B6E6019800280CBF4FF0000EBB
:1022B0004FF0090E3CE7019890F800E0304600E747
:1022C0002449254A91F80080244B11780398244A28
:1022D000029204221B78DFF894C0DFF89490DFF8B4
:1022E00094A0027032E616481E49047851F828007E
:1022F0000299013409782044CBEB00000844002BFC
:10230000B8D0BAF1000FB5D1BBF1000FB2D00123A4
:10231000B1E7099A93422FDD0E490F4A91F80080E8
:102320000E4B117803980E4A029202221B78DFF8B6
:102330003CC0DFF83C90DFF83CA0027006E600BF2E
:10234000148AFF1FC89DFF1F749DFF1FF09DFF1F74
:102350000C9CFF1F6C9DFF1F6E9DFF1F6D9DFF1F3F
:10236000DA9DFF1FC489FF1FECF20000FC9DFF1FD8
:10237000B49DFF1FB59DFF1F089A0B49DFF838C0B9
:1023800091F80080DFF83490DFF834A09342074AD8
:10239000074B1178074A1B7802927FF7D7AD039855
:1023A00001220270D2E500BF6C9DFF1F6E9DFF1FD2
:1023B0006D9DFF1FDA9DFF1FFC9DFF1FB49DFF1F3A
:1023C000B59DFF1F2DE9F04F2E4B1B788BB0002BD6
:1023D00053D10E2008F01EF90BF01CFC01462A48D0
:1023E0002A4C2B4DFEF7A6F82748FEF779F80BF09C
:1023F0002BFE80F30C002060FFF728FB2E68012ED7
:102400005AD0022E00F08782032E00F09783214CD1
:102410002368214A214E0993099B17783068204C84
:1024200007210122181A11FB07229042236000F2B3
:102430006D821C4E32689A1A0D2A00F260821A4E82
:1024400032689A1A132A00F25582184E32689A1A84
:10245000252A00F23C82164D2A689B1A502B00F266
:10246000F581144B1B88012B00F00D8204F068FCF1
:1024700004F096FA0BB0BDE8F08F05F033FB0BB01B
:10248000BDE8F08FA99BFF1F4C9DFF1F809DFF1F84
:10249000AC9DFF1FEC9EFF1F1A9DFF1F289DFF1F75
:1024A000449DFF1F209CFF1FF49BFF1FF89BFF1FF5
:1024B000389DFF1F849DFF1FDFF800839A4AB8F8FC
:1024C00000001378834204D0C3B21846137004F09E
:1024D00073FBDFF8E492954AB9F80030117899421D
:1024E00004D0934F3978002940F09887914A2368A7
:1024F0001288914C9A42C0F2EE80904A1278002ADB
:1025000040F0E980DFF8B8A2BAF8003023B98C4B6C
:102510001B88002B00F042858A4A8B4B11881B8850
:102520008A4A0B4412685B109342894A126880F20F
:10253000B78400219342B4BF01230B46049100935A
:10254000ACBF4FF0010B8B4605910E2008F062F8EE
:10255000804B814A1B68176803930133A7F25232FC
:10256000002B8446029240F36A87802BA8BF802309
:102570007A4A7B4912780191002A00F0B6800978E6
:10258000914200F0B280B9F80010DFF82CE29942D5
:1025900001F061816649AEF80030724B4FF0010ED8
:1025A00081F800E01978DFF81CE2019B8EF800103A
:1025B0001A70009B002B00F00781BAF80030002B46
:1025C00000F00281684B1B685A1C002A40F33B87CD
:1025D000802A00F33787654E654966483688098842
:1025E00000683144B0EB610FC1F20982A3F14802E7
:1025F0000F2A02D8473BA8F800300E2008F00AF84E
:102600006FF454731F44874202DC5B4B00221A7044
:102610005A4B1B88002B00F03B84594B594A1B78BE
:102620001178994240D0002B3ED057490E78002EA9
:1026300000F0EE87554991F800C0BCF1000F40F062
:10264000E587534F0097534F53480297504F0078F8
:1026500087F800C04F4F4FF0010E87F800C081F897
:1026600000E0002841F089814C490978002901F0F7
:102670004A804B4903910E460978002941F0408079
:102680004848444F0078397001210297317058B1A1
:102690003F483E490090002008700099029F087052
:1026A000039901263E70087013703F4B1B88A3F1FD
:1026B0001B02012A40F28D861D2B7FF4A9AE394FF3
:1026C0003B78002B41F00C81384E3378002B40F0E2
:1026D000958433709CE62168354A06910698354901
:1026E000106002220B602A600CE71E49DFF8D4E07C
:1026F000097800293FF459AF9EF8000081423FF469
:1027000054AF03984B2841F352801833802BB9F80B
:102710000000A8BF802398423FF447AF26480380BB
:1027200003480123037040E7199DFF1FFC9BFF1F17
:10273000979BFF1F329CFF1FEC9EFF1FA29BFF1F5A
:10274000269CFF1FB89BFF1F7E9DFF1FD09BFF1F76
:10275000F89DFF1FBC9BFF1F889BFF1FE89DFF1F6D
:10276000E09BFF1FE99DFF1F749DFF1F2C9DFF1F16
:10277000269DFF1FC49BFF1F209DFF1F869DFF1FDF
:10278000BA9BFF1F749BFF1F009EFF1F7C9DFF1FB6
:10279000C69DFF1F349CFF1F019EFF1FFD9DFF1F55
:1027A000759BFF1F969BFF1FB29DFF1F929BFF1FF4
:1027B000F09BFF1F409DFF1F489DFF1F349DFF1F83
:1027C000E89BFF1FE19BFF1F029B9C45BFF615AFD7
:1027D0008E4B1B88002B3FF410AFBBF1000F7FF432
:1027E000F1AE8B4B1B881BB1059B002B7FF4EAAE2F
:1027F000049B002B3FF401AF864B1A78002A7FF42C
:10280000FCAEDFF8888298F8006001221A70002E72
:1028100040F09183804B1B78002B01F032817F4B7D
:102820001B78002B01F043817D4B1B78002B7FF43C
:10283000E4AE7C4B1B78002B3FF4DFAEB9F80030E0
:1028400079490A3BA9F800300A70D6E602F0C4FFC5
:10285000764B1B7873B9764B1B785BB9754B1B783D
:1028600043B9754B1B782BB9744B1B7813B901F026
:102870005BFE01E001F064FE23682B60704B1B8857
:10288000012B7FF4F3AD6F4A6F4B11686F481A78D4
:10289000A1F118032A2101FB03F10160002A00F0D5
:1028A000E1826B4A1368994200F37C8380F286834D
:1028B00068480068D0F17F0048BF033080100130C5
:1028C0001B1A994200F37A8313601946CCE2FEF793
:1028D00033FD614B1B881B3B9BB2022B05D85F4B22
:1028E0001B7813B12B68012B01D001F047FE236840
:1028F0003360B0E5FFF744F823683360A5E5FEF7E1
:1029000053F9FEF745FD2368336098E5FEF7C4F8F8
:10291000236833608DE5524A26681288B24204DB90
:10292000464B1B78002B00F064834E4C4E482368C6
:1029300007934E4B079900681B88091A994200F2C9
:10294000AB80002B00F0A880494B198800293FF488
:102950005FAD484B48481B680088B342B8BF334658
:102960009A4241F34580454B1A60DFF8248188F88C
:102970000010344FFEF790F838687F2840F3428605
:102980003F4B7F3883FB0032C317C3EB620303EB7B
:102990004303A0EB830073303A4B01931B883860EC
:1029A000002B40F04A87234B00931B78002B00F04C
:1029B0007384354E3378002B00F06E84DFF8D490AA
:1029C000DFF8BCA04FF0000B0CE003F17300C0B2C5
:1029D00098F8001004F048F933780BF1010B5B45CF
:1029E00040F35A843B6859F8040F1844A0F17F0360
:1029F0008AFB0321DA17C2EB610202EB42027F2855
:102A0000A3EB8203E1DCFDF73DFEE0E7269CFF1F20
:102A10003C9DFF1F209DFF1FFD9DFF1FFE9DFF1F73
:102A2000FF9DFF1F009EFF1F979BFF1F349CFF1FF2
:102A30007C9DFF1FC69DFF1F759BFF1FA29BFF1F55
:102A4000849DFF1FF49DFF1FEF9BFF1F1C9CFF1F1A
:102A50009C9BFF1FCC9DFF1FB29DFF1F969BFF1FDE
:102A6000329CFF1FEC9EFF1FF09BFF1F249CFF1F4B
:102A7000949BFF1F409DFF1FDC9DFF1F789BFF1F46
:102A8000ABAAAA2ACC9BFF1F8889FF1F219DFF1F8D
:102A9000189CFF1F6089FF1F554B56491B6808880B
:102AA0005549B342B8BF33469A4200F38982534E28
:102AB00009888342A8BF0346336000297FF455AFDD
:102AC0009A42C8BF0B4640F38282801AB0F5804F0D
:102AD000AABF9B03C3EB8333013093FBF0F0FDF7F8
:102AE000C1FFC0F3C6100BF095F8454B0646188899
:102AF0000BF090F84349074630460BF0DFF80146EB
:102B000038460BF0DBF831460AF0D0FF4FF07E512B
:102B100006460BF071FA002840F05F873A493046CC
:102B20000BF088FA002840F01C8730460BF0B2FA10
:102B3000C0B2DFF8F48088F800001AE7334B26684B
:102B40001988B14274DD324B1B78002B70D1DFF84D
:102B5000DC9099F800007F2840F3BE86A3F155333E
:102B60007F3803F1004383FB0032C317C3EB6203DA
:102B700003EB4303A0EB83007330264B01931B88C8
:102B8000C0B289F80000002B40F00787224B009369
:102B90001B78002B00F06785204E3378002B00F067
:102BA00062851F4FDFF87C804FF0000A0AE003F1D6
:102BB0007300C0B204F080F833780AF1010A53457B
:102BC00040F3518557F8043F99F800001844A0F1EC
:102BD0007F0388FB0321DA17C2EB610202EB42029A
:102BE0007F28A3EB8203E2DCFDF74CFDE1E700BFA9
:102BF000409DFF1FDC9DFF1F949BFF1F789BFF1FC5
:102C0000809BFF1FCDCCCC3D0000FE42329CFF1FBD
:102C1000A29BFF1FCC9BFF1FC69DFF1F8889FF1F24
:102C20006089FF1FABAAAA2A189CFF1F789DFF1F6F
:102C3000A24F38687F2840F3D181A14B7F3883FBB6
:102C40000032C317C3EB620303EB4303A0EB830023
:102C50007330DFF8B49299F800A0824500F0288222
:102C6000984B1B88002B43D1974A984812680088DC
:102C7000914205DC8242D4BFC1EB0203C1EB0003E9
:102C8000411AB1F5804FA6BF9B030131C3EB8333DB
:102C900093FBF1F0FDF7E6FEC0F3C6100AF0BAFFB1
:102CA0008B4B064618880AF0B5FF8A4980463046A5
:102CB0000BF004F8014640460BF000F831460AF0EC
:102CC000F5FE4FF07E5106460BF096F9002840F0D5
:102CD0006186814930460BF0ADF9002840F030861E
:102CE00030460BF0D7F9C0B2DFF8208288F8000038
:102CF000BAF17F0F40F381847148AAF17F0A80FB0B
:102D00000A304FEAEA73C3EB600000EB4000AAEB25
:102D100080007330714B00931B78C0B289F80000BB
:102D2000002B40F0E1836E4B03931B78002B40F0A7
:102D3000AE856C4B02931B78002B40F051866A4B9A
:102D40000193029B1B78002B3AD0684B1B88182BF1
:102D500017D099F800201344A3F118007F2840F3FE
:102D6000F285574A973B82FB0321DA17C2EB6102D7
:102D700002EB4202A3EB820303F17300C0B203F043
:102D80009BFF5B4A5B4B127833F81230182B17D03D
:102D900099F800201344A3F118007F2840F3DD8543
:102DA000474A973B82FB0321DA17C2EB610202EB31
:102DB0004202A3EB820303F17300C0B203F07CFF75
:102DC000009B1B78002B00F0AE84019B464E1988B7
:102DD000002900F0558538687F2840F35083384B30
:102DE0007F3883FB0032C317C3EB620303EB43035B
:102DF000A0EB830073303860002940F0E984009B29
:102E00001B78002B00F05F813B4E3378002B00F0E5
:102E10005A81DFF8FCA0DFF8F4804FF0000B0CE0E3
:102E200003F17300C0B298F8001003F01DFF33786F
:102E30000BF1010B5B4540F346813B685AF8040FE8
:102E40001F4A1844A0F17F0382FB0321DA17C2EB6B
:102E5000610202EB42027F28A3EB8203E0DCFDF774
:102E600011FCDFE7254B1960254B1B68A92202FBEB
:102E700003F3002BBCBF03F57F533F339B13543B3D
:102E8000194481F30C01282007F04AFFFFF7EEBA3E
:102E9000144E1C481149124A337003700B7003E43E
:102EA00093424FF0000B80F29C800123CDF800B0DC
:102EB000CDF814B00493FFF748BB00BFF49DFF1F8B
:102EC000ABAAAA2A949BFF1F789BFF1FDC9DFF1FC4
:102ED000809BFF1FCDCCCC3D0000FE42C69DFF1F56
:102EE000759BFF1F349CFF1FCC9BFF1FB09BFF1FD8
:102EF000DA9BFF1F8C9DFF1F8889FF1F9C9BFF1F74
:102F0000C089FF1F7C9DFF1F789DFF1F189CFF1F1E
:102F10006089FF1F924B1B78002B7FF46EAB039BE5
:102F2000904A243B83F34703D9B25B20136003F03C
:102F300073FE98F80060032E30D1DFF8808298F895
:102F40000030002B40F03686874F3B78002B40F056
:102F50002486834E3378002B40F01286834B1B78F7
:102F6000002B40F00086824A1380824B1B78002B96
:102F700040F0EC85804B7F221A8098F800306BB9C6
:102F80003B785BB933784BB97C4A7F2107201380AB
:102F900003F042FE7F210B2003F03EFE784B1F68BA
:102FA000FFF72BBB77480068D0F17F0048BF0330A4
:102FB00003EBA00301339942BFF686AC116053E7DF
:102FC000714B09881A6000297FF4CFAC13469842F0
:102FD000D4BFC2EB0003C2EB030376E5FDF752FB5F
:102FE00037E60123CDF810B0CDF800B00593FFF718
:102FF000ACBA01232B60654CFFF70ABA644B6A2018
:10300000198803F08DFF3B783370FFF701BA614BED
:103010001B78002B3AD0604B1B88182B17D099F8DF
:1030200000201344A3F118007F2840F3ED845B4A8D
:10303000973B82FB0321DA17C2EB610202EB4202EB
:10304000A3EB820303F17300C0B203F035FE544AD0
:10305000544B127833F81230182B17D099F80020FF
:103060001344A3F118007F2840F3D2844B4A973BC6
:1030700082FB0321DA17C2EB610202EB4202A3EBEF
:10308000820303F17300C0B203F016FE019B1B889C
:10309000002B00F08C84444B1B78002B40F0818483
:1030A000424B394A198826680020012310602B60A2
:1030B000B142364CBFF6ACA922683D4B0892089A43
:1030C0001A60FFF7A5B9039B1B78002B7AD03B68E9
:1030D000A3F10C007F2840F3F28330488B3B80FB48
:1030E0000320DA17C2EB600000EB4000A3EB800383
:1030F00003F17300DFF8C080C0B298F8001003F04D
:10310000B3FD009B1B78002B5CD02A4E3378002B3C
:1031100058D0DFF8ACA04FF0000B0BE003F17300C8
:10312000C0B298F8001003F09FFD33780BF1010B4B
:103130005B4547DD3B685AF8040F184A1844A0F174
:103140008B0382FB0321DA17C2EB61020C3802EB1E
:1031500042027F28A3EB8203E0DCFDF793FADFE76E
:10316000009EFF1FB49BFF1FFF9DFF1FFE9DFF1FC3
:103170002A9CFF1F019EFF1F949BFF1F709DFF1F36
:10318000889BFF1FCC9DFF1F789BFF1FEC9EFF1F9E
:10319000C09BFF1F349CFF1FB09BFF1FABAAAA2A36
:1031A000DA9BFF1F8C9DFF1F7C9DFF1F329CFF1F22
:1031B0008C9EFF1F8889FF1F189CFF1FFD9DFF1F0E
:1031C0006089FF1F029B1B78002B3AD0AD4B1A88F9
:1031D000182A18D03B681344A3F118007F2840F345
:1031E000B683A94A973B82FB0321DA17C2EB61023F
:1031F00002EB4202A3EB820303F17300A34BC0B2C4
:10320000197803F031FDA2490B78022B00F25383A9
:103210000133DBB20B701A469E4830F81260182E4C
:1032200040F090820422032B03F10106F3B208BFA1
:10323000002330F81360182E40F08382013AF2D157
:103240000B70019B1B88002B00F0CB82009B1B782E
:103250003BB9039B1B7823B9029B1B78002B00F022
:10326000E0838D4B1B78002B00F0D6808B490B78C8
:10327000082B00F2D1808A483A680068894E0133F1
:10328000DBB25F1E101A46F827000B70864B2668CB
:10329000198889F800200BE77F4B1B78002B40F042
:1032A000C1823B68814A1278002A45D0A3F10C0004
:1032B0007F2840F30A83744A8B3B82FB0321DA1791
:1032C000C2EB610202EB4202A3EB820303F1730043
:1032D000C0B298F8001003F0C7FC009B1B7853B3F2
:1032E0006E4E33783BB3DFF8FC91DFF89CA14FF0D2
:1032F000000B0BE003F17300C0B298F8001003F06C
:10330000B3FC33780BF1010B5B4514DD3B6859F8D6
:10331000040F1844A0F18B038AFB0321DA17C2EBD8
:1033200061020C3802EB42027F28A3EB8203E1DC4E
:10333000FDF7A8F9E0E73B685D4A1278002A3DD026
:10334000504A1288182A18D01344A3F118007F2875
:1033500040F30D834C4A973B82FB0321DA17C2EB03
:10336000610202EB4202A3EB820303F17300C0B2DD
:1033700098F8001003F078FC3B6845490A78022A67
:1033800000F2A6820132D2B20A701646414830F8E5
:1033900016E0BEF1180F40F0F0810426032A02F176
:1033A000010E5FFA8EF208BF002230F812E0BEF183
:1033B000180F40F0E181013EF0D10A70019A1288A5
:1033C000002A00F041823B4903220B702A60FFF77C
:1033D0001FB8394F3B78002B3FF476A9374E307831
:1033E00001F036F9364B1B78002B00F091823388C0
:1033F0007E2B00F28D82334A0133108899B23180DE
:10340000002800F09582C9B2C0B22F4E03F004FC30
:103410003B783370FEF7FCBF3A6837E7DBB21846FB
:10342000137003F0D7FB294B1B491A461F4B184654
:1034300000230B703B7013700370FFF757B8012324
:10344000FFF796B880262249224B234A09881B8819
:1034500012680B44B2EB630FBFF6CFA8164B1B7874
:10346000002B40F0FE81B9F800301C4AB3423FF413
:10347000C4A81B4B168001221A70FFF7BEB8FDF7D7
:1034800001F9B8E4B09BFF1FABAAAA2A189CFF1F42
:10349000DA9BFF1F8C9DFF1F7C9DFF1F8889FF1FEC
:1034A000989BFF1F6489FF1F329CFF1F759BFF1FA6
:1034B000349CFF1F789DFF1F969BFF1FC09BFF1F23
:1034C000029EFF1F049CFF1F929BFF1FC69DFF1FB4
:1034D000269DFF1F2C9DFF1FC49BFF1F489DFF1FA4
:1034E000979BFF1F6089FF1FC14B01931B88002B17
:1034F00040F06C83BF4B0393BF4B0293BF4E3378B6
:103500006BB3DFF81483DFF8F8A24FF0000B09E08B
:1035100003F17300C0B203F0CFFB33780BF1010B62
:103520005B451CDD58F8043F99F800001844A0F1F1
:103530007F038AFB0321DA17C2EB610202EB42022E
:103540007F28A3EB8203E3DCFDF79CF8E2E7AA4BBC
:10355000029303F0B1FB009B1B78002BCED1039BA1
:103560001B78002B3FF4EDAB99F80030A3F10C0071
:103570007F2840F3A781A2488B3B80FB0320DA170A
:10358000C2EB600000EB4000A3EB800303F173008B
:10359000C0B203F091FB009B1B78002B00F08081F0
:1035A000964E3378002B00F06582DFF86C82DFF8EE
:1035B00050A24FF0000B0AE003F17300C0B203F019
:1035C0007BFB33780BF1010B5B457FF7BAAB58F807
:1035D000043F99F800001844A0F18B038AFB0321F3
:1035E000DA17C2EB61020C3802EB42027F28A3EB30
:1035F0008203E1DCFDF746F8E0E75046FDF742F8CC
:10360000FFF788BBFDF73EF8FFF7C6B9002008704A
:103610007C49087840B17C4900910978002900F084
:10362000A981009F002139707849097800297FF429
:1036300020A8002E67D1002865D1754E724F96F8EC
:1036400000E06C4E03966C4E02966A4E71493070E3
:10365000694E0097087038703070BEF1000F7FF42B
:103660001AA8FFF721B8634B1B78002B3FF4CFACAF
:1036700099F80030A3F10C007F2840F3C281604A22
:103680008B3B82FB0321DA17C2EB610202EB4202A1
:10369000A3EB820303F17300C0B203F00DFB009BA8
:1036A0001B78002B3FF4B3AC544E3378002B3FF41F
:1036B000AEAC594FDFF848814FF0000A0AE003F141
:1036C0007300C0B203F0F8FA33780AF1010A5345E7
:1036D0007FF79DAC57F8043F99F800001844A0F11B
:1036E0008B0388FB0321DA17C2EB61020C3802EB73
:1036F00042027F28A3EB8203E1DCFCF7C3FFE0E793
:103700000398002101704249097800293EF4CCAFAA
:10371000394902910978002900F088810298002136
:103720000170FEF7C1BF039B1B78002B7FF44DABEC
:10373000029B1B78002B7FF448AB019B1988FFF795
:103740004ABB0B703B681E44A6F118007F2840F36B
:1037500001812B4B973E83FB0632F317C3EB6203C9
:1037600003EB4303A6EB830606F173002B4BC0B2B9
:10377000197803F079FA64E50A707344A3F118002C
:103780007F2840F3F1801E4A973B82FB0321DA1722
:10379000C2EB610202EB4202A3EB820303F173006E
:1037A000C0B298F8001003F05FFA3B6806E6243BCD
:1037B000002BB9F8000040F32F8198423EF4F5AE9B
:1037C0009BB21748A9F8003001230370FEF7EDBE45
:1037D000DFF84880C0B298F8001003F045FAFFF710
:1037E0000EBB0E4B3878197803F03EFA2EE500BF79
:1037F000CC9BFF1F759BFF1F349CFF1F8889FF1FF9
:10380000ABAAAA2A019EFF1FC69DFF1FFD9DFF1F99
:10381000969BFF1F7C9DFF1F6089FF1F189CFF1F49
:10382000979BFF1F7F21402003F0F6F9B349B44A6C
:103830003B680B600021117034E5C0B298F80010AD
:1038400003F012FAFFF7AFB8D8B298F8001003F0FF
:103850000BFA3B68B7E5AB4BDFF8ECE21978FEF703
:10386000A4BE4B2E40F3A9801836802EB9F8003044
:10387000A54AA8BF8026B3427FF4FBADFEF7BDBECC
:1038800099F8000003F018FA3188FFF7A4BA9F4BAB
:1038900001931B88002B7FF45AAE9D4B029363E685
:1038A000029B1B78002B7FF450AA039B1B78002BF4
:1038B0007FF48BAA41E7002213460A70ACE4FCF7C0
:1038C000E1FE17E4FCF7DEFE62E6FCF7DBFEFFE458
:1038D000002216460A7059E5FCF7D4FEFFF74DB9F1
:1038E0008C4E307800F0B4FE8B4B1B781BB13388C4
:1038F0007E2B40F2A780894B1B7823B13388854A01
:10390000002B40F0AB80864E3B783370FEF780BDD5
:10391000824B1B78002BF6D033887E4A002BF2D0E6
:103920008049013B088899B2118000287FF46BAD73
:10393000C8B27B4E03F0E4F93B783370FEF768BD04
:103940007F20FFF7D1B9FCF79DFEFFF717BAFCF710
:1039500099FE53E4FCF796FE08E7FCF793FEFFF7A9
:103960002CBA7F20FFF7E5B8FCF78CFE18E7FCF7D0
:1039700089FEFCE4664F6C4902974FF0000C81F819
:1039800000C0009F02994FF0010E87F800E081F817
:1039900000C049E60120FFF7A7B903F08DF9FFF752
:1039A000F5B80021402003F037F9FFF779BB99F80B
:1039B000000003F081F9FFF76EBB243E002EB9F83A
:1039C00000303ADDB3423EF418AEB6B2574BA9F818
:1039D000006001221A70FEF710BE0120FFF7A9B89F
:1039E0004A4B01931B88002B7FF4B3ADFFF7A9B9B5
:1039F0004F4A8342A8BF03461360FEF7B6BF164680
:103A00002CE5FCF73FFE47E6FCF73CFEFFF71CBB4E
:103A1000FCF738FEFFF737BB01283EF4C6AD0123A3
:103A2000CFE699F8000003F047F91AE44148009006
:103A300041483D490390FEF72EBE012B3EF4DDAD1B
:103A40000126C3E701339BB23380D9B20520344E3F
:103A500003F0E2F83B783370FEF7DABC013B9BB22F
:103A6000D9B205202E4E138003F0D6F83B78337080
:103A7000FEF7CEBC029B1B78002B7FF466A9FFF7F4
:103A8000A4B92E4B1B782BB32D4B1B78002B7EF447
:103A9000B4AD2C4B1B78002B3EF4AFADB9F8003021
:103AA00022490A33A9F800300A70FEF7A6BD244B5C
:103AB0001B78002B7EF4A1AD224B1B78002B3EF42B
:103AC0009CADB9F800301949013BA9F800300A70E3
:103AD000FEF793BD1A4B1B78002B7FF41BAA194BE2
:103AE0001B78002B3EF489ADB9F800300F49013343
:103AF000A9F800300A70FEF780BD00BF989BFF1F39
:103B00008889FF1FE99DFF1F489DFF1FCC9BFF1F5A
:103B1000349CFF1FC09BFF1F029EFF1F019EFF1FC3
:103B2000929BFF1F049CFF1F7C9DFF1F979BFF1F05
:103B3000789BFF1FC69DFF1F759BFF1FFE9DFF1FEC
:103B4000FF9DFF1F009EFF1FE19BFF1F224B0022D6
:103B50007F2107201A8003F05FF87F210B2003F0FC
:103B60005BF8FFF70ABA1D4B01227F2107201A805C
:103B700003F052F87F210B2003F04EF8FFF7F5B960
:103B8000174B04227F2107201A8003F045F80021FB
:103B90000B2003F041F8FFF7E1B9114B02227F211E
:103BA00007201A8003F038F87F210B2003F034F847
:103BB000FFF7CFB90A4B002107201E8003F02CF835
:103BC0007F210B2003F028F8FFF7BEB9054B0393C4
:103BD000054B0293BDE400BF949BFF1F2A9CFF1F6F
:103BE000709DFF1F759BFF1F349CFF1F38B506F0AB
:103BF000ADFD0E4804F0E4FC0D4804F0E1FC0D4876
:103C000004F0DEFC00234FF07E5201210A48FCF74D
:103C10002DFC0A4B0A4A0B49802400251C711846CA
:103C20001D60BDE838400AF055BA00BFA89BFF1FD1
:103C3000D49BFF1F309CFF1F4C9DFF1FD09DFF1F7B
:103C40001C89FF1F2906000043682A20198803F0F9
:103C500067B900BF10B5044622206368198803F0D5
:103C60005FF9E36824201988BDE8104003F058B9D3
:103C700010B504460A206368198803F051F9E36817
:103C80000C201988BDE8104003F04AB910B504466D
:103C900006206368198803F043F9E368082019884F
:103CA000BDE8104003F03CB910B50446022063683B
:103CB000198803F035F9E36804201988BDE810403D
:103CC00003F02EB970B50E4C84B0122504220123E6
:103CD00006460390029320468DE824001423102109
:103CE00005F072FE062209230293039601952046F1
:103CF00000921423102105F067FE04B070BD00BFD0
:103D0000289EFF1F2DE9F041224D82B0012602B20C
:103D100084B20092284601967823192105F09AFD75
:103D200004F10C0212B28DE844002846A71978234A
:103D3000192104F1020805F08DFD3FB20FFA88F851
:103D400019233A46284619460196CDF8008005F019
:103D500081FD78233A4628461946CDF80080019621
:103D600004F10A070B3405F075FD3FB224B2782345
:103D70003A46284619468DE8500005F06BFD192398
:103D800000943A4601962846194605F063FD02B0B4
:103D9000BDE8F081289EFF1F2DE9F0411E4682B04C
:103DA0001446002A6AD0099B4D4A00EBC305012C3A
:103DB0006F8929896868A7EB010382FB03E21A4433
:103DC0004FEAE373C3EBA21302887BD0042C38D1F3
:103DD00012FA83F3994203DC9F423946A8BF194681
:103DE000089A0180B6F90030BDF920803D48971D42
:103DF0004FF0000E3FB2194642460097CDF804E05E
:103E000005F028FD29896A896B68521A1B885C2A8B
:103E1000A3EB010359DD03EB43030132C3EB43136F
:103E200093FBF2F303F11B0213B201203280194617
:103E30004246019000972B4805F00CFD2A4B0022CA
:103E40001A702A4B022CB3F9001045D0082C31D13E
:103E500000221A8091422DD0089AB6F900302148EC
:103E60000632012412B2009219460194BDF92020B5
:103E700005F0F0FC204602B0BDE8F0811C4D1D4A63
:103E80002B681268CB1A93420F4617D9164A33880B
:103E900011781448012918BF01241470089A0632B9
:103EA0001BB212B28DE814001946BDF9202005F0AE
:103EB000D1FC2F60012002B0BDE8F081204602B0A5
:103EC000BDE8F0819BB2D31A84E75C2101FB03F3C8
:103ED00093FBF2F21B32A7E74A1C12B21A80B9E731
:103EE000C94216B2289EFF1FAE9EFF1F109EFF1FE5
:103EF0008C9EFF1FD400010030B583B000230C4618
:103F000005B2009326225B231C210C4805F0F2F930
:103F1000294601232622094804F0FCFC002C24B287
:103F200005DB214601232622044804F0F3FC044A61
:103F3000044B15801C8003B030BD00BF289EFF1FBE
:103F4000628AFF1F648AFF1FF0B59B4C237883B001
:103F50001BB19A4B4FF6FF721A80994BB3F90030A0
:103F6000C3B9984A954B1068B3F9002080F30C0050
:103F70005B2303FB00F000131C3082425ED04FF045
:103F8000FF31FFF7B9FF904805F018FA00232370BE
:103F900003B0F0BD012B36D0022B6ED0032B53D0D3
:103FA000042BF3D1252200258DE8240076231C2143
:103FB0008548864E864F05F04DFC17E0B0F5AF7F83
:103FC000A8BF4FF4AF70323803FB00F387FB032127
:103FD000DB17C3EB61111C3109B201231D442522FB
:103FE000794804F097FC0C2D00F08480E9B2794800
:103FF00004F04EFB56F8042B801A31284FF05B0377
:10400000DCDC1C21E9E7744B1A68B2F52F7F32DB48
:1040100041F25C239342A8BF1346A3F52F735B22A2
:104020006E4802FB03F380FB0320DB17C3EBA020E9
:104030001C30624BB3F900308342A0D1684BB3F916
:10404000003001339BD1A1E7664B1B68B3F5FA7FC3
:1040500011DBB3F57A6FA8BF4FF47A63A3F5FA7258
:1040600061485B2303FB02F380FB0320DB17C3EBF8
:1040700020201C30DDE71C20DBE75C4B1B68B3F520
:10408000FA7F33DBB3F57A6FA8BF4FF47A63A3F5F9
:10409000FA7255485B2303FB02F380FB0320DB1716
:1040A000C3EB20201C30524B1B68B3F5FA7F1FDB9B
:1040B000B3F57A6FA8BF4FF47A63A3F5FA724A4951
:1040C0005B2303FB02F381FB0321DB17C3EB2121FD
:1040D0001C313A4BB3F9003083427FF452AF404B6E
:1040E000B3F900308B427FF44CAF4FE71C20DAE786
:1040F0001C21EEE7262200258DE8240076231C21D2
:1041000031483C4E324F05F0A5FB16E0B0F5AF7FCD
:10411000A8BF4FF4AF70323803FB00F387FB0321D5
:10412000DB17C3EB61111C3109B201231D442622A8
:10413000254804F0EFFB0C2D0CD0E9B22E4804F01A
:10414000A7FA56F8042B801A31284FF05B03DDDC08
:104150001C21EAE7272200258DE8240076231C2174
:104160001948264E1A4F05F075FB17E0B0F5AF7FE2
:10417000A8BF4FF4AF70323803FB00F387FB032175
:10418000DB17C3EB61111C3109B201231D44272247
:104190000D4804F0BFFB062D3FF4F5AEE9B2184818
:1041A00004F076FA56F8042B801A31284FF05B039E
:1041B000DCDC1C21E9E700BF069EFF1F628AFF1FAF
:1041C0000C9EFF1F809DFF1F289EFF1F188AFF1F48
:1041D0004B48371BD49BFF1F849BFF1FD305854192
:1041E000648AFF1FC49BFF1F011FB812D09BFF1FD3
:1041F000F89DFF1F3089FF1F309CFF1F488AFF1F5B
:10420000A89BFF1F2DE9F04FDFF8EC82B74CB8F9FF
:1042100000604D7854F8264087B08246039305B17C
:104220000D78DFF8FCB2002A34D19BF800308BBB4C
:10423000AF4EB6F90000002800F0CE80012800F053
:104240002481012032232A46019000935146A94B34
:104250002046FFF7A1FD00250746B6F90030022BE6
:1042600040F3F48000233380B8F90030A24A002BD9
:10427000C0F2F880042BC4BF00231380039B002BE3
:1042800040F0F680002D0CBF38464FF0FF3007B0ED
:10429000BDE8F08F964EE3682268984804930027A3
:1042A000059237808BF8007004F07CFF1120FFF737
:1042B00029FD4FF0010919232821CDF80490009120
:1042C000242219468D4805F0C5FA78232821242296
:1042D000CDF8049000918948194605F0BBFA49468B
:1042E000864805F04DFE02221921844805F044FE5F
:1042F000DDF8149048460AF0C3FC494602467F4860
:1043000005F0D4FF7D4805F0E7FF394614227B48CD
:1043100005F032FE03227A49784805F0C7FF774856
:1043200005F0DAFF39462322744805F025FE032202
:104330007449724805F0BAFF704805F0CDFF049B40
:10434000002B72D10123704A18461370FFF7BAFC94
:10435000208963896768191A5C293A885BDC131A1B
:104360005C2202FB03F292FBF1F31B33674A6348C2
:10437000138001271BB21A2219468DE884001422EB
:1043800005F068FA049BDBB1218A638AE768581A52
:104390005C283A886FDD521A02EB4202C2EB4212ED
:1043A000431C92FBF3F31B33524A544813800127FA
:1043B00038221BB28DE884001946322205F04AFAF1
:1043C000534A544BB6F90000012111704FF6FF72A9
:1043D0001A8000287FF432AFDFF848914E4AD9F8AE
:1043E00000301268C3EB0A0393424CD9464B1A784B
:1043F000012A18BF012018700127FFF763FCC9F8D4
:1044000000A0012D4ED0042D59D0022D60D0082DD2
:1044100064D0002521E7121A02EB4202C2EB4212DD
:104420004B1C92FBF3F31B33A0E72F20FFF76AFC32
:1044300039463222314805F09FFD032237492F4883
:1044400005F034FF2D4805F047FF7BE77FF40CAF04
:10445000E368002B3FF406AFB8F90030264A002B82
:10446000BFF608AF04231380039B002B3FF40AAF71
:10447000FFF76AFD06E7511A5C2202FB01F292FB8C
:10448000F0F31B3390E70746BBE7002714238DE8C2
:1044900088002A4651461D4B2046FFF77DFC3D46CD
:1044A0000746DAE6B8F800308BF800500133A8F878
:1044B0000030636983B1002520469847CDE6B8F8FF
:1044C00000300122013BA8F800308BF80020F0E713
:1044D000012333800025C7E61D46BEE6636900223E
:1044E00032804FF0FF35002BE6D1BDE6688AFF1F12
:1044F000109EFF1F0A9EFF1F0C9EFF1F289EFF1F7E
:104500007CF5000080F50000AE9EFF1F089EFF1F97
:10451000069EFF1F628AFF1FD400010084F5000081
:104520000E9EFF1F8C9EFF1F01210D2006F088BDEF
:1045300000210D2006F084BD01460D2006F080BD4F
:1045400008B50D2006F082FDB0FA80F149090D2072
:10455000BDE8084006F074BD10B5002144080D20E8
:1045600006F06EFD204606F0A7FD0D20012106F0A5
:1045700067FD2046BDE8104006F09EBD2D4A2E4B3B
:1045800010881B68984210B549DA2C4A1288141A10
:104590009A42A8BF1A46B4F5157F36DA121A40F2CD
:1045A000532303FB02F393FBF4F105310A2006F0D9
:1045B000B7FB234B1978C9B3224B23491B6840F240
:1045C000271283F3070302FB03F381FB0321194442
:1045D000DB17C3EBA1110531092006F0A1FB1B4B32
:1045E0001968F1B181F3070140F22712164802FB66
:1045F00001F380FB03211944DB17C3EBA111053143
:104600001620BDE8104006F08BBB131A4FF415724C
:10461000611C02FB03F393FBF1F10531C6E70021B6
:10462000C4E71620BDE8104006F07ABB092006F06A
:1046300077FBD4E7329CFF1F789BFF1FDC9DFF1F99
:10464000EF9BFF1FCC9DFF1F09040281989DFF1F58
:104650007F2838B5A8BF7F200F4C4FF4167202FB9D
:1046600000F284FB02311144D2170546C2EBA111BE
:104670000A2006F055FB7F3D4FF4967303FB05F3CC
:1046800084FB03211944DB17A3EBA1110920BDE82A
:10469000384006F045BB00BF09040281024B4E20A2
:1046A000198802F03DBC00BFCC9BFF1F024B442089
:1046B000198802F035BC00BFB09BFF1F024B1020D1
:1046C000198802F02DBC00BF349DFF1F024B2C2027
:1046D000198802F025BC00BFA49BFF1F024B1E20BF
:1046E000198802F01DBC00BFA09BFF1FC3680E20ED
:1046F000198802F015BC00BF024B2820198802F06F
:104700000FBC00BF889DFF1F024B6420198802F078
:1047100007BC00BF849DFF1F024B5A20198802F07E
:10472000FFBB00BF8C9BFF1F024B1620198802F0B5
:10473000F7BB00BF949BFF1F024B2E20198802F08D
:10474000EFBB00BF249CFF1F024B3020198802F0F2
:10475000E7BB00BF809BFF1F024B1820198802F0A7
:10476000DFBB00BF369CFF1F024B1A20198802F0E6
:10477000D7BB00BFD69BFF1F024B1C20198802F03D
:10478000CFBB00BFCE9BFF1F024B6620198802F0F3
:10479000C7BB00BFC49DFF1F024B7220198802F0E7
:1047A000BFBB00BFE09DFF1F024B2020198802F015
:1047B000B7BB00BFC29DFF1F024B3220198802F019
:1047C000AFBB00BFB29DFF1F024B6820198802F0EB
:1047D000A7BB00BF049CFF1F024B6C20198802F08E
:1047E0009FBB00BF7C9BFF1F024B6E20198802F00D
:1047F00097BB00BF049EFF1F024B5220198802F096
:104800008FBB00BF6089FF1F024B5020198802F048
:1048100087BB00BF108AFF1F024B5420198802F08B
:104820007FBB00BF128AFF1F024B5C20198802F079
:1048300077BB00BF608AFF1F024B5E20198802F021
:104840006FBB00BF2C89FF1F024B6020198802F04C
:1048500067BB00BF229DFF1F024B5620198802F044
:104860005FBB00BF169CFF1F38B5094D462420468C
:1048700002F070FB35F8021B00B28842204601D0DE
:1048800002F04EFB0234A4B24E2CF0D138BD00BF72
:104890008C9DFF1F064B074A10B41C88064B084628
:1048A000002C14BF11461946042210BC0AF0A6BA07
:1048B000E89BFF1F80FC000084FC0000064B074AB9
:1048C00010B41C88064B0846002C14BF114619462C
:1048D000042210BC0AF092BA269CFF1F80FC000044
:1048E00084FC0000064B074A10B41C88064B08469F
:1048F000002C14BF11461946042210BC0AF07EBADF
:10490000869DFF1F80FC000084FC0000064B074AC8
:1049100010B41C88064B0846002C14BF11461946DB
:10492000042210BC0AF06ABA7A9DFF1F80FC0000C6
:1049300084FC0000064B074A10B41C88064B08464E
:10494000002C14BF11461946042210BC0AF056BAB6
:104950002A9CFF1F80FC000084FC0000F0B52B4E59
:104960002B4FDFF8C4E005460FCE87B06C460FC46E
:1049700096E803003B68274A274F44F8040B40F6AB
:10498000CC308342C8BF3A46BEF800602180012E79
:1049900011889278ADF80D108DF80F202AD032D3FF
:1049A00040F6CA02022E18BF00229A4226DCA3F665
:1049B00098031A491A4AC3EB031381FB03011944F4
:1049C000DB17C3EB6123243382FB0321DA17C2EB2D
:1049D000A10202EB8201A3EB4103303330328DF8A8
:1049E00013308DF811206946284616220AF006FA7F
:1049F00007B0F0BD40F698029A42D8DD094B18681E
:104A0000CDF81100EFE740F6FC02CEE798FC00007D
:104A10009C9DFF1F8CFC000088FC00003B773B98AE
:104A20006766666690FC0000169DFF1FF8B5174C80
:104A3000174E2278174D33782F888E46003218BFD4
:104A4000012201467046FFF7DDFB002398423370D8
:104A5000237015DB14BF012000202B889F420ED04D
:104A600040F23A72A3F5AF730B490C4C02FB03F30F
:104A700081FB0312DB17A3EB621332332360F8BD13
:104A80000749012218460A702270E6E70C8BFF1FC7
:104A9000219EFF1FD89DFF1FB5814E1B008AFF1F5F
:104AA000A49EFF1F014B187802F0D2B9889EFF1F09
:104AB000014B187802F0E6B92090FF1F134BB3F9B1
:104AC000003030B583EAE374A4EBE374002BA0B2AA
:104AD00018DB012300E0134603EB830252009442EB
:104AE000F9DA0B4D90FBF3F285FB03E403FB1200B4
:104AF000DB173032D3EBA40380B201F8012BF1D1E4
:104B00000B7030BD2D230B700131E2E72090FF1FA9
:104B100067666666144BB3F9003070B583EAE375D7
:104B2000A5EBE375002BACB21ADB012300E00346D2
:104B300003EB830040008542F9DA0C4E94FBF3F05E
:104B400086FB03E503FB1044DB173030D3EBA503F2
:104B5000A4B201F8010BF1D105480B70106070BDD3
:104B60002D230B700131E0E78C9BFF1F67666666A3
:104B7000B0FC0000134BB3F9003030B583EAE374A6
:104B8000A4EBE374002BA0B218DB012300E0134672
:104B900003EB830252009442F9DA0B4D90FBF3F2DF
:104BA00085FB03E403FB1200DB173032D3EBA403D5
:104BB00080B201F8012BF1D10B7030BD2D230B70A9
:104BC0000131E2E76089FF1F67666666134BB3F940
:104BD000003030B583EAE374A4EBE374002BA0B299
:104BE00018DB012300E0134603EB830252009442DA
:104BF000F9DA0B4D90FBF3F285FB03E403FB1200A3
:104C0000DB173032D3EBA40380B201F8012BF1D1D2
:104C10000B7030BD2D230B700131E2E7108AFF1FAE
:104C200067666666134BB3F9003030B583EAE37408
:104C3000A4EBE374002BA0B218DB012300E01346C1
:104C400003EB830252009442F9DA0B4D90FBF3F22E
:104C500085FB03E403FB1200DB173032D3EBA40324
:104C600080B201F8012BF1D10B7030BD2D230B70F8
:104C70000131E2E7128AFF1F67666666134BB3F9DC
:104C8000003030B583EAE374A4EBE374002BA0B2E8
:104C900018DB012300E0134603EB83025200944229
:104CA000F9DA0B4D90FBF3F285FB03E403FB1200F2
:104CB000DB173032D3EBA40380B201F8012BF1D122
:104CC0000B7030BD2D230B700131E2E7608AFF1FAE
:104CD00067666666134BB3F9003030B583EAE37458
:104CE000A4EBE374002BA0B218DB012300E0134611
:104CF00003EB830252009442F9DA0B4D90FBF3F27E
:104D000085FB03E403FB1200DB173032D3EBA40373
:104D100080B201F8012BF1D10B7030BD2D230B7047
:104D20000131E2E72C89FF1F67666666054B1B8829
:104D30001BB9054B186808607047044B1868086079
:104D4000704700BFCC9BFF1FB8FC0000B4FC000004
:104D5000164B1B880BB31BB230B583EAE374A4EB8C
:104D6000E374002BA0B21CDB012300E0134603EB2D
:104D7000830252009442F9DA0D4D90FBF3F285FB69
:104D800003E403FB1200DB173032D3EBA40380B241
:104D900001F8012BF1D10B7030BD064B186808608B
:104DA00070472D230B700131DEE700BFA09BFF1F72
:104DB0006766666684FC0000164B1B880BB31BB24B
:104DC00030B583EAE374A4EBE374002BA0B21CDBE0
:104DD000012300E0134603EB830252009442F9DA08
:104DE0000D4D90FBF3F285FB03E403FB1200DB1790
:104DF0003032D3EBA40380B201F8012BF1D10B7058
:104E000030BD064B1868086070472D230B700131C8
:104E1000DEE700BFB69DFF1F6766666684FC000084
:104E2000164B1B880BB31BB230B583EAE374A4EBBB
:104E3000E374002BA0B21CDB012300E0134603EB5C
:104E4000830252009442F9DA0D4D90FBF3F285FB98
:104E500003E403FB1200DB173032D3EBA40380B270
:104E600001F8012BF1D10B7030BD064B18680860BA
:104E700070472D230B700131DEE700BF949BFF1FAD
:104E800067666666BCFC0000174B1B881BB31BB231
:104E900070B583EAE375A5EBE375002BACB21EDBBE
:104EA000012300E0034603EB830040008542F9DA6A
:104EB0000E4E94FBF3F086FB03E503FB1044DB1777
:104EC0003030D3EBA503A4B201F8010BF1D10848AF
:104ED0000B70106070BD074B1868086070472D2379
:104EE0000B700131DCE700BF249CFF1F676666661C
:104EF00094FC000084FC0000164B1B880BB31BB213
:104F000030B583EAE374A4EBE374002BA0B21CDB9E
:104F1000012300E0134603EB830252009442F9DAC6
:104F20000D4D90FBF3F285FB03E403FB1200DB174E
:104F30003032D3EBA40380B201F8012BF1D10B7016
:104F400030BD064B1868086070472D230B70013187
:104F5000DEE700BF809BFF1F6766666684FC00007B
:104F6000164B1B880BB31BB230B583EAE374A4EB7A
:104F7000E374002BA0B21CDB012300E0134603EB1B
:104F8000830252009442F9DA0D4D90FBF3F285FB57
:104F900003E403FB1200DB173032D3EBA40380B22F
:104FA00001F8012BF1D10B7030BD064B1868086079
:104FB00070472D230B700131DEE700BFC49DFF1F3A
:104FC0006766666684FC0000164B1B880BB31BB239
:104FD00030B583EAE374A4EBE374002BA0B21CDBCE
:104FE000012300E0134603EB830252009442F9DAF6
:104FF0000D4D90FBF3F285FB03E403FB1200DB177E
:105000003032D3EBA40380B201F8012BF1D10B7045
:1050100030BD064B1868086070472D230B700131B6
:10502000DEE700BFE09DFF1F6766666684FC000048
:10503000174B1B881BB31BB270B583EAE375A5EB56
:10504000E375002BACB21EDB012300E0034603EB4B
:10505000830040008542F9DA0E4E94FBF3F086FBA4
:1050600003E503FB1044DB173030D3EBA503A4B2F8
:1050700001F8010BF1D108480B70106070BD074BAF
:105080001868086070472D230B700131DCE700BF02
:10509000C29DFF1F67666666C0FC000084FC0000BE
:1050A000074B1B88022B06D0012B0CBF054B064B70
:1050B000186808607047054B18680860704700BFA3
:1050C000229DFF1FC8FC0000CCFC0000C4FC0000B7
:1050D000054B1B881BB1054B186808607047044BD3
:1050E00018680860704700BF169CFF1FD4FC0000C2
:1050F000D0FC000008B5702001F02CFF044B19888B
:10510000884204D07020BDE8084001F009BF08BD06
:10511000169DFF1F08B5742001F01CFF044B198871
:10512000884204D07420BDE8084001F0F9BE08BDF3
:10513000A89DFF1F38B5FCF789FC0D4B1B7833B9D0
:105140000C4B1020198801F0EBFE012038BD0A4DF0
:105150000A4C2B782288B3FA83F382F008025B09A9
:10516000114642202B70228001F0DAFE002038BD6B
:10517000969BFF1F349DFF1F1A9DFF1FDE9DFF1F83
:10518000184B1A8852B3184A128830B50A80B3F9FE
:105190000030002B83EAE374A4EBE374BCBF2D233F
:1051A0008B70A0B2ACBF02310331012300E0134683
:1051B00003EB830252009442F9DA0C4D90FBF3F2B8
:1051C00085FB03E403FB1200DB173032D3EBA403AF
:1051D00080B201F8012BF1D10B7030BD044B18687F
:1051E00008607047D69BFF1FD8FC000067666666A4
:1051F00084FC000010B40A4B0A4C0A4693E80300F2
:1052000083B0238802AC04E9030004EB8303104657
:1052100053F8081C052203B010BC09F0EFBD00BF15
:105220000CF60000849DFF1F30B40A4B0A4D0C465B
:1052300093E8070084B02B8804AD05E9070005EB6F
:105240008303204653F80C1C042204B030BC09F040
:10525000D5BD00BF14F60000169DFF1FF0B40C4D25
:105260000C4F0E460FCD8CB001AC0FC40FCD0FC448
:1052700095E807003B8884E807000CAA02EB83034B
:10528000304653F82C1C04220CB0F0BC09F0B6BD1B
:1052900020F60000709DFF1FF0B40A4D0A4F0E4625
:1052A0000FCD86B001AC0FC42A683B88226006AAE5
:1052B00002EB8303304653F8141C042206B0F0BC02
:1052C00009F09CBD4CF60000369CFF1FF0B40A4D5F
:1052D0000A4F0E460FCD86B001AC0FC42A683B883A
:1052E000226006AA02EB8303304653F8141C0C22FA
:1052F00006B0F0BC09F082BD60F60000CE9BFF1F37
:10530000F0B40A4D0A4F0E460FCD86B001AC0FC463
:105310002A683B88226006AA02EB8303304653F8D2
:10532000141C042206B0F0BC09F068BD74F600003D
:10533000A89DFF1F164B1B880BB31BB283EAE370BB
:10534000A0EBE370002B30B584B21DDB012300E03D
:10535000134603EB830252009042F9DA0D4894FBA6
:10536000F3F280FB03E503FB1244DB173032D3EB8F
:10537000A503A4B201F8012BF1D10B7030BD084692
:105380000422054909F03ABD2D230B700131DDE7F8
:10539000049CFF1F67666666DCFC0000F0B40A4DE3
:1053A0000A4F0E460FCD86B001AC0FC42A683B8869
:1053B000226006AA02EB8303304653F8141C042231
:1053C00006B0F0BC09F01ABD88F600007C9BFF1FF8
:1053D00070B53C4D2B780646002B35D11C467378B2
:1053E0000BB9204670BDFCF731FB374A374B3848C4
:1053F000127831781B78007802EB43034A1E03EBE6
:1054000080030E2AEDD801A050F822F07554000058
:1054100097540000E353000075540000E35300006C
:10542000E3530000E353000063540000E353000023
:10543000E3530000E3530000E3530000E353000094
:10544000E35300005F540000AE21224803F05AFCF1
:10545000204803F0A7FE00232B700124BFE706F0CD
:105460003DF9AF211B4803F04DFC1B4A012313708B
:105470002B70B6E783B91948038804294FF6FF71EA
:1054800003F1FF320CBF01230B46134403F07F03EB
:10549000013303800FE073B1013B114A32F813303E
:1054A0004BB10E4E0F481049104A3380012300269D
:1054B00006700B701370084A0221012311702B70C3
:1054C000204670BD0C8BFF1FC79DFF1FC09DFF1F97
:1054D000C89DFF1F289EFF1FA49EFF1F489DFF1F02
:1054E000089DFF1FFC9BFF1F979BFF1FB09EFF1F88
:1054F00010B5064B064C1A882046012101F0FEFC2F
:1055000021884220BDE8104001F00ABDE89BFF1F42
:10551000DE9DFF1F10B5064B064C1A88204602215F
:1055200001F0ECFC21884220BDE8104001F0F8BCFD
:10553000269CFF1FDE9DFF1F10B5064B064C1A88E8
:105540002046052101F0DAFC21884220BDE8104008
:1055500001F0E6BC869DFF1FDE9DFF1F10B5064BC8
:10556000064C1A882046002101F0C8FC2188422000
:10557000BDE8104001F0D4BC7A9DFF1FDE9DFF1FE7
:1055800008B5122001F0E6FC054B1988884206D0C8
:10559000122001F0C5FCBDE8084001F0D9BB08BDF0
:1055A000709DFF1F08B5582001F0D4FC054B1988E9
:1055B000884206D0582001F0B3FCBDE8084001F055
:1055C000C7BB08BDB69DFF1F08B5142001F0C2FC83
:1055D000054B1988884206D0142001F0A1FCBDE8D3
:1055E000084001F0B5BB08BD2A9CFF1FF0B480EA5B
:1055F000E075A5EBE0750028ACB21FDB1DBF2B23C7
:105600000B704E1C0E46012300E0134603EB830291
:1056100052009542F9DA0B4F94FBF3F287FB030536
:1056200003FB1244DB173032D3EBA503A4B206F818
:10563000012BF1D133700846F0BC70472D230B705D
:105640004E1CE0E767666666084B188828B10D288F
:1056500007D00D3800B2FFF7C9BF054A10680860CF
:105660007047044A10680860704700BF049EFF1F1F
:1056700084FC0000E0FC0000174B18880C2813D0B5
:10568000192815D01A2817D01B2819D01C281BD070
:105690001D281DD01E2803D00C3800B2FFF7A6BF6E
:1056A0000E4A1068086070470D4A1068086070471D
:1056B0000C4A1068086070470B4A10680860704711
:1056C0000A4A106808607047094A10680860704705
:1056D000084A106808607047B29DFF1FFCFC00007C
:1056E000E4FC0000E8FC0000ECFC0000F0FC000022
:1056F000F4FC0000F8FC0000034B1888A0EB8000CD
:10570000400000B2FFF772BF889EFF1F024B18884F
:10571000033800B2FFF76ABF889DFF1F024B18884D
:105720000C3800B2FFF762BF909BFF1F024B188836
:10573000183800B2FFF75ABFB09BFF1FC368188824
:10574000183800B2FFF752BF30B5134C85B00125B1
:105750002B463C2202212046009503F049FB2046BF
:1057600003F020FD00224021802320460191009378
:1057700011460A4B029504F0C3F9204603F01EFEC1
:1057800007480849084A0023036083800B608B8028
:105790001360938005B030BD289EFF1F28F80000DD
:1057A000149EFF1FA89EFF1F949EFF1F10B500EBC5
:1057B000C00000F10F02D2B293B284B09C1E981CBC
:1057C0003D2303918DE819003921024804F0FCF8CB
:1057D00004B010BD289EFF1F014B01221A707047B4
:1057E000219EFF1FF0B585B0634C644B0293644A61
:1057F000019204230093634E634B644F644D204633
:105800004022802103F0FCF82046624A6249634C42
:1058100008F060FCB761624FF761624FAF61624FA1
:10582000EF61624FA7616248624FE761624F876133
:105830006249634FC761634F8F61634A634FCF61B2
:10584000634F9761634B644FD761644F9F61644EB0
:10585000644FDF61644FB761644D654FF761654F19
:10586000AF61654C654FEF61654F6648A761664F54
:10587000E761664F66498761664FC761664F674A51
:105880008F61674FCF61674F674B9761674FD761F4
:10589000674F684E9F61684FDF61684F684DB76121
:1058A000684FF761684F694CAF61694FEF61694FAD
:1058B000A7616948694FE761694F876169496A4F24
:1058C000C7616A4F8F616A4A6A4FCF616A4F9761B9
:1058D0006A4B6B4FD7616B4F9F616B4E6B4FDF61B4
:1058E0006B4FB7616B4D6C4FF7616C4FAF616C4C98
:1058F0006C4FEF616C4FA7616C486D4FE7616D4F66
:1059000087616D496D4FC7616D4F8F616D4A6E4FF5
:10591000CF616E4F6E4B97616E4FD7616E4F6F4E7A
:105920009F616F4FDF616F4F6F4DB7616F4FF761D1
:105930006F4F704CAF61704F70487149EF61714F9C
:10594000714DA761E561714F714D724CDFF8E8E16F
:10595000714A724B8761C5618C61714EC1F81CE060
:10596000704F714D714C724872499761D5619C615D
:10597000D861B16005B0F0BD289EFF1FA086010070
:10598000801A0600708DFF1F6090FF1F1D570000DA
:10599000A48EFF1F1C89FF1F598A0000148EFF1F51
:1059A000ED4600000D570000F94600009548000044
:1059B000508CFF1FF1540000BD480000048DFF1FF4
:1059C00015550000E54800002490FF1F39550000E0
:1059D000F5510000BC8CFF1F094700000D49000075
:1059E0004C8DFF1F5D550000F9560000288DFF1FEC
:1059F000A54A0000BD4A0000808EFF1FB14A00008A
:105A000029520000088CFF1FF55000005D52000075
:105A10000C8FFF1F81550000B94D0000988CFF1FAF
:105A2000A5550000154B0000C48BFF1F194700004F
:105A300035490000788FFF1FC9550000214E000036
:105A4000748CFF1F29470000894E0000948DFF1FB2
:105A500039470000F94E0000348BFF1F4947000012
:105A600099520000E08CFF1F59470000815100004F
:105A70005C8EFF1F69470000CD520000FC8FFF1FA6
:105A800079470000614F0000F08DFF1F894700003B
:105A9000C94F0000588BFF1F9947000001530000B9
:105AA000308FFF1F1551000031500000388EFF1F4E
:105AB000A9470000795600007C8BFF1FB947000002
:105AC00035530000108BFF1FC94700009D53000095
:105AD0007C8AFF1FD947000049560000CC8FFF1F6A
:105AE000E9470000754B00002C8CFF1FF9470000B0
:105AF000CD4B0000E88AFF1F09480000A08BFF1F64
:105B0000C88EFF1F254C0000194800007D4C000086
:105B100029480000D54C0000C48AFF1FA08AFF1F3F
:105B2000F08FFF1FA150000049480000D150000035
:105B300059480000F160000039480000F0B5461CEB
:105B400083B00D460127032336B22AB204463146FC
:105B50008DE888002448ADB203F0CCFE0C23AA1CCB
:105B600012B200930197052321B21F4803F0C2FE31
:105B70001E4A1F4B12881B68BA422AD023D3022A1E
:105B800010D11C4CA3F6CA0384FB03241C44DB176E
:105B9000C3EB24140A2CA8BF0A2424EAE474A2B29A
:105BA00023B202E000231A461C460D35AA1A012032
:105BB0000093019012B2314603230B4803F018FE04
:105BC000204603B0F0BD0C4CA3F6FC0384FB032479
:105BD000DDE7084CA3F6980384FB03241C44DB1781
:105BE000C3EBE404D6E700BF289EFF1F169DFF1FEE
:105BF0009C9DFF1F898888881F85EB512DE9F04304
:105C00008FB283B0DFF84C80BD1D461D2DB204B2AB
:105C100036B24FF001090AB223463146404600959C
:105C2000CDF8049003F016FE2A463346214640463E
:105C30008DE8200203F00EFE07F10C0200953346BA
:105C400012B22146CDF80490404603F003FE03B0A3
:105C5000BDE8F083289EFF1F2DE9F043804685B004
:105C6000002956D10121304804F08AF92F4998F8CB
:105C7000062098F8083011F80290994522DA4FEA88
:105C800089064D460C24D8F80C3027489B595F688C
:105C900022B2002104F070F9384608F0F1FF3946CD
:105CA0000246214804F002FB1F4804F015FB98F857
:105CB000083001350934AB42A4B206F1040601DD17
:105CC000422CE0D1B9F1000F13D109F10609994531
:105CD0000CDA3C2301213B220391029300930192B1
:105CE00039233F223A21104803F06EFE05B0BDE88B
:105CF000F0830F2301213B22039102930093019231
:105D000039230C223A21084803F05EFE98F8083047
:105D1000DBE700213423009301913F230C2202484A
:105D200003F066FD9EE700BF289EFF1FA89EFF1F91
:105D300010B5104C0121204604F028F9204601211D
:105D400004F01EF920463422552104F015F92046AE
:105D50000222094904F0AAFA20460522074904F064
:105D6000A5FA204604F0B8FA2046BDE8104003F03A
:105D700025BB00BF289EFF1F00FD000004FD0000A2
:105D800070B50D46064608F07BFF00EB400084002E
:105D9000002D36D0284608F073FF00EB400040008D
:105DA00023185B1003F16001091A282209B2174871
:105DB000C3F1600404F0E0F80121144804F0E0F8B5
:105DC000284608F05DFF29460246104804F06EFAA6
:105DD0000E4804F081FA02210C4804F0D1F821B2F7
:105DE00021220A4804F0C8F8304608F049FF31463D
:105DF0000246064804F05AFA0448BDE8704004F030
:105E00006BBA6410C4F16004E5E700BF289EFF1F71
:105E100010B50D4B1B5C51F82340237884B013B1AF
:105E2000012004B010BD04AA01A942F8103D20468B
:105E3000A3699847A38A9B07F2D401A80099FFF7AA
:105E40009FFF012004B010BD149EFF1F2DE9F04FED
:105E50002F4DDFF8CCB0DFF8C4A0DFF8C8900FCD2D
:105E600091B003AC0FC40FCD0FC40FCD0FC42B687E
:105E700023600025A8462F462E4600E09846BAF833
:105E8000003024495BF8232028461123FAF7D4FD7B
:105E900000EBC00400EB840089FB00340444C0170D
:105EA000C0EB6434C4F13C00C6F13C0207F141018F
:105EB000012600B208F1410300901BB2019612B214
:105EC00009B2154803F0C6FC08EB060305F21115EC
:105ED0003C2B2646ADB24746D0D134226B210E482A
:105EE00004F04AF800210C4804F04AF80B4B1B88D8
:105EF00010AA02EB830353F8344C204608F0C0FE8E
:105F000002460548214611B0BDE8F04F04F0CEB975
:105F10009CF60000C8F20000289EFF1FA49BFF1FF4
:105F2000E0F1000009000280214B70B5B3F90030A8
:105F300083EAE374A4EBE374002B82B0A1B22FDBFD
:105F400068466D46012300E0134603EB83025200CE
:105F50009442F9DA174E91FBF3F286FB03E403FB5C
:105F60001211DB173032D3EBA40389B205F8012BF1
:105F7000F1D119462B70FFF703FF0F4B1B786BB164
:105F800001210E4803F0FCFF332274210B4803F07B
:105F9000F3FF01220A49094804F088F902B070BDF4
:105FA0002D238DF800300DF101056846CAE700BFCA
:105FB000349DFF1F676666661A9DFF1F289EFF1FA0
:105FC0009400010010B5424C424882B003F0EAF858
:105FD0002378C3B906213F4803F0D2FF2378012B71
:105FE00037D90A22022B11463A486BD003F0C4FF7E
:105FF00039490322374804F059F9364802B0BDE860
:10600000104004F069B9354B1A7801210523002AA4
:1060100035D10191009311462E4803F06BFC304BB3
:106020001A78002A36D0052301220192009300221B
:106030000A21284803F0DCFB2A4B1A78002A35D1C4
:1060400001210523019100931421224803F052FC01
:10605000C0E7254C2388092B32D9632B8CBF0A213A
:106060001F210A221B4803F087FF2188194804F0EA
:1060700083F9184802B0BDE8104004F02DB90022A1
:10608000019100931146134803F0B2FB144B1A78A8
:10609000002AC8D105230121019100930A210D484E
:1060A00003F028FC0F4B1A78002AC9D001220523DF
:1060B0000192009300221421064803F099FB89E71E
:1060C0003021CEE703F058FF0322084992E700BFD2
:1060D000B09EFF1F289EFF1F10FD0000C79DFF1FE1
:1060E000C09DFF1FC89DFF1F489DFF1F0CFD0000A6
:1060F000F8B56D4D287840B96C4B1B6899425CD35C
:106100006B4A012313702B70F8BD0C4600266948BA
:10611000664F03F047F804F6AC53324665483B60DF
:1061200031212E7003F028FF01216248624D03F0F7
:106130002DFF31465F4803F023FF05225F495D488C
:1061400004F0B4F85B4804F0C7F80C221021594859
:1061500003F012FF0B225A49564804F0A7F8052213
:106160005849544804F0A2F8524804F0B5F8564B88
:1061700050481C68A4F69803C3EB031385FB032562
:106180001D441021DB172022C3EB652503F0F4FE2C
:1061900040F6CC339C4205F124054FF022014FF02C
:1061A00004000BDCFFF7CAFC484B1C88064674B39E
:1061B000012C46D0022C41D00120F8BDFFF71EFD76
:1061C000092243493B4804F071F82A22102139483A
:1061D00003F0D2FE3F4C374884FB0534EB17C3EB8A
:1061E000A404214604F0C8F801223B49314804F0D8
:1061F0005DF804EB8401A5EB41012E4804F0BCF8E6
:10620000012236492B4804F051F80120F8BD3449E9
:106210001022284804F04AF8264804F05DF82A22A3
:106220001021244803F0A8FE3146224804F0A4F8C7
:1062300007222C491F4804F039F8CBE70C222A49E1
:10624000E7E70C2229491B4804F030F8194804F00C
:1062500043F82A221021174803F08EFE31461548D4
:106260001C4E04F089F807221E49124804F01EF85B
:1062700086FB0536EB17C3EBA60631460D4804F046
:106280007BF8224614490B4804F010F806EB86010F
:10629000A5EB4101074804F06FF822460F49054875
:1062A00004F004F82046F8BD0C8BFF1F909EFF1FE2
:1062B000A49EFF1F289EFF1F3B773B9814FD000004
:1062C0001CFD000004FD00009C9DFF1F169DFF1F8C
:1062D00028FD00006766666608020100780101007B
:1062E00034FD000048FD000060FD000050FD00008E
:1062F0002DE9F041754C2278002A05460F4614BF5F
:106300004FF001084FF000084ED1714E3368CB1AA0
:10631000B3F5FA6F04D86B78A3B94046BDE8F081B5
:106320006C4B6D486D49DFF8D0E11A7001230370A2
:106330000988237026208EF8002000F0F1FD6B788C
:10634000002BEAD03760FBF781FB654A654B664955
:10635000127828781B78097802EB4303421E03EB7E
:1063600081030E2AD9D801A151F822F05D64000002
:10637000296400001B6300005D6400001B630000D3
:106380001B6300001B630000116400001B6300001E
:10639000C36300001B6300001B6300001B6300005D
:1063A0001B630000BF630000AF215048484E02F05D
:1063B000A9FCFFF707FE002337602370ABE705F069
:1063C0008DF94A4802F0EEFE0221484803F0D8FD5C
:1063D0000F222321454803F0CFFD052244494348BD
:1063E00003F064FF414803F077FF1E2223213F485A
:1063F00003F0C2FD05223F493C4803F057FF3B48EC
:1064000003F06AFF394802F0D9FF00F0ADFC84E7E1
:10641000394D2B78012B50D9304B2620198800F0AC
:106420007FFD00232B7078E7002B3FF476AF013B14
:10643000324A32F81330002B3FF46FAF274C30480C
:1064400025492D4A23804FF001080023037081F86D
:10645000008082F80080FFF7B5FD5EE793B1013B55
:10646000264A32F8131019B31C4B254D1A4C224AF8
:1064700019800026012326202E702370137000F04F
:106480004FFD15E0154C1E4922880B7004284FF66D
:10649000FF7002F1FF310CBF012202460A440E4E8A
:1064A000154D02F07F0201320121228031702B70E4
:1064B000FFF788FD4FF001082FE70649064A012340
:1064C0000020087013702370A6E700BF0C8BFF1F1D
:1064D000A09EFF1FA49EFF1F979BFF1F489DFF1FAD
:1064E000C79DFF1FC09DFF1FC89DFF1F289EFF1F48
:1064F00070FD000078FD0000B09EFF1F089DFF1F8B
:10650000FC9BFF1F2DE9F04F05468BB00F46AD48B1
:106510000121164603F03AFDAA8812F0010440F06A
:10652000B080DFF8CC8298F80030002B7DD1AB79B9
:10653000A54AD15CA1B9DFF8BCA279781AF803901A
:1065400041B339780139072900F2B780DFE811F04B
:10655000F1005401B5006C01B500B500B500E900CB
:106560007C78002C00F0CA800139EC68387854F847
:106570002170FC68411EB4F80080072900F2A78052
:10658000DFE811F074015901A5006C01A500A50018
:10659000A5009F00DFF854A2DAF80020B21AB2F585
:1065A000967F75D9894A107801281ABF012010708A
:1065B0001170874A18BF0146D05CC0EB0900C0B219
:1065C000FFF7F4F80124CAF80060AB889B0770D588
:1065D0007B78002B6DD0FBF739FA7E4B7E4A7F48E3
:1065E0001B78127839780078022515FB02330A29C6
:1065F00003EB800300F04E810C295AD1002B58D0B8
:1066000003F11900764E774A013B0021400080B229
:1066100026F813100123157088F8003000F080FC74
:10662000714B032220461A702FE0664802F0BAFD33
:106630000121644803F0A4FC62482246214603F08D
:106640009BFCAB88580725D42C68204608F018FB23
:10665000214602465B4803F029FE5A4803F03CFEFF
:10666000092201238DE80C0000217F23554803F007
:10667000F1F800212846FFF7EFFA002388F80030F0
:1066800055E7AB683146384698470BB0BDE8F08F08
:106690000846FAE72B6804A8984704A808F0F0FA1F
:1066A00004A90246474803F001FE464803F014FEE1
:1066B000D6E720460BB0BDE8F08F00240AF803901F
:1066C00083E70021D1543846FB699847FC68A4F859
:1066D0000080002725223C238DE8840041211822D8
:1066E000384803F085F8E968A879FFF791FB374A45
:1066F0003E4B17701E600BB0BDE8F08F3B490A6837
:10670000B21AB2F5967FD4D9304F0E603E78012E82
:1067100000F0B480E968184601233B70FFF778FB6E
:10672000B3E7304AE9791170012288F8002000248B
:10673000C4E72A7A013A4A45BFDD09F10104E4B20F
:10674000A145BAD0224E16F803B0CBEB0900C0B277
:106750000021FFF72BF82B7A052BD9461BD9CBEB61
:106760000402042A40F3AE80A4F1040BBBF1000F35
:10677000C0F2B080063B5B45A8BF5B465FFA83F979
:10678000AA791348B15C994205D000F80290012122
:106790002846FFF761FAC9EB0400C0B201210B4E95
:1067A000FFF704F80021342301910093054831706C
:1067B00040230B223F21A14603F01AF80124AB79B4
:1067C0007CE700BF289EFF1F949EFF1FAE9EFF1F09
:1067D000A89EFF1FC79DFF1FC09DFF1FC89DFF1FD5
:1067E000089DFF1FA49EFF1FB09EFF1F8C9EFF1FD2
:1067F0000C8BFF1F149EFF1F0FFA89F1E868604C95
:1068000050F821602168049134785E49049808604A
:10681000002C71D0012C7FF450AF5B4A317A88F89C
:1068200000401170002449E7B9F1000F50D009F180
:10683000FF34E4B284E7B98A01F0040189B2002987
:106840003FF440AF3B6A03929847039A00283FF415
:106850003DAFAB79FC680021D15438E77B8A4345D2
:106860003CD908F101081FFA88F830E73B8A434514
:106870003BD208F1FF381FFA88F828E725238DE876
:10688000180042483C703C231822412102F0B0FF1E
:106890003046FAE6002B3FF40CAF3D4A3D4E1188DE
:1068A000394A03F11900013B400080B226F8131069
:1068B000012388F80030157000F032FB364B20467B
:1068C0001D70E2E6002A3FF755AF04F1FF3B4DE7AC
:1068D0004C46F3E64FF000094B4651E7BB8ADA0716
:1068E0007FF5F5AEB7F81080F1E6BB8AD9077FF5E2
:1068F000EEAEB7F81280EAE62849C85CC0EB0900A2
:1069000009F1010EC0B201214FF0340B02F803E08F
:10691000FEF74CFFB6681D48019440230B223F212F
:106920000124CDF800B002F063FF40230B223F2189
:106930001648CDF800B0019402F0DCFF2146134860
:1069400003F01EFB304608F09BF9A0EB800000F13D
:106950005F0109B20F220D4803F00EFB304608F02C
:106960008FF931460246094803F0A0FC074803F0BE
:10697000B3FCE968A879FFF74BFAAB799EE600BF54
:10698000EC9EFF1F8C9EFF1FA49EFF1F289EFF1FD3
:10699000489DFF1F089DFF1FB09EFF1FA89EFF1F61
:1069A0002DE9F047DFF808926D4B99F800601B68FD
:1069B000DFF800A282B0003601934FF0030018BF49
:1069C0000126019F9AF8008004F040FB0546042050
:1069D00004F03CFB0446052004F038FB800040EA4C
:1069E0004404062004F032FB2C4364B25D4944EABF
:1069F000C0000A7880F00F03DBB29A425A4A3CD0BA
:106A00001760002259480B7003788DF800808DF8CC
:106A1000012053B3564A12684EF66021BA1A8A42D0
:106A200019D8022B59D0012B5FD0062B48D0032B4D
:106A300063D0042B69D0052B77D0072B7DD0082B92
:106A400000F08380092B68D016B14A4802F0B6FCEA
:106A500002B0BDE8F087484A484C0023012123706A
:106A600003701360938089F800103A4669464448E1
:106A7000FFF748FD3043C6B2E6E71268BA1A1E2A8D
:106A80006BD99AF80020934222D0394C3D488AF8BD
:106A90000030012B276082EA030207609846B1D0DC
:106AA000042BAFD137480068381AB0F5C87FA9D990
:106AB000354C2068381A3228A4D927601A46A1E735
:106AC0003A4669463148FFF71DFD3043C6B2BBE781
:106AD000012B4FF00002E3D1E4E73A4669462C4827
:106AE000FFF710FD3043C6B2AEE73A466946294883
:106AF000FFF708FD3043C6B2A6E73A466946264886
:106B0000FFF700FD3043C6B29EE73A466946234888
:106B1000FFF7F8FC3043C6B296E73A46694620488C
:106B2000FFF7F0FC3043C6B28EE73A4669461D488F
:106B3000FFF7E8FC3043C6B286E73A4669461A4892
:106B4000FFF7E0FC3043C6B27EE73A466946174895
:106B5000FFF7D8FC3043C6B276E7002252E700BF09
:106B6000EC9EFF1FB19EFF1F1C9EFF1FA49EFF1FD8
:106B70009C9EFF1F289EFF1F949EFF1FAF9EFF1F1E
:106B8000D4F70000B49EFF1F249EFF1F28FC0000C6
:106B900098F70000F8F60000DCF600002CF7000083
:106BA000E8F600003CF700007CF70000F08FFF1FC4
:106BB0000C8BFF1F209EFF1F28B11028044BA8BF7D
:106BC000102018607047024B01201860704700BF0A
:106BD000B89EFF1F38B50F4D2B78013B01381B02C3
:106BE000C4B203F47063200443F4404343F00C0345
:106BF00000F4FE00184305F091FB2868013860F0AE
:106C00003F00C0B204F0B8FB2046BDE8384004F0B5
:106C1000B3BB00BFB89EFF1F70B5124D2B78013B70
:106C20001B0203F47063064643F430430806320443
:106C300000F0FE4043F00B03034302F4FE00184350
:106C40000C4605F06BFB2868013860F04F00C0B2BD
:106C500004F092FB304604F08FFB2046BDE8704004
:106C600004F08ABBB89EFF1F70B5124D2B78013B14
:106C70001B0203F47063064643F410430806320413
:106C800000F0FE4043F00903034302F4FE00184302
:106C90000C4605F043FB2868013860F06F00C0B275
:106CA00004F06AFB304604F067FB2046BDE8704004
:106CB00004F062BBB89EFF1F38B5104D2B78013B26
:106CC0001B0203F47063044643F41043000443F0D2
:106CD000090300F4FE00184305F020FB2868013882
:106CE00060F06F00C0B204F047FB204604F044FBA4
:106CF0000020BDE8384004F03FBB00BFB89EFF1F36
:106D000038B50E4D2B78013B1B0203F4706304462B
:106D100043F45043000443F00D0300F4FE00184315
:106D200005F0FCFA2868013860F02F00C0B204F0CA
:106D300023FB2046BDE8384004F01EBBB89EFF1F71
:106D400008B5002005F0B4FB0028FAD108BD00BF4B
:106D500008B564210720FFF75FFF7F210B20BDE806
:106D60000840FFF759BF00BF10B500217B20FFF797
:106D700053FF0024E0B2FFF79FFF0134022004F02C
:106D80009BF9802CF6D110BD10B504464FF440603D
:106D900004F0A2FA04F0FAFA2CB1102C044BA8BFAC
:106DA00010241C6010BD024B01241C6010BD00BFEC
:106DB000B89EFF1F10B5044641F0E00004F0DCFA75
:106DC00004F07F0004F0D8FAC4F3C610BDE8104008
:106DD00004F0D2BA38B5134D2B78044641F6FF7251
:106DE000A0F50050824203F1FF33A8BF02461B0208
:106DF00002F5005203F47063100443F4604343F05F
:106E00000E0300F4FE005204184302F0FE42104349
:106E100005F084FA296801392046C9B2BDE8384036
:106E2000FFF7C8BFB89EFF1F38B504460D46F020D7
:106E300004F0A2FA35B1254414F8010B04F09CFAD1
:106E4000AC42F9D1F720BDE8384004F095BA00BF54
:106E500000B50B4B83B00246998818680090032A4E
:106E6000ADF8041002D903B05DF804FB68460621B2
:106E70008DF80520FFF7D8FF03B05DF804FB00BFD5
:106E80003801010000B50B4B024683B018689988A1
:106E90000090131F4C2BADF8041002D903B05DF81D
:106EA00004FB684606218DF80520FFF7BDFF03B0FF
:106EB0005DF804FB40010100030203F4FE43C0F34C
:106EC000C6101843704700BF03784078DB0103F415
:106ED0007E5300F07F001843704700BF82B002AAC3
:106EE000114642F8040D002012F8013B03F07F0325
:106EF000914243EA0020F7D102B07047003210B44B
:106F000003884FF0010404FA01F418BF012202FAC9
:106F100001F123EA04020A43028010BC704700BF5B
:106F200070B5CEB20C46054603F058FC864203D03D
:106F30003146284603F06CFC0135284603F04EFC30
:106F4000240A844205D021462846BDE8704003F05B
:106F50005FBC70BD38B5054603F040FC4FF000043F
:106F600060F30704681C03F039FC60F30F24A0B23F
:106F700038BD00BFF8B504460020FFF7EBFF002C3A
:106F800000F0CD834FF4AF610220FFF7C9FF4FF44B
:106F90007A610420FFF7C4FF4FF496610620FFF7E3
:106FA000BFFF4FF4FA610820FFF7BAFF4FF4AF615B
:106FB0000A20FFF7B5FF40F6FC010C20FFF7B0FFF9
:106FC0004FF496612220FFF7ABFF4FF416612420A7
:106FD000FFF7A6FF7D212A20FFF7A2FF0C210E203C
:106FE000FFF79EFF01211020FFF79AFF02211220D8
:106FF000FFF796FF00211420FFF792FF00211620D3
:10700000FFF78EFF02211820FFF78AFF01211A20C7
:10701000FFF786FF02211C20FFF782FF04211E20BC
:10702000FFF77EFF14212020FFF77AFF01212620A1
:10703000FFF776FF03212820FFF772FF04212C20A1
:10704000FFF76EFF0F212E20FFF76AFF002130208F
:10705000FFF766FF0C213220FFF762FF002134208A
:10706000FFF75EFF00213620FFF75AFF002138208E
:10707000FFF756FF00213A20FFF752FF00213C2086
:10708000FFF74EFF00213E20FFF74AFF002140207E
:10709000FFF746FF00214220FFF742FF1F21442057
:1070A000FFF73EFF13214620FFF73AFF0E2148204D
:1070B000FFF736FF11214A20FFF732FF0A214C204B
:1070C000FFF72EFF00214E20FFF72AFF0621502058
:1070D000FFF726FF02215220FFF722FF0C21542048
:1070E000FFF71EFF00215620FFF71AFF002158204E
:1070F000FFF716FF01215A20FFF712FF03215C2042
:10710000FFF70EFF0A215E20FFF70AFF0021602033
:10711000FFF706FF04216220FFF702FF0121642030
:10712000FFF7FEFE00216620FFF7FAFE0B21682024
:10713000FFF7F6FE7F216A20FFF7F2FE00216C20A8
:10714000FFF7EEFE00216E20FFF7EAFE002170201F
:10715000FFF7E6FE00217220FFF7E2FE0021742017
:10716000FFF7DEFE23210020FFF7DAFE0220FFF703
:10717000F1FEB0F5805F034680F01184D24A04200E
:107180001380FFF7E7FEB0F5805F034680F0FE83D3
:10719000CE4A06201380FFF7DDFEA0F52F739BB2C9
:1071A000B3F57A6F024606D940F628210620FFF78C
:1071B000B7FE40F62822C64B08201A80FFF7CAFE09
:1071C000A0F52F739BB2B3F57A6F024606D940F64D
:1071D000E4410820FFF7A4FE40F6E442BD4B0A203C
:1071E0001A80FFF7B7FEA0F5FA739BB240F6AC51D8
:1071F0008B42024606D94FF4AF610A20FFF790FE9A
:107200004FF4AF62B44B0C201A80FFF7A3FEA0F539
:10721000FA739BB240F6AC518B42024606D940F657
:10722000FC010C20FFF77CFE40F6FC02AB4B0E206D
:107230001A80FFF78FFE1828034600F2A183A84AA0
:1072400010201380FFF786FE431E9BB20F2B0246D1
:1072500004D901211020FFF763FE0122A14B122067
:107260001A80FFF777FE0A28034600F283839E4ABE
:1072700014201380FFF76EFE0128034604D9002175
:107280001420FFF74DFE0023984A16201380FFF7C5
:1072900061FE7F28034600F26783954A1820138019
:1072A000FFF758FE0428034600F25883914A1A203B
:1072B0001380FFF74FFE0C28034600F249838E4AE5
:1072C0001C201380FFF746FE0428034600F23A8391
:1072D0008A4A1E201380FFF73DFE0928034600F26C
:1072E0002B83874A20201380FFF734FE462803466D
:1072F00000F21C83834A22201380FFF72BFEA0F5A7
:10730000FA739BB240F6AC518B42024606D94FF459
:1073100096612220FFF704FE4FF496627A4B2420F8
:107320001A80FFF717FEA0F5FA739BB240F6AC5136
:107330008B42024606D94FF416612420FFF7F0FD78
:107340004FF41662714B26201A80FFF703FE7F2848
:10735000034600F2E5826E4A28201380FFF7FAFD0B
:107360000628034600F2D6826A4A2A201380FFF7D5
:10737000F1FDA0F132039BB2B3F5967F024604D92A
:107380007D212A20FFF7CCFD7D22634B2C201A8023
:10739000FFF7E0FD0C28034600F2B6825F4A2E207C
:1073A0001380FFF7D7FD1E28034600F2A7825C4A30
:1073B00030201380FFF7CEFD0928034600F26382D8
:1073C000584A32201380FFF7C5FD1E28034600F2FD
:1073D0005482554A34201380FFF7BCFD7F280346B2
:1073E00000F24582514C36202380FFF7B3FD7F2801
:1073F000034600F2368238206380FFF7ABFD7F281A
:10740000034600F228823A20A380FFF7A3FD7F28DD
:10741000034600F21A823C20E380FFF79BFD7F28A1
:10742000034600F20C823E202381FFF793FD7F2864
:10743000034600F2FE8140206381FFF78BFD7F2829
:10744000034600F2F0814220A381FFF783FD384D0F
:1074500028804420FFF77EFD3028034600F2DD81BE
:10746000344A46201380FFF775FD3028034600F2AA
:10747000CE81314C48202380FFF76CFD3028034635
:1074800000F2BF814A206380FFF764FD3028034685
:1074900000F2B1814C20A380FFF75CFD3028034649
:1074A00000F2A3814E20E380FFF754FD012803463C
:1074B00004D900214E20FFF733FD00231F4A50203E
:1074C0001380FFF747FD3BE0329CFF1FDC9DFF1F51
:1074D000EA9BFF1FB09DFF1F7E9DFF1FB89BFF1FF4
:1074E000909BFF1F349DFF1F709DFF1F2A9CFF1F55
:1074F000949BFF1F369CFF1FD69BFF1FCE9BFF1F39
:10750000A09BFF1FC29DFF1F2C9DFF1F269DFF1FDD
:10751000489DFF1F889DFF1FD89DFF1FA49BFF1F35
:10752000249CFF1F809BFF1FB29DFF1F089DFF1F14
:10753000DE9DFF1FB09BFF1F8C9DFF1FCC9BFF1F7D
:10754000431E9BB20B2B024604D906215020FFF7A5
:10755000E7FC0622CF4B52201A80FFF7FBFC0428E1
:10756000034600F23C81CC4A54201380FFF7F2FC22
:10757000431E9BB21D2B024604D90C215420FFF759
:10758000CFFC0C22C54B56201A80FFF7E3FC0128E4
:10759000034604D900215620FFF7C2FC0023C04A4D
:1075A00058201380FFF7D6FC7F28034600F2118194
:1075B000BC4A5A201380FFF7CDFC431E9BB2092B17
:1075C000024604D901215A20FFF7AAFC0122B64B3A
:1075D0005C201A80FFF7BEFC431E9BB2102B0246B4
:1075E00004D903215C20FFF79BFC0322AF4B5E20F4
:1075F0001A80FFF7AFFC431E9BB21D2B024604D935
:107600000A215E20FFF78CFC0A22A94B60201A8019
:10761000FFF7A0FC0228034600F2D580A54A6420AB
:107620001380FFF797FC0128034604D90121642049
:10763000FFF776FC0123A04A62201380FFF78AFC43
:10764000C31E9BB2012B024604D904216220FFF71E
:1076500067FC0422994B66201A80FFF77BFC7F2889
:10766000034600F2AA80964A68201380FFF772FC56
:107670007F28034600F29B80924A6A201380FFF71E
:1076800069FC7F28034600F28C808F4A6C201380AF
:10769000FFF760FC042803467DD88C4A6E201380D7
:1076A000FFF758FC192803466FD8894A70201380C9
:1076B000FFF750FC0228034661D8864A72201380E7
:1076C000FFF748FC0628034653D8834A74201380EA
:1076D000FFF740FC042846D82B88DFF81CE27F4FD8
:1076E0007F4A804D804E814C814903F0010CAEF8F9
:1076F00000C0C3F3400EA7F800E0C3F38007178073
:10770000C3F3C0077B4A2F70C3F30017C3F34015C0
:10771000C3F38013378025800B801080F8BD4FF6AF
:10772000FF7398423FF42EAC23283FF41FAD172877
:107730007FF628AC19287FF691AC1B287FF6AEACFB
:107740001C283FF4C3AC1E287FF6C8AC1F283FF4AA
:10775000CDAC20283FF4E6AC21283FF4EFAC222842
:107760007FF400ADF2E474200021FFF7D9FB002084
:10777000B2E700217220FFF7D3FB0023A5E7002129
:107780007020FFF7CDFB002397E700216E20FFF765
:10779000C7FB002389E700216C20FFF7C1FB002312
:1077A0007BE77F216A20FFF7BBFB7F236DE70B217F
:1077B0006820FFF7B5FB0B235EE700216620FFF78B
:1077C000AFFB00234FE700216020FFF7A9FB002358
:1077D00024E700215820FFF7A3FB0023E8E602215D
:1077E0005220FFF79DFB0223BDE60A214C20FFF744
:1077F00097FB0A2356E611214A20FFF791FB11233C
:1078000048E60E214820FFF78BFB0E233AE61321B2
:107810004620FFF785FB13232BE61F214420FFF7AB
:107820007FFB1F231CE600214020FFF779FB00238C
:1078300009E600213E20FFF773FB0023FBE5002152
:107840003C20FFF76DFB0023EDE500213A20FFF718
:1078500067FB0023DFE500213820FFF761FB0023F1
:10786000D1E500213620FFF75BFB0023C3E50021B3
:107870003420FFF755FB0023B4E50C213220FFF73D
:107880004FFB0C23A5E500213020FFF749FB002327
:1078900096E500BF108AFF1F6089FF1F128AFF1F35
:1078A000169CFF1FB69DFF1F8C9BFF1F608AFF1F4A
:1078B0002C89FF1F229DFF1F849DFF1FD89BFF1F48
:1078C000C49DFF1F049CFF1FC09BFF1F7C9BFF1FCD
:1078D000049EFF1F169DFF1FE09DFF1FE89BFF1FDB
:1078E000269CFF1F1A9DFF1F249DFF1F869DFF1FC3
:1078F0003C9DFF1FA89DFF1F7A9DFF1F0F212E207B
:10790000FFF70EFB0F2352E504212C20FFF708FBA5
:10791000042343E503212820FFF702FB032323E58B
:1079200001212620FFF7FCFA012314E51421202071
:10793000FFF7F6FA1423DDE404211E20FFF7F0FA26
:107940000423CEE402211C20FFF7EAFA0223BFE45D
:1079500001211A20FFF7E4FA0123B0E402211820E4
:10796000FFF7DEFA0223A1E400211620FFF7D8FA80
:10797000002392E402211220FFF7D2FA022376E4D8
:107980000C210E20FFF7CCFA0C2358E44FF47A6157
:107990000420FFF7C5FA4FF47A63FFF7F9BB4FF401
:1079A000AF610220FFF7BCFA4FF4AF63FFF7E6BB0D
:1079B000F8B5872006F0C8FB204B214A054603CBCB
:1079C0001368C5F803001A0C7620C5F807102B8041
:1079D000AA70FFF771FA2E46002426F80B0FA0B20A
:1079E000FFF7B8FAFFF768FA0234762C26F8020F90
:1079F000F5D16C1E05F182064FF0FF3014F8013FFF
:107A0000082758400F4B40F300017A1E0B4012F03C
:107A1000FF0783EA5000F5D1B442EFD1C043FFF72E
:107A20005DFA3A46C5F883008721284604F0C4FC75
:107A30002846BDE8F84006F08FBB00BF4C010100AE
:107A4000480101002083B8EDF0B50E4B0E4C054601
:107A500093E8070085B024682E88AD7801AB83E8F1
:107A60000700270C184600220B21ADF804408DF8C2
:107A70000670ADF80C608DF80E5004F09DFC05B05A
:107A8000F0BD00BF5801010048010100F0B5124BE4
:107A9000124D1E68124F0FCD87B06C460FC495E88B
:107AA000030044F8040B38683B79CDF80D00320C24
:107AB000232021808DF802208DF81130ADF8006070
:107AC000FFF7FAF90022ADF80B001221684604F026
:107AD00073FC07B0F0BD00BF480101006401010064
:107AE00004FD0000002004F0E3BC00BF02F02EBE45
:107AF00070B5124C82B00025402306462946204628
:107B0000009301958023202201F072FE2022294655
:107B1000204602F031FA2046012102F037FA3046C1
:107B200007F0AEF831460246204602F0BFFB204681
:107B300002B0BDE8704001F041BC00BF289EFF1FAD
:107B4000F0B5862983B075D90546441E00F182063A
:107B50004FF0FF3014F8012F08275040404A40F3FF
:107B600000017B1E0A4013F0FF0782EA5000F5D1A6
:107B7000B442EFD1C043FFF7B1F90146D5F8830015
:107B80000190019A914202D0B2F17F2F0BD105F101
:107B90000B00FFF799F976280BD03248FFF7A8FFC2
:107BA000002003B0F0BD3048FFF7A2FF384603B015
:107BB000F0BD05F10D00FFF787F9232840D100241F
:107BC00040F6AC5613E004281AD0062821D0082825
:107BD0001FD00A2828D00C2822D1A1F5FA7292B21F
:107BE000B24201D8FFF79CF90234762C0ED004F192
:107BF0000D002844FFF768F9022C0146A0B2E2D13B
:107C0000B1F5805FEED30234762CF0D1012003B0C1
:107C1000F0BDA1F52F7292B2B2F57A6FE4D8E1E728
:107C2000222801D0242811D1A1F5FA7292B2B242D1
:107C3000DAD8D7E70D48FFF75BFF002003B0F0BDAF
:107C40000B48FFF755FF002003B0F0BD2A28C9D12B
:107C5000A1F1320292B2B2F5967FC5D8C2E700BF59
:107C60002083B8EDA8010100940101007C0101000E
:107C7000BC01010003290CD970B5461C82B0054631
:107C80000C46304603222A4907F068F810B102B0CA
:107C900070BD70470B2C05D905222649281D07F019
:107CA0005DF840B12448FFF723FF244802B0BDE847
:107CB0007040FFF7C9BE05F10901032201A807F0D2
:107CC0009DF801A803221E4907F048F8D8B1032205
:107CD0001C4901A807F042F808B301A803221A4979
:107CE00007F03CF8B0B91948FFF702FFA11E89B2AE
:107CF0003046FFF725FF0028C9D0154802B0BDE87F
:107D00007040FFF7F5BE1348FFF7F2FEFFF750FE95
:107D10001148F3E71148FFF7EBFE1148C6E7114899
:107D2000FFF7E6FE02B0BDE87040FFF7AFBE00BF50
:107D300048010100D4010100DC010100F001010053
:107D4000F40101001C0201003402010038020100AC
:107D50004C020100F80101000C0201006002010068
:107D600074020100200201002DE9F043174D2B6839
:107D700083B081460F469046F3B1154E34880A19F8
:107D800092B218461146328006F05CFD28603A46F1
:107D90004946204402F06CFDB8F1000F09D031884B
:107DA0002868FFF767FF286806F0D6F900232B60E4
:107DB000338003B0BDE8F083054E0193084631805F
:107DC00006F0C2F9019B28601C46E0E7C09EFF1F39
:107DD000BC9EFF1F10B51F4C4FF4FA70FCF7BCFBA4
:107DE000204601F0DFF900221146204602F0C4F8D7
:107DF0002046012102F0CAF82046002102F0C0F816
:107E00000B221549204602F051FA204602F064FA8E
:107E10000F221249204602F049FA204602F05CFA8D
:107E20000F490722204602F041FA204602F054FA98
:107E3000204601F0C3FA0B4B0B4A1A604FF4FA705C
:107E4000FCF78AFBFFF722FE0848BDE81040FFF769
:107E50004FBE00BF289EFF1F780201008402010070
:107E60009402010078A0FF1F697D00009C020100C0
:107E70000020704790F8392090F83800101A7047A9
:107E800090F8383090F839209A4205D95A1C0344AA
:107E900080F83820187E70474FF0FF30704700BFE1
:107EA00090F8383090F839209A4286BF1B18187E17
:107EB0004FF0FF30704700BF704700BF38B5054630
:107EC000B0F85E0090B195F85D301446C3F1210220
:107ED00094420CD805F13B001844224602F0C8FC3D
:107EE00095F85D30234485F85D30204638BD01208B
:107EF00014462871EEE700BFB0F85E306BB190F821
:107F00005D30202B07D8C218013380F85D30012086
:107F100082F83B107047012303710020704700BFB7
:107F20000023426980F8383080F8393080F85C30BE
:107F300080F85D3080F85E3080F85F3006CA30B47B
:107F40000D68046943662A4383660A60A370426928
:107F500090F861301649146813441D7A5B7B01EB7D
:107F6000C5051B026D6803F4E06343F064032B60F6
:107F700090F8623013449D7CDB7D01EBC5011B0250
:107F8000496803F4E06343F064030B6021685368BD
:107F9000194205D0036927225A70036904229A7195
:107FA000036920225A71036980229A7030BC70479D
:107FB000D00D010043690CCB12681A420CD0094B5A
:107FC00099420AD9084B9942036994BF1A220D229B
:107FD0005A70036904229A717047036927225A7004
:107FE000F7E700BF7F1A06003F420F0010B5026995
:107FF000D378DBB2D90604463DD510215806D1709E
:1080000038D503F0040303F0FF02002B51D03D49A3
:10801000626E00230B7084F85D30002A5BD09047BD
:1080200094F85D30002B56D02369D0229A702369D2
:1080300094F83B201A712369012284F85C20022203
:10804000DA7010BD304B84F860009C424AD02F4B50
:108050009C4252D094F8391013791F29DBB207D80B
:108060002848007820B16018013184F8391003766F
:108070000223D37010BD5906C3D4917801F01001CA
:1080800001F0FF000029DDD013F001031ED194F8A8
:108090005C1094F85D00884281BF4B1C091984F87C
:1080A0005C3091F83B3013712369D0229A702269B9
:1080B000DEE7236984F83920C0229A702369114AC7
:1080C0001979012111700222DA7010BDC02393705A
:1080D00022691379CCE70122002384F85D2084F81B
:1080E0003B30A1E7626994F86130094913440322E7
:1080F000187A02F043FD2269ACE7626994F86130B6
:108100000449F3E7C49EFF1F6090FF1FCC90FF1F40
:1081100075810000818100000369DB7803F0200392
:1081200073B190F860300133DBB2012B80F860301E
:108130001AD9426990F861301344187A02F09ABD56
:1081400070B5426903F0FF0590F8613013440446AE
:10815000187A02F08FFDA36E5BB184F8385094F862
:108160003900BDE87040184790F85F30002BE0D030
:10817000704770BD0148FFF7CFBF00BF6090FF1F81
:108180000148FFF7C9BF00BFCC90FF1F2DE9F047A2
:10819000374FDFF8E0903B68026982B006460093F3
:1081A000DDF800800021A025D3789B065BD53B68D5
:1081B0000193019BC8EB03030F2BF5D949B1102B99
:1081C000F2D000209070336980229A7002B0BDE82E
:1081D000F087726996F8613013440521187A02F02D
:1081E00043FF726996F861301344012193F812A09D
:1081F000504602F039FF09240021504602F020FFCA
:108200002B46013BFDD10121504602F019FF2B46C0
:10821000013BFDD1013CEFD1706996F8611001443A
:108220004FF4A0720C7A4B7B09EBC4011B02496826
:1082300003F4E06343F064030B6096F86230034498
:10824000997CDB7D09EBC1011B02496803F4E06303
:1082500043F064030B60013AFDD13269D3789B0689
:108260004FF00101A3D4012002B0BDE8F08700BFA8
:10827000EC9EFF1FD00D0100F0B503691222DA70E9
:108280000269937803F0200385B004460D46002B65
:108290005ED0B42393703C4922690B680093009E22
:1082A00005E00B680193019B9B1B042B42D8D378FC
:1082B00003F0200303F0FF00002BF2D094F85D30B0
:1082C000002B31D04FF0000E4FF0020C04EB0E03E8
:1082D00093F83B3013710B680393039F206907E009
:1082E0009B060DD50B680293029BDB1B052B28D840
:1082F000C378DBB203F0020202F0FF06002AEFD0DF
:1083000080F803C02669F378DBB2DF0632462DD44D
:108310009F062BD5DB0731D40EF1010E94F85D30AA
:108320005FFA8EFE7345D1D800201DBB002384F870
:108330005E3004E09070236980229A70042005B0BA
:10834000F0BD86702369802204209A7005B0F0BDCC
:1083500003F0FF06FFF71AFF10B9042005B0F0BDC7
:10836000236984F85F60B0229A7094E78023B37029
:108370000420DAE726698023B370D7E7BEF1000F47
:108380000CBF02200320F6E7EC9EFF1F2DE9F04111
:1083900006690025122780F8385080F83950F770A8
:1083A000D0F810C09CF802E00EF0200E88B0044611
:1083B000884615461E46BEF1000F49D0B4238CF8FE
:1083C0000230784B21691A680092DDF800E006E07F
:1083D0001A6801920198CEEB0000042830D8C878C2
:1083E00000F0200000F0FF070028F1D04FEA48021B
:1083F00042F00102D2B20A711A680292DDF808E076
:10840000206906E01A6803920399CEEB0101052961
:108410002AD8C17801F0020101F0FF070029F1D04C
:108420004FF0020C80F803C02269D17811F01107D7
:1084300022D12DBB002E0CBFA0238023937003E01C
:108440008F70236980229A70384608B0BDE8F081A9
:108450000EF0FF07FFF79AFE0028F5D0236984F895
:108460005F70B0229A70ACE787702369802238462B
:108470009A7008B0BDE8F081802393700027E3E78D
:10848000012D75D0A021917021690A79BE466746F9
:108490004FF0A80C1A680492049805E01A68059237
:1084A000059A121A052A4AD8CA7802F0020202F086
:1084B000FF08002AF2D0CF702169CA78D2B212F038
:1084C000100F08465AD1920658D5013DEDB2012D44
:1084D00049D0BEF11F0F3BD90A79012DDAD11A68B4
:1084E0000692069D05E01A680792079A521B052A14
:1084F00046D8C27802F0020202F0FF01002AF2D050
:108500000223C3702269D378DBB2D9063AD49B0622
:1085100034D5B023BEF11F0F93703FD8226904EB0E
:108520000E0312791A760EF1010E5FFA8EFE16B165
:10853000236980229A7084F839E0774684E781F8CD
:108540000280236980229A70774684F839E07BE7BD
:1085500004EB0E0291F8048082F818800EF1010EEF
:108560005FFA8EFEB9E781F802C021690846B0E7DC
:10857000A82191702069BE460279B0E7774663E78B
:108580008170DEE71021A023D170013BFDD122696B
:10859000937803F0F7037746937055E723691B79C7
:1085A000C5E700BFEC9EFF1F0148FFF71FBD00BFDE
:1085B0006090FF1F0148FFF719BD00BFCC90FF1F5F
:1085C000704700BF38B5144C037801225B000546A4
:1085D000204684F83B3084F85E2084F85D20FFF765
:1085E0008BFC20460021FFF747FE0B4C2978012326
:1085F00020461A46FFF7CAFE0128F6D194F8383013
:1086000094F839209A4205D9E218013384F83830B9
:10861000107E38BDFF2038BD6090FF1F38B51B4C61
:10862000037801225B000546204684F83B3084F83D
:108630005E2084F85D20FFF75FFC20460021FFF7F5
:108640001BFE124C2978204601230222FFF79EFED2
:108650000228F6D194F8382094F839108A420FD2C3
:10866000531CDBB2A018994284F83830007E0AD936
:10867000234402321B7E84F8382040EA032038BDB0
:108680004FF6FF7038BD40F47F4038BD6090FF1F4B
:108690000C2901D9002070470231490001F0FE0188
:1086A000FFF7BCBF70B50C4C0378164601255B0084
:1086B000204684F83B3084F85E5084F85D50FFF724
:1086C0001BFC31462046FFF717FC29462046BDE833
:1086D0007040FFF7D1BD00BF6090FF1FF8B50546A1
:1086E0000F461646412421463A462846FFF7DAFF50
:1086F000611C0234C9B232462846E4B2FFF7D2FF09
:10870000592CF0D1F8BD00BF38B504460D463548A8
:10871000FFF706FC6322802120462570FFF7C2FF89
:10872000012002F0C9FC204600225E21FFF7BAFFBB
:1087300020465D21FFF746FF242801D0002038BDE8
:10874000204606220C21FFF7C9FF204601222B21DB
:10875000FFF7A8FF204601222C21FFF7A3FF2046A8
:108760000E222D21FFF79EFF204600222E21FFF72B
:1087700099FF204601222F21FFF794FF2046052272
:108780003021FFF78FFF204601223121FFF78AFFBA
:10879000204600223221FFF785FF204600223321A8
:1087A000FFF780FF204600223421FFF77BFF2046A1
:1087B00000223521FFF776FF204600225B21FFF7DC
:1087C00071FF204610225C21FFF76CFF204620221B
:1087D0005D21FFF767FF20468F225E21FFF762FFD2
:1087E000012038BD6090FF1F10B4047F4160022C4F
:1087F000C26002D010BC01F0D7BB836810BC184720
:1088000090E80C00F0B41C6859682568164F174EA4
:1088100029432160164D17491760D6601561116014
:10882000417A154A5C180A3194F8244053F82150D3
:1088300002EBC40149680D60017A5C1803EB810109
:10884000247ECD6902EBC40149680D60817A581815
:1088500003EB810390F83000596B02EBC002F0BCCF
:1088600053681960704700BF01401F0001100038B5
:108870000110007800001F80D00D0100704700BF7C
:10888000F0B50C1EBDF8146034DBB0F90670191990
:10889000B942C4BF3B1B1BB2002BA6461CDD002AFD
:1088A0001146B8BFD11D02F00705CC10826A012025
:1088B00007FB04E1A840012E0A44C0B21ED00CD32D
:1088C000022E09D1013B12FA83F3013A12F8011F7B
:1088D00041409A421170F9D1F0BDC043013B12FAF8
:1088E00083F3C0B2013A12F8011F014093421170A4
:1088F000F9D1F0BD23441BB20024C6E7013B12FAB4
:1089000083F3013A12F8011F01439A421170F9D121
:10891000F0BD00BFF8B50D1E0EDB14461F4606461F
:1089200001F03AFBA84207DD002C05DB304601F0E0
:1089300037FBA04201DCF8BDF8BD304601F02AFB50
:10894000022853D003284BD0012806D16540F38874
:108950006C406540013B5D1B2DB2012F03D02AD333
:10896000022F14D0F8BD002C2246B6F90630B06AAA
:10897000B8BFE21D42F3CF0202FB035504F0070427
:10898000435D012101FA04F41C434455F8BD002C59
:108990002246B6F90630B06AB8BFE21D42F3CF02F4
:1089A00002FB035504F00704435D012101FA04F4BE
:1089B0005C404455F8BD002C2246B6F90630B06A3A
:1089C000B8BFE21D42F3CF0202FB035504F00704D7
:1089D000435D012101FA04F423EA04044455F8BD7F
:1089E0003389013B591B25460CB2B6E7F188328921
:1089F0000139013A4D1B141B2DB224B2ADE700BF63
:108A00002DE9F041079E9DF91880089D04461F46F8
:108A100000F0C0FF0D4B0E480E4984F83380FF2252
:108A2000002F08BF1F4684F82F20002384F8302031
:108A300084F8312084F832202060A665E5656762FD
:108A400061652362A3622046BDE8F0816090FF1F4C
:108A5000280301000110013810B50446806A034B59
:108A6000236008B105F078FB204610BD2803010003
:108A7000F8B5436ADBB190F82C200125AA4083F8B1
:108A80003B2083F85E5083F85D500446406A0368DB
:108A90000E461B6800219847606A036831461B68D0
:108AA00098472946606ABDE8F840FFF7E5BBC26B0E
:108AB000C56C1368046A23EA050313604CB122688D
:108AC0004FF00043D3625163D36A002BFCDA936BFF
:108AD000F8BD836B466B0825802410E03768426C34
:108AE0003A4332601F68826C3A431A601A68876C96
:108AF000013D22EA07024FEA54041A6007D02142DE
:108B0000ECD13268476C22EA07023260EAE7F8BD2E
:108B100070B50446406A0D4600282BD0A16DFFF7C2
:108B200049FA002D20460CBFA621A721FFF7A0FF80
:108B3000606A20B1E16DBDE87040FFF73BBA216C7F
:108B4000226D0868236A02430A6093B1DA7A82B11F
:108B5000D00703D5224A99691160DA7A910703D5C3
:108B6000204AD9691160DA7A520702D51E4A1B6A77
:108B7000136070BD236A002B2BD0D97A626DE1B1EE
:108B800072B6D97ACE0706D51848D968066831403A
:108B900099610160D97A880706D515481969066870
:108BA0003140D9610160D97A4E0705D5114859691C
:108BB000066831401962016062B61B68D96891424B
:108BC00007D00D4818600D49DA6042F08040186106
:108BD0001960226C216D136823EA01031360A0E77A
:108BE00000E100E004E100E008E100E080E100E0F5
:108BF00084E100E088E100E001403F0000003F80A8
:108C0000436A2DE9F04105460E469046002B3ED0C2
:108C100090F82C100124A14083F83B1083F85E40AB
:108C200083F85D40406A036800211B6808F1FF3744
:108C30009847FFB2B8F1000F23D03744A046013E59
:108C4000686A16F8011F03681B6898470134B74229
:108C5000E4B216D0202CF3D10121686AFFF70CFB97
:108C600095F82C206B6A520083F83B2083F85E80D5
:108C700083F85D80686A036800211B6898470124B7
:108C8000DEE7686A0121BDE8F041FFF7F5BAC26B83
:108C9000C16C136823EA010306EB080413604FF06C
:108CA0000048A6420ED02B6A16F801EB63B11A6891
:108CB000C2F82C80C2F834E0D36A002BFCDAA6425A
:108CC000936BF0D1BDE8F081AB6BD5F834C00820D0
:108CD0008021DCF800206F6C1EEA010F14BF3A43BC
:108CE000BA43CCF800201A68AF6C3A431A601A688D
:108CF000AF6C013822EA07024FEA51011A60E8D14D
:108D0000CFE700BF70B50446406A0D46002828D062
:108D1000A16DFFF74FF920462946FFF7A9FE606ACB
:108D200020B1E16DBDE87040FFF744B9216C226DC0
:108D30000868236A02430A6093B1DA7A82B1D007E5
:108D400003D5234A99691160DA7A910703D5214A3C
:108D5000D9691160DA7A520702D51F4A1B6A13607B
:108D600070BD236A002B2BD0D97A626DE1B172B647
:108D7000D97ACE0706D51948D96806683140996175
:108D80000160D97A880706D5154819690668314007
:108D9000D9610160D97A4E0705D51248596906682C
:108DA00031401962016062B61B68D968914207D0F0
:108DB0000D4818600D49DA6042F080401861196072
:108DC000226C216D136823EA01031360A3E700BF3F
:108DD00000E100E004E100E008E100E080E100E003
:108DE00084E100E088E100E001403F0000003F80B6
:108DF0002DE9F041044686B0806A9DF830801E4619
:108E00000F461546B4F90830002800F04281DA1DFB
:108E100048BF03F10E02B4F90630D21003FB02F290
:108E2000002105F0BDFCB4F90820202A00F392804F
:108E3000B4F90610A34B0120203A733902EBD27229
:108E400001EBD1714FF0200E029073208DE80140AC
:108E500042F34F0241F34F01204600F051FE606A99
:108E600084F82D70002800F04D81002D40F08A809C
:108E7000B4F90830202B14BF3D253C2584F82C5034
:108E8000B8F1000F40F0858006B394F93300002854
:108E900018DBC0B2012102F0E7F8012194F8330099
:108EA00002F0CEF8012002F007F9002194F8330017
:108EB00002F0C6F80A2002F0FFF8012194F833000E
:108EC00002F0BEF8606A002800F08280A16DFFF712
:108ED00071F804227C492046FFF792FE217A01397D
:108EE000C9B22046FFF7C4FD784904222046FFF7A7
:108EF00087FE94F92D30012B14BF14211021204638
:108F0000FFF7B6FD042272492046FFF779FEB4F957
:108F10000630802B00F09280602B00F0A680D921D3
:108F20002046FFF7A5FD94F92D30012B14BFF12148
:108F300022212046FFF79CFD204606226549FFF7C7
:108F40005FFE606A50B3E16DFFF734F8012006B0B0
:108F5000BDE8F081B4F906105F4B0120403A523968
:108F60004FF0400E029002EBD272522001EBD17111
:108F70008DE8014042F34F0241F34F01204600F0DB
:108F8000BFFD6CE76DB284F82C50B8F1000F3FF4D0
:108F90007BAFFEF7C5FF002E94D076E7216C226DE3
:108FA0000868236A02430A6073B1DA7A62B1D007B3
:108FB00003D54A4A99691160DA7A91077CD452073D
:108FC00002D5474A1B6A1360012006B0BDE8F08154
:108FD000236A002B2BD0D97A626DE1B172B6D97AAF
:108FE000CF0706D53F48D9680568294099610160D7
:108FF000D97A8E0706D53C48196905682940D96198
:109000000160D97A4D0705D5384859690568294066
:109010001962016062B61B68D968914207D0344872
:1090200018603449DA6042F0804018611960226C9F
:10903000216D136823EA010313604AE7B4F908308D
:10904000202B00F08680402B7FF469AF2A49204610
:109050000322FFF7D5FD94F92D30012B14BFCF214A
:109060009F212046FFF704FD59E7B4F90830102B83
:109070007FF455AF214920460322FFF7C1FD94F943
:109080002D30012B14BFAF2110212046FFF7F0FC3B
:1090900045E7DA1D48BF03F10E02B4F90630D210DD
:1090A00003FB02F21046059205F04EF8A06200287C
:1090B0003FF44DAF059AB3E6114AD9691160DA7AE7
:1090C0007DE700BF80030100600501006405010029
:1090D000680501006C0501007405010000E100E075
:1090E00008E100E080E100E084E100E088E100E0E8
:1090F00001403F0000003F807C0301003408010074
:1091000004E100E0012194F83100244F01F0ACFFAC
:1091100094F83200012101F0A7FF94F9312094F96D
:10912000323057F83220E26357F83330206A236434
:109130000125E56425651A682A431A6078B1B8F1FB
:10914000000F3FF428AFFFF75BFB002E3FF4BAAEF1
:109150009BE6042212492046FFF752FDDFE629462E
:1091600094F82F0001F080FF294694F8300001F0B8
:109170007BFF94F92F2094F9303057F83220626346
:1091800057F833306564A5641A68A36322F00102BE
:109190001A60002E3FF496AE77E600BFD00D0100B6
:1091A00078030100B0F90820D31D48BF02F10E0377
:1091B000B0F90620806ADB1002FB03F2002105F003
:1091C000EFBA00BFF0B50029BDF814502EDBB0F99E
:1091D0000660B1422ADA002A59DBB0F90870144659
:1091E0001C44BC42C4BFBB1A1BB2002B1EDDD2B252
:1091F000D408D0F828E016FB041112F00702DBB205
:109200000EEB010421D0C2F10807FAB2374F9342A6
:10921000BF5C0CD2C3EB020CFF2646FA0CF6012D04
:1092200007EA06073FD005D3022D36D0F0BD012D49
:1092300039D030D21EF8016026EA07070EF8017017
:109240009342F3D3B0F906100C449A1AD2B2072A0B
:1092500010D9022D36D0002D14BFFF26002613464C
:109260002670083BB0F90610DBB2072B0C44F7D888
:1092700002F00702002AD9D01D4B012D9B5C1DD0A6
:1092800017D3022DD2D1227853402370F0BD13445E
:109290001BB20022A1E7022D25D11EF80160774004
:1092A0000EF80170CCE71EF8016037430EF801702C
:1092B000C6E7227822EA03032370F0BD2278134325
:1092C0002370F0BD11462378DB4323700839B0F9D1
:1092D0000630C9B207291C44F5D812F00702A5D000
:1092E000034B9B5CCFE73444AFE700BF180301009A
:1092F0000803010070B4C47DBDF80C50022C18D0D6
:10930000032C1FD0012C0BD0002A03DBB0F908403E
:10931000944201DC70BC7047039570BCFFF7B0BA93
:10932000C4880395013CA41A0A4621B270BCFFF719
:1093300049BF0689C488013E641AB21AE41A12B2FF
:1093400021B2E1E704890395E41A641A114622B2B6
:1093500070BCFFF737BF00BF70B4C57DBDF80C60AF
:10936000022D1AD0032D12D0012D03D0039670BC0C
:10937000FFF728BFC488E41AA41A0A4621B2002ABB
:1093800003DBB0F90840944213DC70BC70470489D9
:10939000013C641A114622B2F1E7C488058903969C
:1093A000013CAD1AED1A621A11B22AB270BCFFF775
:1093B00009BF039670BCFFF763BA00BF2DE9F843FD
:1093C0000446406A002863D0A16DFEF7F3FD052234
:1093D00074492046FFF714FCA1790139C9B220462F
:1093E000FFF746FBB4F90820E588A66AD31D48BFFD
:1093F00002F10E03DB10626A15FB03F51FFA85F814
:10940000002A7BD094F82C300125AB4082F83B3009
:1094100082F85E5082F85D50606A036840211B68E4
:1094200008F1FF379847BFB2B8F1000F23D0374497
:10943000A846013E606A16F8011F03681B6898473A
:109440000135B742EDB216D0202DF3D10121606A6B
:10945000FEF712FF94F82C20636A520083F83B2039
:1094600083F85E8083F85D80606A036840211B6832
:1094700098470125DEE70121606AFEF7FDFE606A7C
:10948000002800F08D80E16DBDE8F843FEF792BD45
:10949000236A002B2BD0D97A626DE1B172B6D97AEA
:1094A000CE0706D54048D968056829409961016012
:1094B000D97A8D0706D53D48196905682940D961D3
:1094C0000160D97A480705D53948596905682940A6
:1094D0001962016062B61B68D968914207D03548AD
:1094E00018603549DA6042F0804018611960226CDA
:1094F000216D136823EA0103136068E7E26BE36CF4
:109500001168276A0B4306EB080913604FF0004E01
:109510004E450DD016F801CB2FB33A68C2F82CE0B7
:10952000C2F834C0D36A002BFCDA4E45936BF1D1FC
:10953000226C236D11680B43136097B1FB7A83B1E2
:10954000D90703D51D4BBA691A60FB7A9A0703D570
:109550001B4BFA691A60FB7A5B0702D5194B3A6A12
:109560001A60BDE8F883A36BD4F83480082080210A
:10957000D8F80020656C1CEA010F14BF2A43AA43E7
:10958000C8F800201A68A56C2A431A601A68A56CEE
:10959000013822EA05024FEA51011A60E8D1B7E723
:1095A000276AC5E71003010080E100E084E100E0E4
:1095B00088E100E001403F0000003F8000E100E062
:1095C00004E100E008E100E02DE9F04F85B09946A4
:1095D000BDF93870BDF83CA0BB1AC1EB090B002BDC
:1095E000B8BF5B42BBF1000FB8BFCBF1000B5B45CE
:1095F0000D4616460093804648DC4D453A463346B4
:109600004CDC194613460A46C5EB09019B1A89B280
:10961000002B0CB2B8BF5B4204EBD474BE42ACBFAB
:109620004FF0FF3201224D45039102924FEA64044C
:1096300029DC9BB201930DE0D8F80070BF69B847F0
:10964000019BE41AA3B21CB20135002C2DB211DB30
:10965000A94518DB009B5B452A46534631464046E8
:10966000EADCD8F80020534697692946324640463E
:10967000B847E5E7029A1644039AA94502EB0304AA
:1096800036B224B2E6DA05B0BDE8F08F4A462B4682
:10969000B94635464D4517461E46B2DD3046294689
:1096A0003E464D4607468946AEE700BF10B4046803
:1096B0002469A44610BC604730B40468BDF8085063
:1096C0000295A46BA44630BC604700BF30B4046868
:1096D000BDF808500295E46BA44630BC604700BF5B
:1096E00070B40468BDF90C60BDF810500396049581
:1096F000246CA44670BC6047704700BF10B582B0B0
:10970000B0F90C2001910168009200220C6CB0F9B4
:109710000A301146A04702B010BD00BF704700BF1D
:1097200001F003010129C17506D0032904D0C288C4
:1097300003894281838170470289C3884281838182
:10974000704700BF2DE9F0410568134E6F6986B080
:10975000B7420446BDF8308010D1013B13441BB220
:109760000093CDF804800B46AD6A2046A8472368D5
:10977000DB6AB3420AD106B0BDE8F08105930492DA
:109780000391B84703A925680EC9E6E7204606B04D
:10979000BDE8F041184700BFF99600002DE9F041FF
:1097A0000568124E6F6986B0B7420446BDF8308036
:1097B0000FD1013BCDF804800B4400921BB2AD6A7F
:1097C0002046A8472368DB6AB3420AD106B0BDE849
:1097D000F081059304920391B84703A925680EC947
:1097E000E7E7204606B0BDE8F0411847F9960000CB
:1097F0002DE9F04F0568DFF858B06F6985B05F4517
:109800000646BDF93890BDF83CA00C46904615D1EF
:109810001F19BC420CDACDF800A0214601342D6A94
:109820004B464246304624B2A847BC423568F2DB7C
:10983000EB6A5B4507D105B0BDE8F08F0393B847ED
:109840003568039BE4E7304605B0BDE8F04F1847A4
:10985000F99600002DE9F04387B099420546BDF91D
:109860003840BDF83C6025D0A24212D00768DFF82E
:109870008080D7F81490C14532D18DE85000284639
:10988000BC6AA0472B68DB6A434524D107B0BDE81A
:10989000F083994202DD08461946034628680E9671
:1098A000C46B01335B1A1BB22846A44607B0BDE85F
:1098B000F0436047A24202DD134622461C46286858
:1098C0000E96631C846B9B1A1BB22846A44607B0F5
:1098D000BDE8F0436047284607B0BDE8F0431847AD
:1098E000059304920391C84703A92F680EC9C4E7E2
:1098F000F99600002DE9F04FD0F800E0DFF89090E5
:10990000DEF814B083B0CB450446BDF93080BDF815
:1099100034A00D4617461E4631D1CDF800A0DEF822
:1099200024B0294633463A462046D8472368CDF826
:1099300000A008F1FF323A44D3F824B0294612B20D
:1099400033462046D8472368CDF800A02946D3F8EF
:1099500020B03A4643462046D8472068CDF800A0BC
:10996000711E29444346056A09B23A462046A84773
:109970002368DB6A4B4506D103B0BDE8F08FD847BA
:10998000D4F800E0C9E7204603B0BDE8F04F18471F
:10999000F9960000F0B4002401264FF6FF75094F38
:1099A00007600471C475C48104824476C4618675FD
:1099B000067685824582C180028141818281F0BC28
:1099C000704700BF400801002DE9F04F85B00668E0
:1099D000BDF84450BDF93880CDF8008004460195AB
:1099E000D6F848B00392BDF93C60BDF94070894695
:1099F0009A46D84723680195009742465146D3F8C6
:109A0000488020463346C0472068039B0E930F953D
:109A1000856C4B463A4631462046AC4605B0BDE81B
:109A2000F04F60472DE9F04F87B01746BDF9404031
:109A300000912546E91D059344BF2B4603F10E0115
:109A40000268BDF8486053690294C91003912B491C
:109A5000BDF9444001968B42824645D1002C3CDD45
:109A6000029B3C445E1EB6B24FF0000923B2049341
:109A700001364D46029B002B28DD059B002403EB9D
:109A8000090806E0EDB22B0604F1010411D4A64248
:109A90001CD0A1B211F0070F23B24FEA4505F1D156
:109AA000002BB8BF0733DB10013418F803502B0626
:109AB000EDD5009BD2F818B019443A4609B2019B83
:109AC0005046D847A642DAF80020E2D1039B01377E
:109AD0009944049B3FB2BB42CCD1D36A074A93421C
:109AE00006D107B0BDE8F08F9847DAF80020B5E757
:109AF000504607B0BDE8F04F184700BFF996000088
:109B000070B4BDF90C60BDF91050BDF81440039657
:109B10000495059470BCFFF785BF00BF2DE9F04F99
:109B200093B090460591C1691090BDF87000079000
:109B3000BDF874909DF878A00493002900F0CD80C2
:109B40000A7A0AC9894604998A1AD2B203EBC20377
:109B5000BAF1010FDA780B9293F905201E8893F879
:109B600002B00F9293F9064079D913B2099323B248
:109B70000C93109B1A68A94B1193194653698B4299
:109B800040F0A6800B9B002B55D01FFA88F30021D4
:109B90000D93C8462344DDF8409006910E930F467E
:109BA0000C46BBF1000F3FD0BDF818100C9B03977B
:109BB0001FFA8AF0CB1813FB00F304900E980144AF
:109BC0000D98034409B21BB20A910893002505E0E1
:109BD0000135EBB264009B45E4B222D9039B2B44D0
:109BE000590703D1731C18F806409EB22306EFD51F
:109BF000099BBDF81000E91811FB00F10598BAF1B6
:109C0000010F0FFA8AF301441CD0079801900093CA
:109C1000D26909B217464846089AB847D9F80020D1
:109C2000D6E7039F5F44FFB2069B0B99013306936F
:109C3000DBB29942B5D8D36A119A934243D113B09B
:109C4000BDE8F08F0F9B191893690A9A29441F46A3
:109C500009B2079B4846B847D9F80020B8E7002367
:109C60000C93099385E70A9A0D9B0132013B52B28E
:109C700013F0FF030A920D936FD1DDF81890079B44
:109C8000DDF83C80DDF820A04B4517D0BAF1010F7C
:109C900000F0C8800B9A109DCDF804900BEB8B015F
:109CA0004FEACB030A4400931146DEF81C405346AA
:109CB000424609B22846A047D5F800E0DEF82C302D
:109CC000119A9342BBD0109813B0BDE8F04F1847DB
:109CD000109D284698472A6854E7109A0598B2F9CB
:109CE0000A308342ABDDB2F90C304345A7DD0623D1
:109CF00013FB0A03002BA2DD08EBCA03002B9EDD39
:109D0000537E2BB9049BAF2B02D90133DBB20493F2
:109D1000109BD3F800E0414B11931A46DEF8143043
:109D2000934240F08E801FFA88F30E9308339BB263
:109D3000BDF81420059305230D9300230A93CDF855
:109D40003C800FFA8AF3DDF84080CDF818900B9232
:109D50001FFA8AFBCDF820A099460A9ABDF8100098
:109D60000B9C0E9D0523194611FB00232C48114620
:109D7000C75C039702FB0B4214FA81F312B21BB2C9
:109D800009920C932C462E461CE0089B0999012B46
:109D90002AB24B4640462DD0079F0197CDF8009040
:109DA000DEF81CA0D047D8F800E0039B5B08013424
:109DB0000393059BA4B25D445E44A342ADB2B6B228
:109DC0003FF451AF039BD807DFD4079B069A934219
:109DD000EBD0089B012B16D0069B0193CDF8009089
:109DE000DEF81CA009994B4632B24046D047D8F85D
:109DF00000E0DAE7DEF818A0079B0C9922B2D04702
:109E0000D8F800E0D1E7DEF818A00C9913464046D8
:109E100022B2D047D8F800E0C7E700BFF9960000AB
:109E2000900801000B99109DCDF800900531DEF8E7
:109E3000204009B2424608232846A047D5F800E052
:109E40003CE7109C20469847D4F800E06BE700BF41
:109E5000F0B5C36985B004462BB30A2968D00D2933
:109E60004AD01A7A914247D3587A884244D35D68DF
:109E70008A1A05EBC205AA78002A50D0E878002893
:109E80004DD0207E00283AD095F905E0B4F90E00B7
:109E9000A67DB4F90A70724406FB0202BA4262DC83
:109EA000B4F9102030E00A2956D00D2924D0027EC2
:109EB000002A4BD0B0F90E00A57DB4F90A60062245
:109EC00012FB0502B2423EDD228AE38102EBC502AB
:109ED00012B218462282A78A668A02950B468DE83E
:109EE000C00001462046FFF719FEA37DE28903EB7F
:109EF000430302EB4303E381012005B0F0BDA67DDF
:109F0000B4F90E00B4F91020B4F814E0678A029690
:109F10000B468DE8804001462046FFF7FFFD29797A
:109F2000E389A27D012001FB0233E38105B0F0BD8E
:109F30000022C2819A7A817D038A01FB0233038267
:109F4000012005B0F0BDB4F91020C4E7857DB4F957
:109F50001020B0F90E00BEE7028A817DC38102EBBA
:109F6000C1030382C8E70020E0819B7A228A03FBB9
:109F7000062212B22282C7E7C1810282704700BF67
:109F8000002908BF01218175704700BF818241828D
:109F9000704700BFC07D7047B0F90A00704700BF2E
:109FA000B0F90C00704700BF10B4EFF3108272B626
:109FB000437F33B9017F012907D003290FD0012343
:109FC000437702B962B610BC7047124C2168A1B148
:109FD000114943610B68836108605861EFE70F4CDA
:109FE000216881B10E4943610B6883610860586143
:109FF0000C4B4FF080511960E1E7074B41618161E3
:10A0000020601860DBE7064B4161816120601860C9
:10A01000EEE700BFD89EFF1FD49EFF1FC89EFF1F04
:10A02000CC9EFF1F04ED00E070B5EFF3108272B616
:10A030000C4C206880B10C4E00254369236073B13D
:10A040009D6102B962B6457783689847EFF3108245
:10A0500072B620680028F0D102B962B670BD3360D4
:10A06000EFE700BFC89EFF1FCC9EFF1FFFF7DCBFBE
:10A07000184A30B41468002C27D0036821688B423A
:10A080000ED2CB1A00218460C1602360E0601060B2
:10A090000223037530BC704711688B42144608D305
:10A0A000A2685B1A0360002AF6D18260C460A060D7
:10A0B000EEE7D268C2608460E060C568CB1A022215
:10A0C000A8602360027530BC70478460C460106073
:10A0D000DEE700BFD09EFF1FF8B5224E34682CB3D8
:10A0E0002368002B3AD1204F1D4604E03468ECB1C0
:10A0F0002368002B32D1A36803B1DD60206933608F
:10A10000036825751B68BB4221D1037F4560022B84
:10A11000C46020D0FFF748FF6368002BE6D02360BF
:10A120002046FFF7A5FF3468002CE1D1EFF3108340
:10A1300072B60E4A00211068116003B962B628B1E8
:10A140008468FFF795FF20460028F9D1F8BD224624
:10A1500000219847E0E783689847DDE7013B2360EB
:10A16000E4E700BFD09EFF1FE9870000E09EFF1FCD
:10A17000024A136801331360FFF7AEBFEC9EFF1F66
:10A18000704700BF0368F0B4FBB1002501249D6057
:10A19000DC601B4C1A601C44241104F144056A1154
:10A1A000032692009E60174F0679174B47F824103C
:10A1B00002F1604202F5614205F01F05012000FA3C
:10A1C00005F5E6541560F0BC7047104C236843F465
:10A1D0000003236000BF0E4B0E4DA4F58734A4F599
:10A1E0009E7401261E60234604609C68002CD0D01B
:10A1F0001033AB420360F8D1002303601846E2E756
:10A20000008FFCBF3891FF1F44E400E03C80044015
:10A2100000700340407103400168A9B10B4BF0B4DA
:10A220000B441B110A4E0B4F0B4D46F8237003F1E4
:10A23000440202F01F0401235211A340002445F8F8
:10A2400022308C600460F0BC704700BF008FFCBF00
:10A250003891FF1F81A1000080E100E0024A034B1A
:10A26000012111601B6818470C7103403891FF1FD2
:10A27000024A034B012111605B6818471C710340BF
:10A280003891FF1F024A034B012111609B68184758
:10A290002C7103403891FF1F024A034B01211160CA
:10A2A000DB6818473C7103403891FF1FF8B50E4634
:10A2B00071B17AB10746144600253B6816F8011BB8
:10A2C0001B6838469847013C0544F6D12846F8BD3E
:10A2D0000846F8BD1046F8BD00B5064A0368128866
:10A2E0005B6883B001A9ADF804200222984703B04F
:10A2F0005DF804FB900D0100F0B507468BB0002A15
:10A3000033D0012A08BF0A2251B3212400E0F4B25D
:10A31000B1FBF2F502FB1511C8B2092900F13001B9
:10A3200098BFC8B20AA988BF3730214488BFC0B2DD
:10A3300001F8240C661E2946002DE8D133B1013CFA
:10A34000E4B20AAB23442D2203F8242C3B6801AA73
:10A3500011195B683846C4F1220298470BB0F0BD72
:10A3600030228DF825202124E8E70368C9B21B6854
:10A3700098470BB0F0BD00BF0029BABF49422D235A
:10A3800000230A22FFF7B8BF374A384913681B0673
:10A39000FCD40B6813F08003F8D172B634490A7804
:10A3A000002A5FD0334A3448F0B4344C176806684A
:10A3B0002568D4680C303E44143200681268304F6F
:10A3C00035442C4420440244C2F34E022D4E2E4804
:10A3D0002E4D2F4C42F400423A60376806682D68D3
:10A3E0002C4A24680C303E44006812682A4F3544D9
:10A3F0002C4420440244C2F34E02284E2848294DE2
:10A40000294C42F400423A60376806682D68274AB2
:10A4100024680C303E4400681268254F35442C44B3
:10A4200020440244C2F34E02224E2348234D244CC2
:10A4300042F400423A60376806682D68214A246871
:10A440000C303E440068126835442C4420440244D9
:10A45000C2F34E021C4842F4004202600B7062B626
:10A46000F0BC704762B6704724B0034024B00B4084
:10A47000E59EFF1F38B003403CB0034040B00340AE
:10A480002CB0034058B003405CB0034060B00340C0
:10A4900064B003406CB0034030B0034038B00B40B0
:10A4A0003CB00B4040B00B4044B00B404CB00B40B4
:10A4B0002CB00B4058B00B405CB00B4060B00B4070
:10A4C00064B00B406CB00B4030B00B4030B4294846
:10A4D000294A2A4B2A4D6024E121047011701B780F
:10A4E000284C082B30D00A2B2748284937D00C2B72
:10A4F0000CBF35223D2212232A60236002600B60CC
:10A50000234B24491B78244ABBB101230B60136001
:10A51000224B23491B78234A012B26D9042B0FD920
:10A52000082B1ED9102B94BF862387230B60136042
:10A530001D4B01221A7030BC70470B601360E7E7B7
:10A5400084230B601360F3E700F58E200F49083079
:10A55000012213232A60236002600B60D0E73922B6
:10A56000F7E785230B601360E2E780230B6013603D
:10A57000DEE700BF00400740014007404891FF1F51
:10A5800008B003400CB0034008B00B400CB00B40C7
:10A59000E89EFF1F20B0034020B00B404991FF1FF1
:10A5A00024B0034024B00B40E59EFF1F0C2830B4BC
:10A5B00017D91023984228BF18461C46104A114D3F
:10A5C0001178181A8C42287018D00F4913700B7824
:10A5D00023B10E490E4A00230B60136030BCFFF715
:10A5E00075BF0A2802D90C231C46E7E7082802D9C0
:10A5F0000A231C46E2E708231C46DFE730BC70470D
:10A600004891FF1FE49EFF1FE59EFF1F24B00340FB
:10A6100024B00B4028282FD8334B2DE9F0411E5C85
:10A62000FF2E2BD0314B1B78002B2AD132062CD495
:10A6300072B62F4D2F4C2F46012326602B7062B629
:10A6400072B623681B060CD43B781BB9F4E72B7851
:10A65000002BF1D062B602F09BF972B6236818069F
:10A66000F5D5254B1B6800222A7062B6234A107864
:10A6700043FA00F0BDE8F081002070470020BDE8FB
:10A68000F081FFF781FE3206D2D572B61C4DDFF89D
:10A690007C801C4C06F04007FFB206F03F06D8F85D
:10A6A0000030DFB123F01003C8F80030012326602A
:10A6B000134A2B7062B672B6236819060CD413784D
:10A6C0001BB9ECE72B78002BE9D062B602F060F9F9
:10A6D00072B623681B06F5D50B4BC3E743F0100396
:10A6E000C8F80030E2E700BF940D0100E59EFF1FAF
:10A6F000E79EFF1F00B0034010B00340E49EFF1F21
:10A70000E69EFF1F00B00B4010B00B400CB00B409A
:10A710000A4A0B49136843F4805313600B7843B91A
:10A72000084BC0221A70084B80F30C0000B218804E
:10A730007047044B80221A70F5E700BF2C8004405C
:10A74000E89EFF1F21C00C4000C00C40F0B51B4B21
:10A750001B4E596818689A68DB6885B06C460FC450
:10A76000337899071DD5174A174C1378174913F0FA
:10A77000700318BF1370164A164B802717700026F7
:10A780003320032226706D4608701A7072B6043C9E
:10A7900045F001052046A84762B6237813F0700300
:10A7A00009D10D4B064901E0013B02D00A78D207DE
:10A7B000FAD505B0F0BD237005B0F0BDC00D0100A5
:10A7C0000100024000000240040002400B00024071
:10A7D000070002400A000240410D0300B0F5006F7F
:10A7E0000AD210B5094B1B78DB07044606D504F1E5
:10A7F000A0500078C0B210BD00207047FFF7A6FF40
:10A8000004F1A0500078C0B210BD00BF01000240AA
:10A81000B0F5006F17D238B50F4B1B78DA070D462D
:10A82000044611D504F1A0500378AB420AD00B4A7C
:10A83000137813F0700318BF1370074A057013786C
:10A84000DB07FCD538BD7047FFF780FF04F1A0504F
:10A850000378AB42EBD1F5E7010002400000024073
:10A8600008B5F5F721FFF7F7ADFD02F091F8FAE72B
:10A87000844641EA000313F003036DD1403A41D30B
:10A8800051F8043B40F8043B51F8043B40F8043BCA
:10A8900051F8043B40F8043B51F8043B40F8043BBA
:10A8A00051F8043B40F8043B51F8043B40F8043BAA
:10A8B00051F8043B40F8043B51F8043B40F8043B9A
:10A8C00051F8043B40F8043B51F8043B40F8043B8A
:10A8D00051F8043B40F8043B51F8043B40F8043B7A
:10A8E00051F8043B40F8043B51F8043B40F8043B6A
:10A8F00051F8043B40F8043B51F8043B40F8043B5A
:10A90000403ABDD2303211D351F8043B40F8043BF9
:10A9100051F8043B40F8043B51F8043B40F8043B39
:10A9200051F8043B40F8043B103AEDD20C3205D309
:10A9300051F8043B40F8043B043AF9D2043208D001
:10A94000D2071CBF11F8013B00F8013B01D30B8873
:10A9500003806046704700BF082A13D38B078DD051
:10A9600010F003038AD0C3F10403D21ADB071CBF23
:10A9700011F8013B00F8013B80D331F8023B20F88D
:10A98000023B7BE7043AD9D3013A11F8013B00F8C6
:10A99000013BF9D20B7803704B7843708B7883704E
:10A9A0006046704708B5104C08E0236859050DD47F
:10A9B00023681A050FD42368DB0411D423685803D5
:10A9C000F3D500F08DFE23685905F1D502F044F867
:10A9D00023681A05EFD502F0D5F82368DB04EDD51E
:10A9E00000F0F0FCEAE700BF3480044008B5FFF750
:10A9F000D9FF00BF014B10221A807047002005408C
:10AA0000704700BF094908B50B6830B16A46184461
:10AA1000A2F58052904202D20860184608BD03F0A9
:10AA200065FB0C2303604FF0FF3008BD4C91FF1F06
:10AA3000FEE700BFEFF3138070B9EFF310836BB93B
:10AA4000EFF305825AB94FF48070EFF311832BB105
:10AA5000984228BF184670474FF0FF3070470F2AC2
:10AA600001D81846F1E7014BD05CEEE7F0E300E0D7
:10AA7000F0B44D1E2E46002400E00134B0FBF2F38A
:10AA800002FB1300092800F130078ABF3730F8B203
:10AA9000C0B206F8010F1846002BEED10A19537008
:10AAA0004CB1107815F8016F28700133E01A834219
:10AAB00002F80169F5DB0846F0BC7047704700BF3B
:10AAC00010B40F4B53F8302092F880422CB1012380
:10AAD00069B182F8803010BC704703EBC0035B683B
:10AAE0001A6841B922F002021A6010BC704782F85D
:10AAF000003110BC704742F003021A6010BC70476E
:10AB0000D00D01001C4A02EBC00301295B6811D083
:10AB100004291BD052F83000002280F8802229B18D
:10AB2000022920D0032922D01A6070474FF4807286
:10AB30001A60704752F830004FF4A27280F8801209
:10AB40001A601A6822F020021A60704752F830101A
:10AB50004FF4A272012081F880021A601A6842F054
:10AB600020021A60704740F203121A6070474FF4D7
:10AB700081721A60704700BFD00D0100212848D8AB
:10AB8000F8B5042A44D8DFE802F0484B4E034500EC
:10AB90004FF410262B4B03EBC0030D465C68216875
:10ABA00011F4E06148D0284B284A2949C3F89C2178
:10ABB00004F140422748C3F8A411A2F59221264F80
:10ABC000C3F8A0017C292548C3F8A871C3F8AC01DB
:10ABD0002CD9A2F594237C2B2AD9A2F596237C2B81
:10ABE00028D9A2F598237C2B29D9A2F59A227C2A70
:10ABF00027D81B4872B6236823F4702343F0807271
:10AC0000C4F384011643236040F82150266062B6E5
:10AC1000F8BD70474FF43026BCE74FF40026B9E783
:10AC20004FF44026B6E74FF42026B3E70D48E1E79E
:10AC30000D48DFE70D48DDE7FFF764FFB3E70C4899
:10AC4000D8E7F8BDD00D01000082FF1FF188FF1F7B
:10AC50009988FF1FC588FF1F6D88FF1F4188FF1F50
:10AC60002892FF1F5091FF1F8891FF1FD891FF1F4F
:10AC70000892FF1F1A4B03EBC00010B4426802F1A8
:10AC80004043A3F592217C2923D9A3F594217C2963
:10AC90000DD9A3F596217C291FD9A3F598217C29EC
:10ACA00019D9A3F59A237C2B11D80E4C00E00E4C39
:10ACB00072B613680D4823F08773C2F3840123F43E
:10ACC000803343F08073136044F8210062B610BCF7
:10ACD0007047074CECE7074CEAE7074CE8E700BF92
:10ACE000D00D01002892FF1F8891FF1FBDAA000010
:10ACF0005091FF1F0892FF1FD891FF1F30B4054BE2
:10AD0000054D064C002210211A602A60206019604F
:10AD100030BC704714D0034004D0034000D003403F
:10AD2000282838B52ED0002904464FDD5F4B1B780C
:10AD3000012505FA03F28A4202D8212837D938BD05
:10AD40000338C2B2012A3AD9202C4AD0192C48D053
:10AD5000574A126802FB011222FA03F31D2800F27F
:10AD60009B80DFE800F0928B847D9999766F9999AA
:10AD70009999999999999968615A53994C9999997E
:10AD800099999945494B1B780B2B08D90C2B1CBF63
:10AD90000C3B19410846BDE83840FFF7B9BCC3F188
:10ADA0000C0399400846BDE83840FFF7B1BC29467E
:10ADB000FFF786FE2946BDE83840FFF7A3BE3D4AAF
:10ADC000126802FB011222FA03F3C7E72128B6D862
:10ADD0000021FFF775FE20460121BDE83840FFF74E
:10ADE00091BE354A126802FB011222FA03F3B5E75D
:10ADF0003249334A0B604FF45173136038BD314907
:10AE0000314A0B604FF45173136038BD2F49304AFB
:10AE10000B6040F24443136038BD2E492E4A0B604C
:10AE200040F24443136038BD2C492D4A0B6040F278
:10AE30004443136038BD2B492B4A0B6040F2444316
:10AE4000136038BD29492A4A0B6040F2444313601D
:10AE500038BD2849284A0B6040F24443136038BD8E
:10AE60002649274A0B6040F24443136038BD254908
:10AE7000254A0B6040F24443136038BD2349244AFD
:10AE80000B604FF45173136038BD2249224A0B60A6
:10AE90004FF45173136038BD212C3FF650AF7F291A
:10AEA000D4BF00210121204693E700BF3092FF1F4D
:10AEB000088003400890034008800B4010800B403E
:10AEC00048A0044018800B404CA004401880034068
:10AED00008B004401080034004B0044040800340A8
:10AEE00018C004403880034014C004402880034048
:10AEF00010B00440208003400CB004403080034078
:10AF000010C00440488003401CC004401890034017
:10AF100034900440109003403090044038B1102821
:10AF200028BF1020044AC3B2107813707047024A39
:10AF300001231078137070473092FF1F2DE9F843FA
:10AF40000E4680463249334D304603F055F847F6F9
:10AF5000122300281ABF1D464FF002094FF00109C5
:10AF6000002425FA04F002F051FE4FF05E5107462E
:10AF700002F0A4FE0146304603F052F830B9013425
:10AF8000072CEED1E80902F041FE0746314638466B
:10AF900002F048FF4FF07C5102F086FD03F07AF892
:10AFA0004FF6FF729042A8F1030328BF1046012B11
:10AFB00029D9B8F1170F17D8174B23FA08F303F064
:10AFC000010383F0010223B9B8F1190F0FD0BDE8D6
:10AFD000F883124B124D13491A6044EAC9042A60DF
:10AFE00008601C60BDE8F883B8F1200FECD10E4B6F
:10AFF0000E4D0F49002244EAC9041A602A60086015
:10B000001C60BDE8F8830B4B0B4D0C49F2E700BF09
:10B01000001BB740006CDC026006F00000800340BB
:10B02000048003400880034000800B4004800B40F4
:10B0300008800B40009003400490034008900340B8
:10B04000212801D8FFF73CBD704700BF212806D852
:10B05000044B53F8303093F80002C0B27047002020
:10B06000704700BFD00D0100212801D8FFF74ABD6D
:10B07000704700BF72B60C490C4B0D4A1B6808683C
:10B08000126862B6520102D5322B88BF01300949DD
:10B09000C3F5BB334FF47A72FF33A1FB031302FBFA
:10B0A00000F000EB93107047EC9EFF1F18E000E0EB
:10B0B00004ED00E0ABAAAAAA2DE9F843054672B652
:10B0C000204F214B214A1B683C68126862B652012E
:10B0D00002D5322B88BF013495B3C3F5BB331C4E68
:10B0E000DFF86490DFF86480FF334FF47A72A6FBD8
:10B0F000031302FB04F404EB931472B6D9F80010A6
:10B100003A68D8F800E062B6C1F5BB33FF33A6FB5E
:10B1100003031EF0806FC4EB93134FF47A7002D0D8
:10B12000322988BF013200FB0233B3F57A7F04D3A2
:10B13000013D05D004F57A74DFE701F029FCDCE776
:10B14000BDE8F883EC9EFF1F18E000E004ED00E08E
:10B15000ABAAAAAAF8B52D4B2D49DFF8D0E0DFF84D
:10B16000D0C02C4E2C4D2D4C2D4A2E4F4FF40000AC
:10B1700018604FF0807018604FF0007018604FF04A
:10B18000806018604FF0006018600020086028237D
:10B190004BF6FF71CCF80010CEF80030336013602E
:10B1A0002B6023603B60B3629362092245F8242C34
:10B1B000C4F8D80F05F57F65C7F8D41F07F5FF273A
:10B1C00007F5FA67C6F8F83F2B6006F5FF26C4F8C6
:10B1D000D42F05F5FD2504F5FF24386006F2F4763A
:10B1E0001148316005F5FF6504F5FD642B602360AF
:10B1F0000260FFF76BF91920FFF75EFF00F0B6FF62
:10B2000040F21310BDE8F840FFF756BF08E100E038
:10B210000480034014800340248003402C800340BA
:10B220001C8003403480034000800B400C800340AE
:10B23000088003402DE9F84F214B1B6807460BB1EE
:10B2400001221A70DFF888901E4D99F80040DFF84F
:10B2500084801D4E0134272C8ABF4FF0000A5FFA0C
:10B2600084FA5446AB462B78A34216D1FFF7E2FB93
:10B2700040281FDC33791B06F5D59BF800300133DD
:10B28000272B86BF00221346DAB218F80330DBB250
:10B29000F3712A702B78A342E8D00C490A4BFFB215
:10B2A00008F804700120AC22087089F800A0DA7058
:10B2B000BDE8F88FFF28D6DD01F06AFBD3E700BFB9
:10B2C000649FFF1F619FFF1F00C00640609FFF1F1C
:10B2D000689FFF1FF89EFF1F1C4BDFF894C01A6881
:10B2E0001B49F0B542F480521A4D1A60DFF884E031
:10B2F000194F1A4E1A4C00238CF800304FF451723B
:10B300002B701F2840F213358EF800303B703370DD
:10B3100025600A6012D819460124124A124D117094
:10B320001248547000212C27402693724FF40034A9
:10B3300091701174D7702E700460F0BDC0F3443169
:10B34000C0F3471400F01F03E7E700BF3480044058
:10B350000CC00440F59EFF1F619FFF1F609FFF1FF1
:10B3600008C0044000C0064031E400E004E100E011
:10B37000F49EFF1F689FFF1F034B1B68DB0401D572
:10B38000FFF758BF704700BF3480044010B5044C2D
:10B39000237823B101F0FCFA2378002BFAD110BDF9
:10B3A000609FFF1F054A064B10781B78C0B2DBB2C6
:10B3B000984238BF4030C01A704700BFF49EFF1F4C
:10B3C000F59EFF1F30B42B4B1A7994061FD52A48DF
:10B3D000DA790378294901333F2B0978C8BF002364
:10B3E0008B42D2B203D0264CD9B2E2540170254A26
:10B3F000116861B1244A1278D2B2934236BFC2F1C9
:10B4000040029B1A9B18272BC4BF01230B70194ABB
:10B41000D378DBB2180611D45A060DD5154B1B791B
:10B420005B0609D5194B1A491B6800220A7003B143
:10B430001A70104B2C22DA7030BC70471179090653
:10B44000EAD5144910480C780178C9B28C420DD065
:10B450004A1C272A84BF00210A460F4D054C98BF7D
:10B46000D1B2AA5CD2B2E2710170D5E76C21D17081
:10B47000D2E700BF00C00640F49EFF1FF59EFF1FED
:10B48000209FFF1FF09EFF1F619FFF1F649FFF1FF4
:10B49000609FFF1F689FFF1FF89EFF1F21282FD866
:10B4A000184B195CFF292BD0174B184ADFF870C0D6
:10B4B00003EBC000F0B54368DFF868E0144F154DAA
:10B4C000154E00241C60DEF80030012043F02003FC
:10B4D0008840CEF8003014604FF4A07338602E60BE
:10B4E000C2F800C0013BFDD113689B05FCD42023AA
:10B4F000013BFDD1094B09B233F8110080B2F0BD18
:10B5000000207047E00E0100D00D01000050044003
:10B51000085004400450044000000203005104405D
:10B5200080014A0038800440431E032B14D872B6B1
:10B530000A4951F8230068B170B4094C058834F801
:10B540001320466841F82360521B24F8132062B68A
:10B5500070BC704762B6704700207047C49FFF1FE1
:10B5600008A2FF1F013803280BD872B6074B53F807
:10B57000203043B100205B680130002BFBD162B664
:10B580007047002070471846F9E700BF18A0FF1F5A
:10B5900030B472B62B4A13781D0706D52A4B196AA8
:10B5A000002936D0996A002941D053781C0706D566
:10B5B000254B196C00293ED0996C002939D093781D
:10B5C000190705D5204B196E002936D0996E89B11F
:10B5D000D3781B0707D51C4BD3F880207AB3D3F858
:10B5E000882011213AB162B6184B00221A7030BC83
:10B5F00000F04ABE0D21154C154D227843F831500C
:10B6000003EBC1030830013A5860227062B630BCC7
:10B61000704704220D4C0F4D217843F8325003EB54
:10B62000C20308304A1E5860227062B6EFE7052157
:10B63000E1E70921DFE70822ECE70C22EAE7102224
:10B64000E8E700BF040F01000080FF1F41A0FF1FBB
:10B65000C800400088004000431E032B1DD81B4A31
:10B66000400140F0100030B4104472B6184CE25C57
:10B67000032A1BD8DFE802F00212151703220D88F7
:10B68000E25410F0080F14BFC823882343EA05438F
:10B6900008310360416062B630BC70470830022256
:10B6A000EDE70522EBE708300422E8E7094A52F803
:10B6B000230038B1084A52F82300416042F82310B1
:10B6C00062B6E9E742F82310034AF7E70080FF1F5C
:10B6D00050A0FF1F18A0FF1F28A0FF1F00BE70472B
:10B6E0002DE9F04FDFF818B3DFF818A387B044E076
:10B6F000AD4F4FEA930807EBC809013ED9F8042083
:10B7000003F00803F6B2A2F1080003F0FF04002BD7
:10B7100040F0018157F838301B0C99B222F8081C10
:10B72000002B00F0EF80A14B22F8064C42F8044CAD
:10B7300053F82620002A00F0CF819D4D55F8263081
:10B7400058609C4C45F8260034F81630194424F80B
:10B75000161000F079FD002800F0C281964A974B40
:10B7600019F0080F00F1080018BF1346C9F80400CB
:10B7700047F8383008238BF800309BF80040E4B2DB
:10B7800065071CD58E4B1B78B3B18E490A7802F041
:10B79000FF0322B1013BDBB20B7003B900BE8A4943
:10B7A0000A7802F0FF032AB1013BDBB20B70002BD9
:10B7B00000F0688100F066FE04238BF8003004F08E
:10B7C000080303F0FF02002B00F0C9809AF8003054
:10B7D000DBB21E098CD19A08DFF8CC9159F83210EF
:10B7E00009EBC200C1F38301013940680C2900F262
:10B7F0008580DFE801F07A7A8383838383834683BD
:10B80000838307000168714D4068714F714E686015
:10B81000296088B240F281610024674B49F83230D8
:10B820004FF0010E88423C60C9F81040C9F818403A
:10B8300086F800E05C4A00F2E780B0F5D06F80F057
:10B840001B82B0F5817F00F0D98100F269818028E8
:10B8500000F02A82822840F0D781A98801F07F0178
:10B86000042900F2D1815C485C4A890008441470C4
:10B87000547001788C0740F1608382F800E0022167
:10B8800073E1534F3A682AB3554B524E55481988C5
:10B890003478057840298E4645F0020828BF4FF0DD
:10B8A000400E002C84F001043470CEEB01010CBF7B
:10B8B0008824C82409EBC80689B285F0010544EA4A
:10B8C0000E447260198049F83840724405700029AE
:10B8D00065D03A603D4B1A88B2F5A06F0ED10021B9
:10B8E0009A785970404B1A7008E038493F4C0D68FF
:10B8F000A54200F09880304949F832103C4A0123B3
:10B90000137037E72C4A2D4B19F0080F18BF134658
:10B9100047F838302EE700F0B7FC364A364952F87F
:10B920002630002B00F0E38058688C5D42F826003A
:10B9300003F10802C9F80420032C05D8DFE804F05D
:10B940002C02292602228A551A8819F0080F0CBFEA
:10B950008823C82343EA024347F838300AE7E00760
:10B9600000F19380210600F1D180A20706D5234A79
:10B97000234913780220DBB213700870E30602D566
:10B980001F4B10221A7007B0BDE8F08F04228A55B1
:10B99000DAE705228A55D7E703228A55D4E7BEF1B4
:10B9A000400F18BF002294E70080FF1FC49FFF1FB5
:10B9B000709FFF1F08A2FF1FC800400088004000C2
:10B9C0004CA0FF1FD59FFF1FC0A0FF1F38A0FF1F67
:10B9D0006C9FFF1FD49FFF1FC020074044A0FF1F84
:10B9E000809FFF1F40A0FF1F9820074021090003F0
:10B9F0009420074018A0FF1F50A0FF1F8820074079
:10BA00008020074090200740B0F5106F00F07C8147
:10BA100040F2A38040F62112904240F07B82A54A7A
:10BA2000012313706AE74C68A3498C427FF463AF2B
:10BA30000178A9297FF45FAF417845297FF45BAF96
:10BA40008178C2297FF457AFC1786B297FF453AF57
:10BA50009A489B4E0178347881F00105002C41F022
:10BA6000020105700CBF8820C82084F0010449F849
:10BA7000310009EBC10193483470002505244D6065
:10BA8000047038E700F064FF94E68F4B89488B49D7
:10BA90001A614FF0020E80F800E08C4F0A708C495A
:10BAA000196099608B4E8C4D8C4C9A610D213970C8
:10BAB000FF213170DFF84CE229702270884D894AED
:10BAC0008EF800109F27012406F8047C5D60047046
:10BAD000DA6007B0BDE8F08F43F82600824D30E60B
:10BAE000824A47F8380013780133137042E68B5DC1
:10BAF000032B00F2BA8001A252F823F075B70000C0
:10BB000075B7000055BB00004FBB00006F49724B7A
:10BB100080220D2008701A70A2077FF52FAF26E74C
:10BB200040F20232904240F0ED81AA8802F07F029A
:10BB3000042A69D86D88002D66D16449CDF804E0E7
:10BB4000920011440A7842F002020A70C1E1012316
:10BB50008B550FE600238B550CE6B0F5086F53D1DB
:10BB60006349644A097811707146ED888D4280F00E
:10BB7000E88252480478402DAE4644F0020C28BFBB
:10BB80004FF0400E02EB0E0309EBCC0102930123B0
:10BB90004A604FEA0E48CEEB050101930025C8220A
:10BBA00042EA080384F0010249F83C303570027023
:10BBB000DFF814C1424BDFF8048149BBBEF1400FEE
:10BBC0007FF42DAF42F0020C09EBCC03029ADFF8B0
:10BBD000F8E05A608DBB0D0445F088059DF80430EF
:10BBE0004EF83C500A4433700470134640297FF4E9
:10BBF00016AF0021404A3B60118010E7AA8802F08E
:10BC00007F02042A40F28B81304A0F23137006E72B
:10BC10004029D7D942F002020CEBC200029E4660D6
:10BC2000BDB19DF8045035481D703346403988F841
:10BC3000004040334CF83200DCE79DF804303370AC
:10BC40000D04029B047045F0C8050B444EF83C50AF
:10BC5000CCE79DF804501D70029B1D4888F80040F9
:10BC6000403940334CF83200C4E719F0080F0CBFDC
:10BC7000022303238B557DE521494A68002AC3D05E
:10BC80006C88B5F804E003E00C314A68002ABBD0A8
:10BC90000B88A342F8D14B887345F5D1240A032CB5
:10BCA0000CBF1178098960E7124A022114705470A0
:10BCB0005BE700BF942007400100040040A0FF1F85
:10BCC000D49FFF1FD59FFF1F0080FF1FC02007408C
:10BCD00088004000882007408020074098200740C7
:10BCE000849FFF1FD89FFF1F709FFF1F41A0FF1F52
:10BCF0004CA0FF1F44A0FF1F809FFF1FC8004000F3
:10BD0000080F01008C200740B248116AAC7804701B
:10BD10000C0600F19881D9F82820AF49100600F1EF
:10BD2000DB81D9F83020AC49120600F1D081D9F876
:10BD30003820A949130600F1C581D9F84020A64949
:10BD4000150600F1BA81D9F84820A349140600F17C
:10BD5000AF81D9F85020A049100600F1A481D9F88C
:10BD600058209D49120600F19981D9F860209A491E
:10BD7000130600F18E81D9F868209749150600F165
:10BD80008381D9F870209449140600F17881D9F89C
:10BD900078209149100600F16D81D9F880208E49F4
:10BDA000120600F16181D9F888208B49130600F151
:10BDB0005581D9F890208849150600F14981D9F8B4
:10BDC00098208549140600F1FF808448844A8549FB
:10BDD00001908548854D864C049700230596029571
:10BDE00080460F4616461D460394306828B14468C5
:10BDF00000F04AFA2046002CF9D100233360029B60
:10BE000038681A46002342F8253028B1446800F00B
:10BE10003BFA2046002CF9D100223A60019A98F8AA
:10BE200000301146002241F8042B039A0191023B95
:10BE30004FF0000122F81510032B07D8DFE803F0BC
:10BE40005D025D024FF0010388F800300135042DDA
:10BE500006F1040607F1040708F10108C5D1654C95
:10BE6000654D2278654B049F059E002110072970BF
:10BE70001A7000F19280624962780A700021C9F854
:10BE80003010C9F838101107DFF84C816ED4A27851
:10BE90005C49DFF844810A7000211207C9F850108C
:10BEA000C9F858104BD4E27857494B4C0A70130725
:10BEB0004FF00001C9F87010C9F8781000F1AE8099
:10BEC00033780193002283F00105C9F89020C9F866
:10BED00098200021029188468E460A464B480478F5
:10BEE00044F0020C09EBCC030393019B002B039B52
:10BEF0005A600CBF8822C82252E64FF0000388F82F
:10BF00000030A3E7B0F5A06F7FF47EAE01230025DB
:10BF10000193DEE740F621229042F7D074E66D8867
:10BF2000002D7FF471AE3A49CDF804E0920011443F
:10BF30000A7822F002020A70CBE7022115E600F02F
:10BF400083F9002800F0EB800830324AC8F864001A
:10BF5000C8F8602000F078F9002800F0DA80083096
:10BF60002D4AC9F86C00C9F868209CE700F06CF90C
:10BF7000002800F0E0800830264AC8F84400C8F8DD
:10BF8000402000F061F9002800F0CF800830224AFC
:10BF9000C9F84C00C9F8482079E700F055F90028A5
:10BFA00000F0A58008301B4AC9F82400C9F82020F9
:10BFB00000F04AF9002800F094800830164AC9F8C9
:10BFC0002C00C9F8282056E7D1F89C00083800F06A
:10BFD0005BF9FAE64CA0FF1F0080FF1F28A0FF1F9F
:10BFE000C49FFF1F18A0FF1F50A0FF1F709FFF1FBF
:10BFF00008A2FF1F040F010041A0FF1FC42007403B
:10C00000C8200740CC200740D020074040A0FF1F99
:10C01000C020074088004000C800400000F014F92C
:10C02000002870D008304F4AC4F88400C4F880203B
:10C0300000F00AF9002860D008304B4AC9F88C009B
:10C04000C9F888203CE7506A083800F01DF962E61C
:10C05000D1F89400083800F017F9B0E6D1F88C0058
:10C06000083800F011F9A4E6D1F88400083800F08F
:10C070000BF998E6C86F083800F006F98DE6486FAE
:10C08000083800F001F982E6C86E083800F0FCF8C4
:10C0900077E6486E083800F0F7F86CE6C86D0838A7
:10C0A00000F0F2F861E6486D083800F0EDF856E669
:10C0B000C86C083800F0E8F84BE6486C083800F027
:10C0C000E3F840E6C86B083800F0DEF835E6486B68
:10C0D000083800F0D9F82AE6C86A083800F0D4F821
:10C0E0001FE62A78C9F8280001322A70C3E62A78A8
:10C0F000C9F8200001322A705AE72A78C9F8880066
:10C1000001322A70DCE62A78C4F8800001322A70F5
:10C110008EE72A78C9F8680001322A70C3E62A78C7
:10C12000C8F8600001322A7014E72A78C9F848007C
:10C1300001322A70ABE62A78C8F8400001322A7032
:10C140001FE740298E4628BF4FF0400E02EB0E033A
:10C1500002930123CEEB01014FEA0E480025019323
:10C16000BCE600BF88004000C8004000F8B500F001
:10C170008FFD294B29482A4C2A4F2B4DDFF8BCC094
:10C18000DFF8BCE0294E00221A605A609A60DA603B
:10C190001A615A619A61DA611A625A629A62DA62C3
:10C1A0001A635A639A63DA631A645A649A64DA64A3
:10C1B0001A655A659A65DA651A665A669A66DA6683
:10C1C0001A675A679A67DA67C3F880200168C3F86C
:10C1D000842041F480210160C3F307212170C3F35F
:10C1E0000740134938701B0E2B70FF238CF800306A
:10C1F000104D8EF8003010480B700123337084F816
:10C20000642070264FF40074102207F82C3C2E7026
:10C21000046081F8F820F8BD0080FF1F34800440DE
:10C220009C200740B0200740B420074094200740DE
:10C230001020074049E400E008E100E080200740CA
:10C2400088200740704700BF72B60D480268B2FAF6
:10C2500082F30F2B10DC4FF00041D94022EA01029B
:10C26000026062B6074803EBC303DB00C21800217B
:10C27000C15010465160704762B60020704700BF41
:10C280003492FF1FBC83FF1F0D4B0E4AC31AA2FB43
:10C2900003231B090F2B0CD80B4A127852B972B624
:10C2A0000A484FF00041026821FA03F31A43026082
:10C2B00062B67047064A1278002AF0D0FFF768B9D4
:10C2C000BC83FF1F398EE33841A0FF1F3492FF1F4C
:10C2D0004CA0FF1F38B50E4B0E4C1B68218805463D
:10C2E0008BB1B1F5917F05D20B4A4B1C55549BB2D3
:10C2F000238038BD0022084898470021064A55543B
:10C300000123238038BDB1F5917FEDD338BD00BF47
:10C3100078A0FF1F12A2FF1F18A2FF1F2DE9F843EC
:10C32000214E224F3168012380463B70B1B1204D30
:10C330004B8801EB8302013300240F2BC2F80880E5
:10C340002C7004D84B8000233B70BDE8F883402359
:10C350000B800320FFF780F93460F4E7DFF8549096
:10C3600099F80030002BF0D0114D45F6215408E02B
:10C37000013C12D02B7883B900F00AFB99F8003009
:10C380007BB10320FFF7EEF80528F1D8FFF75CFF3B
:10C39000014630600028EBD0CAE701232B70BDE8CE
:10C3A000F883BDE8F88300BF94A0FF1F68A0FF1FBB
:10C3B00098A0FF1F4CA0FF1F1201F8B5D5B2A1B382
:10C3C000012943D04378044600781B0643EA004025
:10C3D00040F4704045F004068F1E3043FFF79EFF87
:10C3E000022F04F1020314D9053414F8023C14F8A6
:10C3F000032C14F8010C1B0443EA0223334343EAE1
:10C400000060033FFFF78AFF022F234604F1030475
:10C41000EBD8022F23D0012F0DD045F4774040F008
:10C420000500BDE8F840FFF779BF14482843BDE890
:10C43000F840FFF773BF187845F4770545F0060517
:10C4400045EA0020BDE8F840FFF768BF03780C48D4
:10C4500045EA03452843BDE8F840FFF75FBF1A7877
:10C46000587845F0774545F0070545EA022545EA45
:10C470000040BDE8F840FFF751BF00BF06F0F700ED
:10C4800007F000F738B5084B1C7824B9074D296828
:10C4900009B14B8803B938BD9B000B800320FFF71F
:10C4A000DBF82C6038BD00BF68A0FF1F94A0FF1F01
:10C4B0002DE9F041AD4E33680746002B00F0928025
:10C4C0001D885A88910803EB81010432AA428C68C6
:10C4D00042D25A8004F00F064FEA1428A449A6F16C
:10C4E000080208F00F00C4F30313062A00F1010547
:10C4F0000B701AD9B31E012B5FFA88F04ED9052EA6
:10C5000048D0042E00F0A481731F022B7FD90F2E78
:10C510000ED1F72842D8F02802D0964B1B883BB1A9
:10C52000FFF7D8FE0020BDE8F08127B1BD4202D060
:10C530000020BDE8F081082EC4F3033300F08780AB
:10C54000092E11D00A2E40F094800A2BF0D18A4B8C
:10C550008A4A1B68A02181E01846FFF795FE042057
:10C56000FEF7E2FF3060B5E7092BE1D1270E00F0BE
:10C570007B81834B814A1B689021C4F3074611706D
:10C58000EDB2FCB2002B00F09D80224631462846D9
:10C59000984797E0F02843D9F72841D0F1380E2882
:10C5A000C6D801A353F820F05FC7000043C70000BE
:10C5B00031C7000031C5000031C5000023C70000AD
:10C5C00031C5000003C8000031C50000CDC7000020
:10C5D000E7C700000BC7000031C50000F3C600002C
:10C5E000D7C60000674B1B78002BA1D00420FEF7B4
:10C5F0009BFF0346306000289AD00588002D7FF409
:10C6000060AFFFF741FE35602846BDE8F081FFF7D7
:10C6100061FEC4F30740FFF75DFE072E02D1200E36
:10C62000FFF758FE534B584A198858481468584D1C
:10C63000524A017000270E0AF0201F802E701070E1
:10C640000CB301225348A0470120BDE8F081082B1C
:10C650007FF46EAF504B494A1B688021C4F30746F4
:10C660001170EDB2240E6BB328462246314698472E
:10C6700028E00B2E11D10B2B7FF45AAF474B3F4ACA
:10C680001B68B021EAE7464B1B68002B00F0FB80DB
:10C69000404898470120BDE8F0810C2E40F0008111
:10C6A0000C2B7FF445AF3F4B344A1B68C0211170FF
:10C6B000EDB2C4F30746002B00F0C880284631468F
:10C6C000240E98473849314A314B0D7016701C7052
:10C6D0000120BDE8F081354B1B68002B00F0D680AF
:10C6E0009847C4F30746254BEDB2240E83F800802B
:10C6F000E8E72F4B1B68002BF2D12E4B1B68A3B130
:10C70000FE209847C4F30746EDE72B4B1B68002B30
:10C71000E6D1284B1B6843B1FC209847C4F3074679
:10C72000E1E7264B1B68002BDAD1C4F30746DAE7B2
:10C73000234B1B68C4F30746002BD4D030469847E0
:10C74000D1E7204B1A68002AEFD0260C630C06F0C4
:10C750007F0003F47E531843F6B29047C3E71A4BA9
:10C760001B68C4F30746002BE8D1BCE7A0A0FF1F5D
:10C7700016A2FF1F12A2FF1F7CA0FF1F10A2FF1F07
:10C78000B0A0FF1F4CA0FF1F78A0FF1F14A2FF1F27
:10C7900015A2FF1F18A2FF1FA8A0FF1FACA0FF1F1C
:10C7A00090A0FF1F6CA0FF1F17A2FF1F58A0FF1F24
:10C7B0005CA0FF1F60A0FF1F9CA0FF1F8CA0FF1F9D
:10C7C000A4A0FF1F74A0FF1F88A0FF1F3F4B1B6882
:10C7D000002B85D13E4B1B68002BA6D0FA20984732
:10C7E000C4F307467FE73B4B1B68002B7FF478AF11
:10C7F000374B1B68002B98D0FB209847C4F30746A3
:10C8000071E7354B1B68002B7FF46AAF304B1B6818
:10C81000002B8AD0F8209847C4F3074663E70E2B15
:10C820007FF486AE2D4A2E4B1268E0211970002A43
:10C8300047D0260C610C06F07F0301F47E511943AA
:10C84000EDB2A1F5005128469047F6B2240E39E723
:10C85000FFF740FDC4F30740FFF73CFD200EFFF754
:10C8600039FD0020BDE8F0811E4B1D4A1B68802168
:10C870001170EDB2C4F3074683B1314628463A46FB
:10C8800098473C461EE70120BDE8F081104B1B682D
:10C89000002B3FF44AAFFF20984746E71C4611E7BC
:10C8A0000D2EBCD10D2B7FF443AE0F4B0C4A1B68F1
:10C8B000D0211170EDB2C4F30746002B7FF4FEAE19
:10C8C000C4E7C4F30746EDB2240EFBE684A0FF1FC5
:10C8D00060A0FF1F64A0FF1F54A0FF1F70A0FF1FD8
:10C8E00010A2FF1FA8A0FF1F80A0FF1F38B5164D84
:10C8F0002868E0B101884488A14213DD03191B7A3E
:10C9000083B104F10803C2180C1B002302E012F8E3
:10C91000011F21B10133A342F9D1204638BD1C4685
:10C92000204638BDFFF7B0FC0020286038BD074B1B
:10C930001B780BB9002038BD0220FEF7F5FD2860FA
:10C940000028D7D1F6E700BFBCA0FF1F4CA0FF1FF7
:10C950000D4B1B78BBB910B50C4C216803F0FF02DE
:10C960004B883F2B07DC07330B4401F1470003F8EA
:10C97000012F8342FBD140230B800120FEF76CFE88
:10C980000023236010BD7047B4A0FF1FB8A0FF1F95
:10C9900038B5224C237803B138BD01232370FFF74B
:10C9A000A5FF70BB00F048F840BB00F0DBF810BBFF
:10C9B000FEF7F8FCE0B900232370EFF30583002BAA
:10C9C000EAD1EFF3108172B6154B1868E0B1154C3F
:10C9D0002278CAB945691D6001232370C5B1AA61D7
:10C9E00001B962B600254577836898472570D3E77B
:10C9F00000F020F8DFE700F01BF8D9E700F016F8A8
:10CA0000D3E7FFF71FFCCDE70029C5D162B638BDDB
:10CA1000054B1D600029E5D1E3E700BFC1A0FF1F62
:10CA2000D89EFF1FDC9EFF1FD49EFF1F704700BFD4
:10CA3000704700BF704700BF054A064B10781B784F
:10CA4000C0B2DBB2984238BF4030C01A704700BF56
:10CA5000C8A0FF1FC9A0FF1FF0B4384B1A7912F00D
:10CA6000300F2CD072B6997D01F0FF0200293DD025
:10CA700062B6334F334938780D78334E1C46C0B216
:10CA8000EDB2431C402BE17928BF0023AB4202F1F9
:10CA9000FF32C9B21CBFF154184612F0FF02F0D1A8
:10CAA0002A4B1B68C2B23A704BB1A84236BFC5F1DF
:10CAB0004005401B40192728C4BF01221A701F4996
:10CAC000CA78D2B2150616D452060DD51B4B1B7967
:10CAD0005B0609D51E4B1F491B6800220A7003B173
:10CAE0001A70164B3C22DA70F0BC70474022D9799C
:10CAF0005A7462B6E3E70B791C06E5D5164B174E60
:10CB00001C783378E4B2DBB29C420ED0144D01E0C5
:10CB1000A3420AD00133402B28BF00230879E85CE8
:10CB2000C0B2C871087D0728F2D9DBB2034933705F
:10CB30000B79180644BF7C23CB70C5E700A00640E4
:10CB4000C8A0FF1FC9A0FF1F0CA1FF1FC4A0FF1F8B
:10CB500050A1FF1F4CA1FF1F54A1FF1F4DA1FF1F9C
:10CB6000CCA0FF1F054A064B10781B78C0B2DBB281
:10CB7000984238BF4030C01A704700BFC8A1FF1F9D
:10CB80005DA1FF1FF0B4384B1A7912F0300F2CD092
:10CB900072B6997D01F0FF0200293DD062B6334F95
:10CBA000334938780D78334E1C46C0B2EDB2431C81
:10CBB000402BE17928BF0023AB4202F1FF32C9B21A
:10CBC0001CBFF154184612F0FF02F0D12A4B1B682B
:10CBD000C2B23A704BB1A84236BFC5F14005401B06
:10CBE00040192728C4BF01221A701F49CA78D2B23F
:10CBF000150616D452060DD51B4B1B795B0609D5BD
:10CC00001E4B1F491B6800220A7003B11A70164B95
:10CC10003C22DA70F0BC70474022D9795A7462B66F
:10CC2000E3E70B791C06E5D5164B174E1C783378D5
:10CC3000E4B2DBB29C420ED0144D01E0A3420AD014
:10CC40000133282B28BF00230879E85CC0B2C871E3
:10CC5000087D0728F2D9DBB2034933700B79180637
:10CC600044BF7C23CB70C5E700B00640C8A1FF1FBE
:10CC70005DA1FF1F88A1FF1F58A1FF1FCCA1FF1FAF
:10CC80005CA1FF1FD0A1FF1FC9A1FF1F60A1FF1F53
:10CC900070B584B072B6194B194D1A4870224126EE
:10CCA0000F2480211A702E701A46047019701378A0
:10CCB0001B06FCD5144B186862B6144B144C9842F2
:10CCC00098BF00EB800001A998BF40000A22FDF741
:10CCD000CFFE01A92046002311F8012B01333AB100
:10CCE0000A2B20F8022FF7D11623237004B070BD51
:10CCF0005B00DBB2237004B070BD00BF00000240D7
:10CD00000700024006000240080002407F9698009B
:10CD10000093FF1FFFFFFFFF2DE9F043DFF8EC80DA
:10CD20008BB006460F4600F073F898F900300133D7
:10CD300004460D4637D03046394600F0DFF900286A
:10CD400031D02BA3D3E900233046394600F026FE2C
:10CD5000814668BB28A3D3E900233046394600F05A
:10CD6000FFFD00B398F90030254ACDF82090042447
:10CD700000200021022BCDE90467CDE90267009471
:10CD80000192CDE906012CD0684600F0BDF940B310
:10CD9000089B1BB101F0AAF9089B0360DDE90601BD
:10CDA0000BB0BDE8F083204629460BB0BDE8F08308
:10CDB000134A98F90030019203210022CDE904675B
:10CDC000CDE90267009108922BB90E4B4FF06042FB
:10CDD000CDE90623D8E70C490020022BCDE9060156
:10CDE000D2D101F083F922230360D1E7AFF30080B1
:10CDF000EF39FAFE422E864051302DD5104987C0BA
:10CE0000740F0100FFFFEF470000F07F1693FF1F34
:10CE10002DE9F04FB04F21F00042BA4283B00C46EA
:10CE20004FEAD17605460DD9AC4FBA4225D9C1F3A8
:10CE30001303034340F0EF800EB10020014603B01E
:10CE4000BDE8F08FA64B9A4200F2CC80A54B9A42E7
:10CE500000F2DE808AA3D3E9002300F05DF900220E
:10CE6000A14B00F09BFD002800F0058128462146DB
:10CE700000229D4B00F050F9E1E783A3D3E90023A2
:10CE800000F08CFD002840F0CB802846214680A38E
:10CE9000D3E9002300F064FD0028CED1934B28464F
:10CEA00003EBC60821467CA3D3E9002300F0E6FA91
:10CEB000D8E9002300F030F900F07AFD804600F058
:10CEC00077FA77A3D3E9002306460F4600F0D6FA97
:10CED00002460B462846214600F01CF972A3D3E90E
:10CEE0000023CDE900013046394600F0C7FA8246FA
:10CEF0008B4652465B46DDE9000100F00BF9054622
:10CF00000C462A4623462846214600F0B7FA68A375
:10CF1000D3E9002306460F4600F0B0FA66A3D3E932
:10CF2000002300F0F7F832463B4600F0A7FA64A36E
:10CF3000D3E9002300F0F0F832463B4600F09EFAB9
:10CF400061A3D3E9002300F0E5F832463B4600F048
:10CF500095FA5FA3D3E9002300F0DEF832463B46A2
:10CF600000F08CFA02460B462846214600F0D2F823
:10CF700006460F462846214632463B46B8F1000F8A
:10CF800056D000F07BFA324604460D463B46002060
:10CF90004FF0804100F0BEF802460B46204629467D
:10CFA00000F096FB02460B465046594600F0B2F898
:10CFB000DDE9002300F0AEF80B4602464A490020A6
:10CFC00000F0A8F86FF47F7398454FDA08F57A7887
:10CFD00001EB085100224FF0B87300F04FFA03B094
:10CFE000BDE8F08F424B9A423FF658AF414BF400F8
:10CFF0002344D3E9002300F08DF83F4BC6F101082C
:10D000001C44CDE90001D4E900ABC6EB080870E789
:10D010004FF0000875E702460B4600F07DF80EE77A
:10D0200017A3D3E900231046194600F027FA06E7B4
:10D0300000F024FA0022804689464FF080433046B3
:10D04000394600F067F802460B464046494600F074
:10D050003FFB2A46234600F05DF802460B460020BF
:10D06000214900F057F803B0BDE8F08F01EB0851FB
:10D0700003B0BDE8F08F804643E700BFAFF3008008
:10D080009C7500883CE4377EEF39FAFE422E8640DC
:10D0900051302DD5104987C0FE822B654715F73FCB
:10D0A0000000E0FE422EE63F763C7935EF39EA3D5E
:10D0B000D0A4BE726937663EF16BD2C541BDBB3E9E
:10D0C0002CDE25AF6A56113F93BDBE166CC1663F7C
:10D0D0003E5555555555C53F412E8640FFFFEF7FC4
:10D0E000422ED63FFFFF2F3E0000F03F780F010099
:10D0F000B1A2F03F980F0100880F010041F00041FC
:10D1000001F58010C00F70470020704781F000418A
:10D1100002E000BF83F0004330B54FEA41044FEA1C
:10D12000430594EA050F08BF90EA020F1FBF54EAB7
:10D13000000C55EA020C7FEA645C7FEA655C00F053
:10D14000E2804FEA5454D4EB5555B8BF6D420CDD24
:10D150002C4480EA020281EA030382EA000083EAA7
:10D16000010180EA020281EA0303362D88BF30BD47
:10D1700011F0004F4FEA01314FF4801C4CEA11319D
:10D1800002D0404261EB410113F0004F4FEA0333FC
:10D190004CEA133302D0524263EB430394EA050F87
:10D1A00000F0A780A4F10104D5F1200E0DDB02FAF6
:10D1B0000EFC22FA05F2801841F1000103FA0EF28A
:10D1C000801843FA05F359410EE0A5F120050EF150
:10D1D000200E012A03FA0EFC28BF4CF0020C43FA81
:10D1E00005F3C01851EBE37101F0004507D54FF08E
:10D1F000000EDCF1000C7EEB00006EEB0101B1F5DE
:10D20000801F1BD3B1F5001F0CD349085FEA300023
:10D210004FEA3C0C04F101044FEA445212F5800F2E
:10D2200080F09A80BCF1004F08BF5FEA500C50F1CB
:10D23000000041EB045141EA050130BD5FEA4C0CAE
:10D24000404141EB010111F4801FA4F10104E9D137
:10D2500091F0000F04BF01460020B1FA81F308BF2E
:10D260002033A3F10B03B3F120020CDA0C3208DDFA
:10D2700002F1140CC2F10C0201FA0CF021FA02F1D5
:10D280000CE002F11402D8BFC2F1200C01FA02F145
:10D2900020FA0CFCDCBF41EA0C019040E41AA2BF6A
:10D2A00001EB0451294330BD6FEA04041F3C1CDA32
:10D2B0000C340EDC04F11404C4F1200220FA04F052
:10D2C00001FA02F340EA030021FA04F345EA0301FC
:10D2D00030BDC4F10C04C4F1200220FA02F001FABE
:10D2E00004F340EA0300294630BD21FA04F0294640
:10D2F00030BD94F0000F83F4801306BF81F48011D9
:10D300000134013D4EE77FEA645C18BF7FEA655C4B
:10D3100029D094EA050F08BF90EA020F05D054EA1D
:10D32000000C04BF1946104630BD91EA030F1EBF22
:10D330000021002030BD5FEA545C05D14000494126
:10D3400028BF41F0004130BD14F580043CBF01F519
:10D35000801130BD01F0004545F0FE4141F47001FF
:10D360004FF0000030BD7FEA645C1ABF19461046DA
:10D370007FEA655C1CBF0B46024650EA013406BFDB
:10D3800052EA033591EA030F41F4002130BD00BF9A
:10D3900090F0000F04BF0021704730B54FF4806457
:10D3A00004F132044FF000054FF0000150E700BFD8
:10D3B00090F0000F04BF0021704730B54FF4806437
:10D3C00004F1320410F0004548BF40424FF0000124
:10D3D0003EE700BF42004FEAE2014FEA31014FEA67
:10D3E00002701FBF12F07F4393F07F4F81F06051B6
:10D3F000704792F0000F14BF93F07F4F704730B525
:10D400004FF4607401F0004521F0004120E700BFB7
:10D4100050EA010208BF704730B54FF000050AE03E
:10D4200050EA010208BF704730B511F0004502D53F
:10D43000404261EB41014FF4806404F132045FEA41
:10D44000915C3FF4DCAE4FF003025FEADC0C18BFE6
:10D4500003325FEADC0C18BF033202EBDC02C2F1DC
:10D46000200300FA03FC20FA02F001FA03FE40EA6E
:10D470000E0021FA02F11444C1E600BF70B54FF06E
:10D48000FF0C4CF4E06C1CEA11541DBF1CEA135550
:10D4900094EA0C0F95EA0C0F00F0DEF82C4481EAB8
:10D4A000030621EA4C5123EA4C5350EA013518BFD8
:10D4B00052EA033541F4801143F4801338D0A0FBC5
:10D4C00002CE4FF00005E1FB02E506F00042E0FB72
:10D4D00003E54FF00006E1FB03569CF0000F18BF78
:10D4E0004EF0010EA4F1FF04B6F5007F64F5407420
:10D4F00004D25FEA4E0E6D4146EB060642EAC621B3
:10D5000041EA55514FEAC52040EA5E504FEACE2E1F
:10D51000B4F1FD0C88BFBCF5E06F1ED8BEF1004F22
:10D5200008BF5FEA500E50F1000041EB045170BD9E
:10D5300006F0004646EA010140EA020081EA0301E2
:10D54000B4EB5C04C2BFD4EB0C0541EA045170BDDE
:10D5500041F480114FF0000E013C00F3AB8014F158
:10D56000360FDEBF002001F0004170BDC4F10004A1
:10D57000203C35DA0C341BDC04F11404C4F1200522
:10D5800000FA05F320FA04F001FA05F240EA02007D
:10D5900001F0004221F0004110EBD37021FA04F6B3
:10D5A00042EB06015EEA430E08BF20EAD37070BD6D
:10D5B000C4F10C04C4F1200500FA04F320FA05F0CC
:10D5C00001FA04F240EA020001F0004110EBD370CE
:10D5D00041F100015EEA430E08BF20EAD37070BD3E
:10D5E000C4F1200500FA05F24EEA020E20FA04F317
:10D5F00001FA05F243EA020321FA04F001F00041C6
:10D6000021FA04F220EA020000EBD3705EEA430E36
:10D6100008BF20EAD37070BD94F0000F0FD101F065
:10D620000046400041EB010111F4801F08BF013C9E
:10D63000F7D041EA060195F0000F18BF704703F0DC
:10D640000046520043EB030313F4801F08BF013D63
:10D65000F7D043EA0603704794EA0C0F0CEA13551F
:10D6600018BF95EA0C0F0CD050EA410618BF52EAD9
:10D670004306D1D181EA030101F000414FF00000DF
:10D6800070BD50EA410606BF1046194652EA4306ED
:10D6900019D094EA0C0F02D150EA013613D195EA61
:10D6A0000C0F05D152EA03361CBF104619460AD1A9
:10D6B00081EA030101F0004141F0FE4141F47001B3
:10D6C0004FF0000070BD41F0FE4141F4780170BDA3
:10D6D00070B54FF0FF0C4CF4E06C1CEA11541DBF08
:10D6E0001CEA135594EA0C0F95EA0C0F00F0A7F80A
:10D6F000A4EB050481EA030E52EA03354FEA013137
:10D7000000F088804FEA03334FF0805545EA131349
:10D7100043EA12634FEA022245EA111545EA106511
:10D720004FEA00260EF000419D4208BF964244F1A8
:10D73000FD0404F5407402D25B084FEA3202B61AC7
:10D7400065EB03055B084FEA32024FF480104FF49B
:10D75000002CB6EB020E75EB030E22BFB61A75460F
:10D7600040EA0C005B084FEA3202B6EB020E75EBA2
:10D77000030E22BFB61A754640EA5C005B084FEA0A
:10D780003202B6EB020E75EB030E22BFB61A7546D7
:10D7900040EA9C005B084FEA3202B6EB020E75EBE2
:10D7A000030E22BFB61A754640EADC0055EA060EA3
:10D7B00018D04FEA051545EA16754FEA06164FEAE6
:10D7C000C30343EA52734FEAC2025FEA1C1CC0D192
:10D7D00011F4801F0BD141EA00014FF000004FF01F
:10D7E000004CB6E711F4801F04BF01430020B4F1E0
:10D7F000FD0C88BFBCF5E06F3FF6AFAEB5EB030C98
:10D8000004BFB6EB020C5FEA500C50F1000041EB94
:10D81000045170BD0EF0004E4EEA113114EB5C0461
:10D82000C2BFD4EB0C0541EA045170BD41F4801134
:10D830004FF0000E013C90E645EA060E8DE60CEA3C
:10D84000135594EA0C0F08BF95EA0C0F3FF43BAF59
:10D8500094EA0C0F0AD150EA01347FF434AF95EA10
:10D860000C0F7FF425AF104619462CE795EA0C0FF4
:10D8700006D152EA03353FF4FDAE1046194622E7C1
:10D8800050EA410618BF52EA43067FF4C5AE50EA9B
:10D8900041047FF40DAF52EA43057FF4EBAE12E78B
:10D8A0004FF0FF3C06E000BF4FF0010C02E000BF6C
:10D8B0004FF0010C4DF804CD4FEA410C7FEA6C5C4F
:10D8C0004FEA430C18BF7FEA6C5C1BD001B050EAF2
:10D8D000410C0CBF52EA430C91EA030F02BF90EADD
:10D8E000020F0020704710F1000F91EA030F58BF9C
:10D8F000994208BF90422CBFD8176FEAE37040F0FE
:10D90000010070474FEA410C7FEA6C5C02D150EA9B
:10D91000013C07D14FEA430C7FEA6C5CD6D152EA56
:10D92000033CD3D05DF8040B704700BF844610461B
:10D9300062468C461946634600E000BF01B5FFF71A
:10D94000B7FF002848BF10F1000F01BD4DF808EDEA
:10D95000FFF7F4FF0CBF012000205DF808FB00BFBB
:10D960004DF808EDFFF7EAFF34BF012000205DF815
:10D9700008FB00BF4DF808EDFFF7E0FF94BF012062
:10D9800000205DF808FB00BF4DF808EDFFF7CEFF63
:10D9900094BF012000205DF808FB00BF4DF808EDA2
:10D9A000FFF7C4FF34BF012000205DF808FB00BF73
:10D9B0004FEA410212F5001215D211D56FF47873B7
:10D9C000B3EB625212D94FEAC12343F0004343EA5A
:10D9D000505311F0004F23FA02F018BF4042704735
:10D9E0004FF00000704750EA013005D111F00040BF
:10D9F00008BF6FF0004070474FF00000704700BF55
:10DA00004FEA4102B2F1E04324BFB3F5001CDCF160
:10DA1000FE5C0DD901F0004C4FEAC0024CEA507098
:10DA2000B2F1004F40EB830008BF20F001007047C7
:10DA300011F0804F21D113F13872BCBF01F00040CA
:10DA4000704741F480114FEA5252C2F11802C2F1FC
:10DA5000200C10FA0CF320FA02F018BF40F001007D
:10DA60004FEAC1234FEAD32303FA0CFC40EA0C002F
:10DA700023FA02F34FEA4303CCE77FEA625307D16C
:10DA800050EA01331EBF4FF0FE4040F440007047A3
:10DA900001F0004040F0FE4040F40000704700BF3D
:10DAA00080F0004002E000BF81F0004142001FBF53
:10DAB0005FEA410392EA030F7FEA226C7FEA236C5C
:10DAC0006AD04FEA1262D2EB1363C1BFD218414051
:10DAD00048404140B8BF5B42192B88BF704710F0E7
:10DAE000004F40F4000020F07F4018BF404211F08A
:10DAF000004F41F4000121F07F4118BF494292EAF2
:10DB0000030F3FD0A2F1010241FA03FC10EB0C001D
:10DB1000C3F1200301FA03F100F0004302D54942AA
:10DB200060EB4000B0F5000F13D3B0F1807F06D357
:10DB300040084FEA310102F10102FE2A51D2B1F14F
:10DB4000004F40EBC25008BF20F0010040EA030044
:10DB50007047490040EB000010F4000FA2F10102F1
:10DB6000EDD1B0FA80FCACF1080CB2EB0C0200FA7B
:10DB70000CF0AABF00EBC25052421843BCBFD040C9
:10DB80001843704792F0000F81F4000106BF80F443
:10DB900000000132013BB5E74FEA41037FEA226C06
:10DBA00018BF7FEA236C21D092EA030F04D092F0D1
:10DBB000000F08BF0846704790EA010F1CBF002005
:10DBC000704712F07F4F04D1400028BF40F0004062
:10DBD000704712F100723CBF00F50000704700F082
:10DBE000004343F0FE4040F4000070477FEA2262A9
:10DBF00016BF08467FEA23630146420206BF5FEA7A
:10DC0000412390EA010F40F4800070474FF0000379
:10DC100004E000BF10F0004348BF40425FEA000C40
:10DC200008BF704743F0964301464FF000001CE0E8
:10DC300050EA010208BF70474FF000030AE000BF3E
:10DC400050EA010208BF704711F0004302D540427C
:10DC500061EB41015FEA010C02BF844601460020EE
:10DC600043F0B64308BFA3F18053A3F50003BCFA09
:10DC70008CF2083AA3EBC25310DB01FA02FC6344B6
:10DC800000FA02FCC2F12002BCF1004F20FA02F2BD
:10DC900043EB020008BF20F00100704702F12002B0
:10DCA00001FA02FCC2F1200250EA4C0021FA02F211
:10DCB00043EB020008BF20EADC7070474FF0FF0C16
:10DCC0001CEAD0521EBF1CEAD15392EA0C0F93EA11
:10DCD0000C0F6FD01A4480EA010C400218BF5FEAB3
:10DCE00041211ED04FF0006343EA501043EA511126
:10DCF000A0FB01310CF00040B1F5000F3EBF490020
:10DD000041EAD3715B0040EA010062F17F02FD2A23
:10DD10001DD8B3F1004F40EBC25008BF20F0010006
:10DD2000704790F0000F0CF0004C08BF49024CEA1D
:10DD3000502040EA51207F3AC2BFD2F1FF0340EAAF
:10DD4000C250704740F400004FF00003013A5DDC20
:10DD500012F1190FDCBF00F000407047C2F1000261
:10DD6000410021FA02F1C2F1200200FA02FC5FEA4E
:10DD7000310040F1000053EA4C0308BF20EADC7098
:10DD8000704792F0000F00F0004C02BF400010F40A
:10DD9000000F013AF9D040EA0C0093F0000F01F0B7
:10DDA000004C02BF490011F4000F013BF9D041EAD9
:10DDB0000C018FE70CEAD15392EA0C0F18BF93EADB
:10DDC0000C0F0AD030F0004C18BF31F0004CD8D105
:10DDD00080EA010000F00040704790F0000F17BF8C
:10DDE00090F0004F084691F0000F91F0004F14D0D2
:10DDF00092EA0C0F01D142020FD193EA0C0F03D12A
:10DE00004B0218BF084608D180EA010000F000402C
:10DE100040F0FE4040F40000704740F0FE4040F407
:10DE2000400070474FF0FF0C1CEAD0521EBF1CEAA6
:10DE3000D15392EA0C0F93EA0C0F69D0A2EB0302C4
:10DE400080EA010C49024FEA402037D04FF080535E
:10DE500043EA111143EA10130CF000408B4238BF23
:10DE60005B0042F17D024FF4000C8B4224BF5B1A31
:10DE700040EA0C00B3EB510F24BFA3EB510340EA7F
:10DE80005C00B3EB910F24BFA3EB910340EA9C002D
:10DE9000B3EBD10F24BFA3EBD10340EADC001B019D
:10DEA00018BF5FEA1C1CE0D1FD2A3FF650AF8B4241
:10DEB00040EBC25008BF20F0010070470CF0004C4E
:10DEC0004CEA50207F32C2BFD2F1FF0340EAC25079
:10DED000704740F400004FF00003013A37E792F03A
:10DEE000000F00F0004C02BF400010F4000F013A98
:10DEF000F9D040EA0C0093F0000F01F0004C02BF93
:10DF0000490011F4000F013BF9D041EA0C0195E7FB
:10DF10000CEAD15392EA0C0F08D142027FF47DAF94
:10DF200093EA0C0F7FF470AF084676E793EA0C0F84
:10DF300004D14B023FF44CAF08466EE730F0004C82
:10DF400018BF31F0004CCAD130F000427FF45CAF12
:10DF500031F000437FF43CAF5FE700BF4FF0FF3C80
:10DF600006E000BF4FF0010C02E000BF4FF0010CD3
:10DF70004DF804CD4FEA40024FEA41037FEA226C9C
:10DF800018BF7FEA236C11D001B052EA530C18BFBE
:10DF900090EA010F58BFB2EB030088BFC81738BF23
:10DFA0006FEAE17018BF40F0010070477FEA226C11
:10DFB00002D15FEA402C05D17FEA236CE4D15FEA0D
:10DFC000412CE1D05DF8040B704700BF8446084641
:10DFD0006146FFE70FB5FFF7C9FF002848BF10F102
:10DFE000000F0FBD4DF808EDFFF7F4FF0CBF012047
:10DFF00000205DF808FB00BF4DF808EDFFF7EAFFD1
:10E0000034BF012000205DF808FB00BF4DF808ED8B
:10E01000FFF7E0FF94BF012000205DF808FB00BF80
:10E020004DF808EDFFF7D2FF94BF012000205DF806
:10E0300008FB00BF4DF808EDFFF7C8FF34BF012013
:10E0400000205DF808FB00BF4FEA4002B2F1FE4F2E
:10E050000FD34FF09E03B3EB12620DD94FEA0023AA
:10E0600043F0004310F0004F23FA02F018BF404283
:10E0700070474FF00000704712F1610F01D142026A
:10E0800005D110F0004008BF6FF0004070474FF01E
:10E090000000704742000ED2B2F1FE4F0BD34FF09A
:10E0A0009E03B3EB126209D44FEA002343F000430E
:10E0B00023FA02F070474FF00000704712F1610F31
:10E0C00001D1420202D14FF0FF3070474FF0000003
:10E0D000704700BF0B460146184600F001B800BF6C
:10E0E00013460A460146022000F0BCBE014B1868E8
:10E0F000704700BF4097FF1F70B50F4E0F4D761B46
:10E10000B61018BF002405D0013455F8043B9847D9
:10E11000A642F9D10A4E0B4D761B02F047FFB6100E
:10E1200018BF002406D0013455F8043B9847A64296
:10E13000F9D170BD70BD00BFB80F0100B80F01006C
:10E14000CC0F0100B80F0100024B0146186800F027
:10E150000BB800BF4097FF1F024B0146186800F044
:10E1600045BF00BF4097FF1F2DE9F04F01F10B05A0
:10E17000162D83B0064640F29F8035F0070500F16A
:10E18000BF80A94200F2BC8000F058FBB5F5FC7FCF
:10E19000C0F09C826B0A00F0BA80042B00F28381ED
:10E1A000A80900F1390E4FEA4E033830C44F07EB8F
:10E1B0008303A3F108015C68A14207D1ACE0002A07
:10E1C00080F2AC80E468A14200F0A680636823F08E
:10E1D00003035A1B0F2AF2DDB9493C6901F1080E0D
:10E1E000744500F0B381636823F003035A1B0F2AC0
:10E1F00000F39981002AC1F814E0C1F810E080F220
:10E200009E80B3F5007F80F06781DB0803F1010C8D
:10E2100001229B1002FA03F34A6851F83C80C4F8CB
:10E22000088001EBCC091A43A9F10803E3604A60B6
:10E2300041F83C40C8F80C40831001249C409442B3
:10E2400000F28A80144206D120F0030064001442D8
:10E2500000F10400FAD007EBC009CC468046DCF898
:10E260000C108C4507D173E1002A80F28181C968C6
:10E270008C4500F06D814B6823F003035A1B0F2A75
:10E28000F2DD0C46D1F80CC054F8088F4B1945F05C
:10E2900001054D6042F00101C8F80CC03046CCF8D1
:10E2A00008807B613B61C3F80CE0C3F808E059606B
:10E2B0009A5000F0C5FA1FE0102921D800F0BEFAEC
:10E2C0001025062302207E4F07EB8303A3F10802EB
:10E2D0005C68944200F045816368E168A56823F0BA
:10E2E0000303234430465A68E96042F001028D601E
:10E2F0005A6000F0A5FA0834204603B0BDE8F08F5C
:10E3000000240C232046336003B0BDE8F08F802347
:10E310004FF0400E3F2049E770465DE72344E16837
:10E320005A68A56842F00102E96030468D605A6083
:10E3300000F086FA0834204603B0BDE8F08F23448D
:10E3400030465A6842F001025A6000F079FA083407
:10E35000204603B0BDE8F08FBC68636823F0030873
:10E36000A84504D3C5EB08030F2B00F38C80554B55
:10E37000DFF860911A68D9F8003001332A4404EBC1
:10E38000080A00F0608102F580520F3222F47F62A9
:10E3900022F00F0211463046019200F04BFCB0F122
:10E3A000FF3F8346019A00F05881824500F2FC80CD
:10E3B000454B1968DA451144196000F05381D9F8CA
:10E3C0000000DFF810E101301BBFCAEB0B0A51441B
:10E3D000CEF800B019601BF0070100F01781C1F101
:10E3E0000800C1F58051834408315A44C2F30B023E
:10E3F000C2EB010949463046019300F01BFC431C67
:10E40000019B00F03F81CBEB00024A4442F0010245
:10E410001968C7F808B04944BC42CBF80420196019
:10E42000DFF8A49016D0B8F10F0F40F2FD806268BB
:10E43000A8F10C0323F00703E01802F001024FF0EB
:10E44000050E1A430F2B6260C0F804E0C0F808E024
:10E4500000F21C811D4BBC681A68914288BF19608C
:10E460001B4B1A689142626888BF196022F0030250
:10E470009542A2EB050301D80F2B04DC304600F0D7
:10E48000DFF9002438E7621943F0010345F0010584
:10E4900065603046BA60536000F0D2F90834204617
:10E4A00003B0BDE8F08F142B71D9542B00F2A48077
:10E4B000280B00F16F0E4FEA4E036E3076E600BF78
:10E4C0004497FF1FDCA1FF1FE0A1FF1FD8A1FF1F82
:10E4D000D4A1FF1F509BFF1F5A0A042A5ED9142A99
:10E4E00000F2B38002F15C0149005B3207EB810C62
:10E4F00057F82110DFF8DC81ACF1080C8C4500F0F6
:10E5000088804A6822F00302934202D289688C45CF
:10E51000F7D1D1F80CC07A68C4F80CC0A160CCF86F
:10E520000840CC6088E6631942F0010745F0010518
:10E53000656030464B610B61C3F80CE0C3F808E03E
:10E540005F609A50083400F07BF9D5E64A6873E6BC
:10E5500008F1010818F0030F0CF1080C7FF47FAEEE
:10E5600030E0DC68A34208BF02303FF435AEB3E6CA
:10E570000B440C465A68C96854F8085F42F001021F
:10E580005A603046E9608D6000F05AF9B4E603F154
:10E590005C0E03F15B004FEA4E0307E69A0902F1B5
:10E5A000390149003832A1E7BC424A4B3FF400AF81
:10E5B0009C68626822F003025AE759F808399945C5
:10E5C00040F0828010F0030F00F1FF30F5D17B683E
:10E5D00023EA04037B6064009C423FF6BDAE002C3E
:10E5E0003FF4BAAE1C4240467FF435AE64001C4294
:10E5F00000F10400FAD02EE6B3F5AA7F18D8E80B94
:10E6000000F1780E4FEA4E037730CFE54FF480519A
:10E61000EBE60121D8F80430921001FA02F21A4315
:10E62000C8F80420614677E70123CBF8043025E7DA
:10E6300040F25452934220D8A80C00F17D0E4FEACC
:10E640004E037C30B2E51032A4E6542A26D81A0BC9
:10E6500002F16F0149006E3248E7BC68626822F03F
:10E66000030205E7CAF30B0000287FF4A8AE42447A
:10E67000BB6842F001025A60ECE6FE234FF07F0EC9
:10E680007E2093E501224FF00009C1E604F1080164
:10E69000304600F0ABFCD9F80010DBE6B2F5AA7FFB
:10E6A00005D8DA0B02F17801490077321EE740F213
:10E6B00054518A4205D89A0C02F17D0149007C32FE
:10E6C00014E7FE217E2211E77B6884E7E808431CFB
:10E6D0005B00F8E54497FF1F8842F0B50DD98B1811
:10E6E00098420AD28118002A51D09A1A13F8014D83
:10E6F00001F8014D9342F9D1F0BD0F2A48D941EA02
:10E7000000039B0746D100F1100401F110031546E8
:10E7100053F8106C44F8106C53F80C6C44F80C6C03
:10E7200053F8086C44F8086C103D53F8046C44F836
:10E73000046C0F2D03F1100304F11004E8D8A2F1CA
:10E74000100323F00F0302F00F0E1033BEF1030F7E
:10E750001944034421D91E1F0D467446043C55F844
:10E76000047B46F8047F032CF8D8AEF1040424F0AF
:10E77000030404342344214402F0030262B1013B48
:10E780000A4411F8014B03F8014F8A42F9D1F0BD58
:10E790000346F3E70346F2E7F0BD7246EEE700BF3B
:10E7A00070B4840746D0541E002A41D0CDB203462F
:10E7B00002E0621EE4B3144603F8015B9A07F8D145
:10E7C000032C2ED9CDB245EA05250F2C45EA054587
:10E7D00019D903F110022646103E0F2E42F8105CA4
:10E7E00042F80C5C42F8085C42F8045C02F110024A
:10E7F000F2D8A4F1100222F00F0204F00F0410323C
:10E80000032C13440DD91E462246043A032A46F827
:10E81000045BFAD8221F22F003020432134404F0EE
:10E8200003042CB1C9B21C4403F8011BA342FBD161
:10E8300070BC704714460346C2E700BF704700BF74
:10E84000704700BF024B0A460146186800F002B844
:10E850004097FF1F2DE9F04F174683B0002900F0C5
:10E86000C1800E46814607F10B05FFF7E7FF56F81A
:10E8700004EC162D2EF00304A6F1080840D810224F
:10E880001546AF4241D8944275DAC94B996808EBF6
:10E8900004008842416800F0D98021F0010303445C
:10E8A0005B68DB077DD51EF0010F35D03946484641
:10E8B000FFF75AFC0746E0B156F8043C23F0010389
:10E8C0004344A0F108029A4200F04481221F242A06
:10E8D00000F23181132A00F20481034632461168A6
:10E8E00019605168596092689A603146484600F054
:10E8F0007DFB4846FFF7A4FF384603B0BDE8F08F24
:10E9000025F00705002D2A46BBDA0C230020C9F8A4
:10E91000003003B0BDE8F08F56F8083CC3EB080A9E
:10E92000DAF8043023F0030C04EB0C039342BDDB54
:10E930005746DAF80C1057F8080F221F242AC16036
:10E94000886000F21781132A40F212813168CAF8F8
:10E9500008107168CAF80C101B2A00F22B810836C7
:10E960000AF110023168116071685160B1689160FC
:10E970003E461C46D046631B0F2B1DD8D8F80430EA
:10E9800003F0010323434444C8F80430636843F0B0
:10E99000010363604846FFF753FF304603B0BDE80C
:10E9A000F08F21F003012144914221DBC36882688A
:10E9B0000C46D3609A60DEE7D8F8042008EB050126
:10E9C00002F00102154343F001020B44C8F8045061
:10E9D0004A605A6842F0010208315A60484600F025
:10E9E00005FBD7E7114603B0BDE8F04FFFF7BCBB0E
:10E9F0001EF0010F7FF45AAF56F8083CC3EB080A2B
:10EA0000DAF8043023F0030C01EB0C0E96458BDB97
:10EA1000C36882685746D3609A6057F8081FDAF8CF
:10EA20000C30CB60221F242A996000F29980132AAF
:10EA300062D93368CAF808307368CAF80C301B2AE8
:10EA400000F2A08008360AF1100356E021F0030B13
:10EA5000A34405F11000834559DA1EF0010F7FF43D
:10EA600025AF56F8081CC1EB080ADAF8041021F0AB
:10EA7000030CE34458453FF757AF5746DAF80C10FC
:10EA800057F8080F221F242AC160886000F2B48062
:10EA9000132A40F2A5803168CAF808107168CAF8D4
:10EAA0000C101B2A00F2AF8008360AF11002316800
:10EAB000116071685160B16891600AEB0501C5EBA6
:10EAC0000B0242F0010299604A60DAF8043003F068
:10EAD00001031D434846CAF80450FFF7B1FE38460B
:10EAE0005CE733680360736843601B2A27D800F132
:10EAF000080306F10802F2E63B4632681A607268C3
:10EB00005A60B2689A603E467446D04633E708EBD6
:10EB10000501C5EB0B0B4BF0010299604A6056F8FA
:10EB2000043C03F001031D43484646F8045CFFF72C
:10EB300087FE304632E73146FFF7CEFDD5E6B368B3
:10EB40008360F368C360242A28D000F1100306F123
:10EB50001002C4E650F8043C23F003031C440AE707
:10EB6000314638467446D046FFF7B6FD3E4602E7CA
:10EB70003A46F7E6314638461C46D046FFF7ACFD2C
:10EB80003E46F8E6B368CAF81030F368CAF81430A5
:10EB9000242A1BD010360AF11803AEE7336903614B
:10EBA0007369436106F1180200F1180397E600BF8C
:10EBB0004497FF1FB168CAF81010F168CAF8141022
:10EBC000242A0FD010360AF11802CBE63369CAF8AE
:10EBD00018307369CAF81C3018360AF120038CE724
:10EBE0003A4664E73269CAF818207269CAF81C20EC
:10EBF00018360AF12002B5E6314638460193FFF790
:10EC00006BFD019B59E7B168CAF81010F168CAF8AA
:10EC10001410242A03D010360AF1180247E732698B
:10EC2000CAF818207269CAF81C2018360AF12002A6
:10EC30003DE700BF38B5074C002305460846236072
:10EC4000FBF7E0FE431C00D038BD2368002BFBD04F
:10EC50002B6038BD3CA3FF1FFFFFFFFFFFFFFFFF3F
:10EC6000FFFFFFFFFFFFFFFFFFFFFFFFFFFFFFFFB4
:10EC7000FFFFFFFFFFFFFFFFFFFFFFFFFFFFFFFFA4
:10EC800090F800F06DE9024520F007016FF0000CEC
:10EC900010F0070491F820F040F049804FF0000494
:10ECA0006FF00700D1E9002391F840F000F108006F
:10ECB00082FA4CF2A4FA8CF283FA4CF3A2FA8CF3A7
:10ECC0004BBBD1E9022382FA4CF200F10800A4FA0E
:10ECD0008CF283FA4CF3A2FA8CF3E3B9D1E9042362
:10ECE00082FA4CF200F10800A4FA8CF283FA4CF399
:10ECF000A2FA8CF37BB9D1E9062301F1200182FA53
:10ED00004CF200F10800A4FA8CF283FA4CF3A2FA58
:10ED10008CF3002BC6D0002A04BF04301A4612BA66
:10ED2000B2FA82F2FDE8024500EBD2007047D1E969
:10ED3000002304F00305C4F100004FEAC50514F0F8
:10ED4000040F91F840F00CFA05F562EA05021CBFC9
:10ED500063EA050362464FF00004A9E7002A41D0A8
:10ED600040EA010313F00303F0B425D1032A23D9A9
:10ED700004680D68AC421FD1043A35D0A4F10135C6
:10ED800025EA040414F0803F31D1071D0D1D0DE06C
:10ED900057F8043B0E68A3F10134B34224EA03049C
:10EDA0000AD1043A20D014F0803F23D1032A294607
:10EDB000384605F10405EBD803780C789C4202F143
:10EDC000FF320CD182B114B916E06AB17BB110F8F0
:10EDD000013F11F8014FA34202F1FF32F5D0181B99
:10EDE000F0BC7047104670471046F0BC704718469C
:10EDF000F0BC70470020F3E72046F1E740EA01034A
:10EE00009B0770B42BD1032A29D90C46034621460F
:10EE100054F8046BA6F1013525EA060515F0803F8C
:10EE200006D1043A032A43F8046B2146EFD8A2B175
:10EE30000C781C70013A013301313CB16AB111F810
:10EE4000014B03F8014B013A002CF7D12AB11A44C7
:10EE5000002103F8011B9A42FBD170BC70470346A6
:10EE6000E5E700BF2DE9F047254C2568D5F8484176
:10EE70000646884692469946C4B360681F2817DC48
:10EE8000431C76B104EB80050122C5F888A0D4F8B4
:10EE9000881182401143022EC4F88811C5F80891E8
:10EEA0001ED00230636044F820800020BDE8F08767
:10EEB000144B03B34FF4C870FFF746F90446D0B1C2
:10EEC000D5F84831002780E88800C5F84841384621
:10EED0000123C4F88871C4F88C71002EE1D0D1E709
:10EEE000D4F88C110A43C4F88C21DAE705F5A6742E
:10EEF000C5F84841C1E74FF0FF30BDE8F08700BFDB
:10EF0000A80F010049E10000024B13B1024800F0D4
:10EF100005B870470000000029EF000000230146FB
:10EF20001A461846FFF79EBF38B5074D074C2C1BF5
:10EF3000A41005D0013C55F8043D9847002CF9D1A8
:10EF4000BDE8384002F042B80000000000000000B8
:10EF5000F8B5234F0C460646FFF770FCBB685D68AA
:10EF600025F00305291B01F6EF7121F47F6121F0E3
:10EF70000F01A1F58054B4F5805F07DB0021304616
:10EF8000FFF758FEBB682B44984204D03046FFF789
:10EF900057FC0020F8BD61423046FFF74BFE0130C0
:10EFA0000DD0104BBA6819682D1B45F0010530468D
:10EFB000091B55601960FFF743FC0120F8BD0021D3
:10EFC0003046FFF737FEBA68831A0F2BDEDD064C9A
:10EFD0000449246843F00103001B53600860D5E72F
:10EFE0004497FF1FE0A1FF1F509BFF1F002945D042
:10EFF0002DE9F0410D468046FFF720FC55F8047CD2
:10F000006A4927F00103A5F10804E2188E685068E8
:10F01000B24220F0030062D0FE0750600BD455F8D6
:10F02000087CE41B01F1080EA56875453B446FD0D0
:10F03000E768EF60BD6015186D68ED0742D543F0D5
:10F0400001026260E350B3F5007F18D2DB085A1C5E
:10F050004D6851F83270A76001209B1000FA03F34D
:10F0600001EBC2001D430838E0604D6041F83240BA
:10F07000FC604046BDE8F041FFF7E2BB70475A0A2A
:10F08000042A53D89A0902F139077F0002F13805A2
:10F0900001EB870051F827204449083890424DD0B1
:10F0A000516821F003018B4202D292689042F7D15D
:10F0B000D068E060A2608460D4604046BDE8F04162
:10F0C000FFF7BEBB95683A4FBD4203443FD0D068BE
:10F0D000E86043F0010285606260E350B3E7FF0738
:10F0E000034407D455F8082CA41A1344A068E26816
:10F0F000C26090602F4A126843F001009342606042
:10F100008C60B6D32C4B40461968FFF721FFB0E75F
:10F1100011184968C90744D49168D268CA60034489
:10F1200043F0010091606060E350A2E7142A17D811
:10F1300002F15C077F0002F15B05A9E7AA104B68AA
:10F14000012505FA02F213434B600246B1E743F092
:10F1500001024C610C61E560A5606260E35088E7E4
:10F16000542A06D81A0B02F16F077F0002F16E05D0
:10F170008EE7B2F5AA7F06D8DA0B02F178077F0096
:10F1800002F1770584E740F25450824206D89A0C87
:10F1900002F17D077F0002F17C0579E7FE277E25DD
:10F1A00076E743F001026260E35062E74497FF1F95
:10F1B0004C97FF1F4C9BFF1FDCA1FF1F0000780531
:10F1C0003408540B800C3C0F5C12E015FA19141E25
:10F1D0006022AC265C2B0C30BC34023AFF3FFFFFB0
:10F1E00028F5000004F50000E0F40000BCF4000085
:10F1F000C8F2000014F2000038F200005CF20000D7
:10F2000080F20000A8F30000CCF30000BCF1000085
:10F2100084F300000000580246056608540BD80E1F
:10F220005C12E015FA19141E6022AC265C2B0C301F
:10F23000BC34023AFF3FFFFF000090012003140599
:10F24000D0075A0AAC0DCC10B4146A18E81C34214B
:10F2500080252A2B70301437FF3FFFFF0000C800C5
:10F26000F4018403140508072E091C0CD80EF811AC
:10F27000AE159619401F1C25F22B5834FF3FFFFF97
:10F2800000006400C8009001BC021A04DC059E075F
:10F29000F609800CA00F2413A2174C1D5424442FF0
:10F2A000FF3FFFFF40067805B004E8038403200316
:10F2B000BC025802F40190012C01FA00C80096002B
:10F2C000640032001900FFFF0000FF03FF07FF0B7F
:10F2D000FF0FFF13FF17FF1BFF1FFF23FF27FF2B4E
:10F2E000FF2FFF33FF37FF3BFF3FFFFF010201010D
:10F2F00000010101020101020101010101010201FC
:10F3000001020101020101010000010201010201EB
:10F3100001010100010201010201010002020102DA
:10F3200001010201000202020102010102000102C8
:10F3300002020102010100000002020201020101B9
:10F3400001000002020201020100020202020202A6
:10F350000102000202010202020201010002020295
:10F360000202020201000002020002020202000286
:10F370000102020202020202000200020202020272
:10F380000202FFFF0000D007800CD80E0010C01250
:10F39000EC130C17FA19141E6022AC265C2B0C30EF
:10F3A000BC34023AFF3FFFFF0000580246056608E2
:10F3B000540BD80E5C127017FC21F82A70305834A8
:10F3C000DC37663A8C3C803EFF3FFFFF000058026E
:10F3D00046056608540BA00FD4172823F82A442F9B
:10F3E000643284354038663A8C3C803EFF3FFFFFF4
:10F3F0002C011301FA00E100C800AF0096007D0067
:10F4000064004B003200190000000000CDCC4C3DE0
:10F41000CDCCCC3D9A99193ECDCC4C3E0000803EDF
:10F420009A99993E3333B33ECDCCCC3E6666E63EE8
:10F4300000000000070000000C00000010000000A9
:10F4400013000000180000001C0000000000000075
:10F45000070000000C00000013000000180000006E
:10F460001F00000024000000000000000C0000004D
:10F470001800000024000000300000003C000000E4
:10F480004800000000000000FBFFFFFFF4FFFFFF4B
:10F49000EFFFFFFFE8FFFFFFE3FFFFFFDCFFFFFFE2
:10F4A00000000000F4FFFFFFE8FFFFFFDCFFFFFFAD
:10F4B000D0FFFFFFC4FFFFFFB8FFFFFF000078058C
:10F4C000220B0410B4143219B01DFC214826FE2969
:10F4D000822D383126344637663A223DFF3FFFFF02
:10F4E0000000D007100E88133219AA1E2823742793
:10F4F0005C2B442F643284354038663A8C3C803E25
:10F50000FF3FFFFF0000540BEC13FA1908201C25E5
:10F510003629EC2C0C302C33E8357238663AF63B41
:10F52000863D163FFF3FFFFF0000CC10581BFC211B
:10F53000AC26C62A7C2E3831F4334C36A438983A9F
:10F540005A3C543D803E7A3FFF3FFFFFBCF5000030
:10F55000329CFF1F0000FF0FDC9DFF1F0000FF0F0C
:10F56000A93C000088F50000D89DFF1F32005E0115
:10F570000000000000000000493C00005448520018
:10F58000534E53004D415800544F55434820534566
:10F590004E534500455854524120434F4E54524F0C
:10F5A0004C4C45520000000050495443482042450D
:10F5B0004E4400004249544500000000425245417B
:10F5C000544800FF94F500002C9DFF1FF401A00F8C
:10F5D000269DFF1FF401A00F553C0000B4F500006C
:10F5E000EA9BFF1FBC025C12B09DFF1FBC025C12B5
:10F5F0008D3C0000A8F500007E9DFF1FF401A00FC8
:10F60000B89BFF1FF401A00F713C0000ECFD00004F
:10F61000F4FD0000E0FD0000E4FD0000E8FD000056
:10F6200084FC0000A4FD0000C0FD0000C4FD00003B
:10F63000C8FD0000CCFD0000D0FD0000D4FD00009E
:10F64000D8FD0000ACFD0000DCFD000084FC0000E3
:10F6500080FC0000B4FD0000B8FD0000BCFD00000F
:10F6600084FC0000A4FD0000A8FD0000ACFD00002B
:10F67000B0FD000090FD000094FD000098FD00002A
:10F680009CFD0000A0FD000080FD000084FD000046
:10F6900088FD0000900201008CFD0000FCFD0000D0
:10F6A00000FE000004FE000008FE00000CFE00004A
:10F6B00010FE000014FE000018FE00001CFE0000FA
:10F6C00020FE000024FE000028FE00002CFE0000AA
:10F6D0000100000030FE00000700000000000000F4
:10F6E000010000002D4A0000A8FF000000000501F5
:10F6F00008000000D08DFF1F5D49000006000000DB
:10F7000009000000548FFF1F000000009800010056
:10F710008C000100909DFF1F0000300000000000E1
:10F720003D570000694800000000000034FF000061
:10F730000000010108000000EC8EFF1F94FE000095
:10F74000000002010C0000009C8FFF1F0000000061
:10F750006800010074000100CC9BFF1F0000010045
:10F76000010000002D4D00009D460000000000003B
:10F7700001000000B0FF00000600000030FE0000A5
:10F780000000040508000000E88BFF1F01000000D6
:10F79000A8FF0000090000000000000001000000B8
:10F7A000F162000001000000D0FF00000300000033
:10F7B00000000000B00001008C0001008C9DFF1FC4
:10F7C00000003000000000003D57000069480000C4
:10F7D000000000000000000001000000D153000004
:10F7E00000000000D8FF0000E0FF0000349DFF1F74
:10F7F0000100100006000000295F0000BD46000067
:10F800003551000000000000800001008C00010064
:10F81000929DFF1F00003000000000003D570000D7
:10F820006948000000000000000000000000000027
:10F8300000000000000000000000000000000000C8
:10F8400000000000000000000000000000000000B8
:10F8500000000000000000000000000000000000A8
:10F860000000000000000000000000000000000098
:10F870000000000000000000000000000000000088
:10F880000000000000000000000000000000000078
:10F890000000000000000000000000000000000068
:10F8A0000000000000000000000000000000000058
:10F8B0000000000000000000000000000000000048
:10F8C0000000000000000000000000000000000038
:10F8D0000000000000000000000000000000000028
:10F8E0000000000000000000000000000000000018
:10F8F0000000000000000000000000000000000008
:10F9000000000000000000000000000000000000F7
:10F9100000000000000000000000000000000000E7
:10F9200000000000000000000000000000000000D7
:10F9300000000000000000000000000000000000C7
:10F94000000000000000000000000000007FFFFF3A
:10F95000000003F9FFFFFC0000000000007FFFFF34
:10F96000800007F9FFFFFE000000000000600001BA
:10F97000C0000E198000070000000000006FFFFCAF
:10F98000C0001DD9BFFFF30000000000006FFFFEA4
:10F99000C0003BD9BFFFFB0000000000006C000668
:10F9A000C00077D9B0001B0000000000006C00060A
:10F9B000C000EED9B0001B0000000000006C000683
:10F9C000C001DCD9B0001B0000000800006C00067C
:10F9D000C003B8D9B0001B0000001800006FFFFE84
:10F9E000C0077FD9B0001B0000001800006FFFFCAB
:10F9F000C00EFFD9B0001B0000C01800006000015D
:10FA0000C01C0019B0001B0000C03800006FFBFFD5
:10FA1000803BFFD9B0001B0000C03000006FFDFF2D
:10FA20000077FFD9B0001B0001E03000006C0EE051
:10FA300000EE00D9B0001B0001E03000006C077040
:10FA400001DC00D9B0001B0001B03000006C03B82D
:10FA500003B800D9B0001B0001B03000006C01DC1D
:10FA6000077000D9B0001B00019820C0406C00EE68
:10FA70000EE000D9B0001B00030C20C0C06C007762
:10FA80001DC000D9BFFFFB00030C20C0C06C003BB1
:10FA9000BB8000D9BFFFF300030620C1C06C001D6E
:10FAA000F70000D98000070003032083806C000E5C
:10FAB000EE0000D9FFFFFE000303B183806C000756
:10FAC0005C0000D9FFFFFC000301F187800000000B
:10FAD00000000000000000000300F18D8000000025
:10FAE0000000000000000000030071B98000000069
:10FAF0000000000000000000030031F18000000061
:10FB00000000000000000000030000C180000000B1
:10FB100000000000000000000300000000000000E2
:10FB200000000000000000000300000000000000D2
:10FB300000000000000000000200000000000000C3
:10FB400000000000000000000000000000000000B5
:10FB500000000000000000000000000000000000A5
:10FB60000000000000000000000000000000000095
:10FB70000000000000000000000000000000000085
:10FB80000000000000000000000000000000000075
:10FB90000000000000000000000000000000000065
:10FBA0000000000000000000000000000000000055
:10FBB0000000000000000000000000000000000045
:10FBC0000000000000000000000000000000000035
:10FBD0000000000000000000000000000000000025
:10FBE0000000000000000000000000000000000015
:10FBF0000000000000000000000000000000000005
:10FC000000000000000000000000000000000000F4
:10FC100000000000000000000000000000000000E4
:10FC20000000000000000000580001000000030177
:10FC300006000000B88DFF1F00000000BC0001009E
:10FC40008C000100B09BFF1F00003000000000008E
:10FC50002D570000AD46000000000000000000002D
:10FC60008CFE000058FE0000A09BFF1F0000090052
:10FC700000000000514D0000DD46000000000000C3
:10FC80004F4E00004F46460055534200424154003B
:10FC90004C4F5720000000004D454E55202020209D
:10FCA000202020202058585820592E595600000056
:10FCB00058000000524F54004D454C0044594E002E
:10FCC0006D73000042544800424954004C565200A3
:10FCD0004E524D0052455600312F00004154000055
:10FCE0004D4F4400504244004543420045435300B9
:10FCF0004C564C004C565000474C4400454348007D
:10FD0000762E0000312E342E37000000534554006B
:10FD1000434C52004E755241440000006669726DBA
:10FD20007761726520762E0055534220706F77659B
:10FD300072000000416C6B616C696E6520626174D9
:10FD40007465727900000000302025206174200065
:10FD50004E694D482062617474657279000000003C
:10FD60004C69506F20626174746572790000000004
:10FD7000444F4E275400000050414E4943000000BC
:10FD800045574900455758005341580045565200C1
:10FD900048524D00355448004F43540035444E00FE
:10FDA0004F444E004D5700004650000043460000AF
:10FDB000535000005357000053454C005345450035
:10FDC00042520000564C0000455800004D572B0091
:10FDD00042522B00564C2B0045582B00554E4F00DD
:10FDE000414C4B004E4D48004C4950004252544843
:10FDF0000000000050544348000000002D34000073
:10FE00002D3300002D3200002D3100004C494E00F2
:10FE10002B3100002B3200002B3300002B3400006C
:10FE200053310000533200005A3100005A320000B2
:10FE30005649425241544F00444952454354494F58
:10FE40004E000000434F4E54524F4C005351554505
:10FE50004C434820420000004C4556454C000000F1
:10FE600053454E53452042544500000053515545DB
:10FE70004C4348204C00000053454E5345204C56FF
:10FE80005200000052455455524E00004445505413
:10FE9000480000005345545550204354524C5300E1
:10FEA000455854524120504B4559000046494E4751
:10FEB0004552494E470000004C4556454C204343AF
:10FEC000000000004D4F44204B4559004445474C2D
:10FED00049544348000000004841524D2053454CCE
:10FEE0000000000053455249455300004558435413
:10FEF000204841524D0000004841524D2052414E91
:10FF00004745000045584354204343204200000029
:10FF10004558435420434320410000005049544376
:10FF20004842454E44000000504F52542F474C4425
:10FF3000000000005345545550204252454154485A
:10FF40000000000056454C20424F4F535400000023
:10FF500056454C2044454C415900000043555256EB
:10FF60004500000056454C4F4349545900000000DD
:10FF7000425245415448204154000000434320422E
:10FF80002052495345000000425254482043432028
:10FF900042000000425254482043432041000000E8
:10FFA00041424F55540000004558545241530000FF
:10FFB000524F5441544F52005345545550204354CE
:10FFC0004C000000534554555020425200000000A0
:10FFD00041444A55535400004D4944492043480088
:10FFE0004D4944492043484E4C00000042415420B2
:10FFF0005459504500000000574C204348414E00E2
:020000021000EC
:10000000574C20504F574552000000004641535472
:1000100020424F4F54000000444143204F555400AC
:1000200053504543204B4559000000004C45474183
:1000300043592042520000004C454741435920504B
:10004000420000004F435441564500005452414E77
:1000500053504F5345000000524F5441544F5220CB
:1000600053455455500000005052494F524954597D
:10007000000000004D4F4E4F205052494F000000ED
:10008000524F5441544520340000000053454D491F
:10009000544F4E4553000000524F544154452033B5
:1000A00000000000524F544154452032000000002F
:1000B000524F5441544520310000000050415241FC
:1000C0004C4C454C00FFFFFF01000000C4FF000046
:1000D000040000002C01000000000000A40001004A
:1000E0008C0001008E9DFF1F00003000000000000A
:1000F0003D570000694800000000000001000000BA
:10010000B8FF000005000000000000005CFF0000D8
:100110005CFF0000A49BFF1F00000C000300000018
:100120004D5E0000CD460000000000000100000010
:10013000A0FF0000080000000021110202000000E2
:10014000002111020504FFFF003E7FFF4E7545565A
:1001500049633031000000007676764E7545564989
:10016000636363007676764E754556496330346531
:10017000657676767676767676000000496E7661DC
:100180006C696420636F6E66696720666F726D616B
:1001900074000000496E76616C6964206368656371
:1001A0006B73756D00000000496E76616C696420A8
:1001B000636F6E6669672073697A6500496E766160
:1001C0006C696420636F6E66696720766572736917
:1001D0006F6E00004E75455649000000496E76610D
:1001E0006C6964206D6573736167652E00000000A3
:1001F000653030006330300053656E64696E67208F
:10020000636F6E6669672E2E2E000000436F6E6668
:1002100069672073656E742E000000006330330040
:1002200053656E64696E672076657273696F6E2EB2
:100230000000000063303200526563656976696EC4
:100240006720636F6E6669672E2E2E004E657720DD
:10025000636F6E6669672073617665642E000000C7
:10026000556E6B6E6F776E206D6573736167652E6B
:100270000000000065303100436F6E666967206DD5
:10028000676D7400506F776572206F6666204E75DB
:1002900045564900746F2065786974005265616441
:1002A000792E00FF34800440400000001211FFFF4F
:1002B000FF02020000001310FFFFFF020200000017
:1002C0001800000034800440800000001EFFFFFF83
:1002D000FF02000000001DFFFFFFFF020000000002
:1002E000190000000000000000000000F97E00007E
:1002F000BD7E0000717E0000B97E0000757E0000AA
:10030000817E0000A17E0000000103070F1F3F7FD8
:100310002200FF2100FFFFFF0080C0E0F0F8FCFE9C
:100320000000000000000000519E0000ADA200008F
:10033000717E00007D88000015890000F99600009C
:10034000AD960000E1960000B9960000CD96000041
:10035000C9950000F996000021970000118B00005C
:1003600059930000F5920000F1970000FD960000FF
:1003700055980000F5980000DA02818FDA1281FFAB
:10038000000060000000000000000000000000000D
:1003900000E000000000000000000000000000017C
:1003A000E00000000000000000000000000001F07C
:1003B0000000000000000000000000000003F0004A
:1003C00000000000000000000000000007F0000036
:1003D000000000000000000000000007F80000001E
:1003E000000000000000000000000FF80000000303
:1003F000C0007E000001E0007F0FF800000003C095
:1004000000FE000001E000FFEFF800000003C00064
:10041000FE000001E000FFFFF800000003C000F054
:100420000000000F007FFE7FC0000003C000F0004E
:1004300000000F003FFE7FF83FF1FBCFFCFEF3BC56
:100440003DEFE01FFE7FFF7FFBFFDFFEFEFFBC3DB9
:10045000EFE01FC6FFFF7FFBFFDFFEFEFFBC3DEFAF
:10046000E00FE3C7FE787BC3DE1EF0FFBC3DEF006C
:1004700007FF87FC787BC3DE1EF0F83C3DEF0001F0
:10048000FFFFF0007BC3C01EF0F03C3DEF0001F326
:100490007FE03FFBC3CFFEF0F03C3DEF0003E33FC6
:1004A000807FFBC3DFFEF0F03C3DEF0007E73C0040
:1004B000787BC3DE1EF0F03C3DEF0007FFBE007806
:1004C0007BC3DE1EF0F03C3DEF0007FFFE00787BB3
:1004D000C3DE1EF0F03C3DEF000FFFFE007FFBFF90
:1004E000DFFEF0F03FFDEFE00FFFFF007FFBFFDFDF
:1004F000FEF0F03FFDEFE00FF9FF003E79F9CF9EEF
:10050000F0F01F3DE7E01FF1FF00000000000000D9
:1005100000000000001F80FF007FFFFFFFFFFFFFC4
:10052000FFFFFFE01C007F007FFFFFFFFEB46D8830
:100530008D18E000001F007FFFFFFFFE95AD7DB529
:1005400077E000000F007FFFFFFFFEA5AD9D8D1936
:10055000E0000006007FFFFFFFFEB5ADEDB57EE0D9
:10056000AED580A8D300408D2000A1C8DB40A4A652
:100570002EAFFFFF0000000000018000000000001F
:1005800000000000038000000000000000000007E1
:10059000C000000000000000000007C000000000D4
:1005A00000000000000FC00000000000000000007C
:1005B0001FE00000000000000000001FE00000003D
:1005C0000000000000003FE000000000000000000C
:1005D000003FF00000000000000000007FF000007D
:1005E00000000000001FF87FF00000000000000085
:1005F0003FFE7FF0000000000000003FFF7FF000A2
:100600000000000000001FFFFBE0000000000000F1
:10061000000FFFF9FFC00000000000000FFFF9FF0E
:10062000F800000000000007FFF1FFFF00000000DD
:10063000000003FC73FFFF80000000000001FE3F8C
:10064000FFFF80000000000000FF1E0FFF00000001
:10065000000000007FFE1FFC000000000000003FC3
:10066000FFFFF8000000000000000FDFFFE00000C7
:1006700000000000001F19FFC00000000000000083
:100680003F3CFF00000000000000007E7CF80000FE
:100690000000000000007FFE7C0000000000000061
:1006A00000FFFFFC0000000000000000FFFFFE0054
:1006B00000000000000000FFFFFE0000000000003E
:1006C0000001FFEFFE0000000000000001FFCFFE70
:1006D0000000000000000003FF07FE000000000013
:1006E000000003FC07FE0000000000000003F00310
:1006F000FE00000000000000018000FE000000007D
:100700000000000000007E0000000000000000006B
:10071000003E000000000000000000000C0000008F
:10072000000000078000FC000003C00000000780FC
:1007300001FC000003C0000000078001FC00000372
:10074000C0000000078001E00000001E000000075C
:100750008001E00000001E007FE3F79FF9FDE778CD
:100760007BDFC0FFF7FFBFFDFDFF787BDFC0FFF73A
:10077000FFBFFDFDFF787BDFC0F0F787BC3DE1FFE9
:10078000787BDE00F0F787BC3DE1F0787BDE00008F
:10079000F787803DE1E0787BDE007FF7879FFDE112
:1007A000E0787BDE00FFF787BFFDE1E0787BDE00CD
:1007B000F0F787BC3DE1E0787BDE00F0F787BC3DD9
:1007C000E1E0787BDE00F0F787BC3DE1E0787BDE9E
:1007D00000FFF7FFBFFDE1E07FFBDFC0FFF7FFBFDA
:1007E000FDE1E07FFBDFC07CF3F39F3DE1E03E7B7A
:1007F000CFC00000000000000000000000FFFFFF6D
:10080000FFFFFFFFFFFFFFC0FFFFFFFFFD68DB11E2
:100810001A31C0FFFFFFFFFD2B5AFB6AEFC0FFFF3D
:10082000FFFFFD4B5B3B1A33C0FFFFFFFFFD6B5B20
:10083000DB6AFDC0DA0281FF00000000000000005A
:10084000519E0000ADA20000717E00007D88000076
:1008500031AA0000F9960000AD960000E196000074
:10086000B9960000CD960000C9950000F9960000E9
:10087000219700001D970000459700009D970000FC
:10088000F1970000FD96000055980000F5980000D3
:1008900000000000003E5B4F5B3E3E6B4F6B3E1C1A
:1008A0003E7C3E1C183C7E3C181C577D571C1C5E31
:1008B0007F5E1C00183C1800FFE7C3E7FF00182408
:1008C0001800FFE7DBE7FF30483A060E26297929B2
:1008D00026407F050507407F05253F5A3CE73C5AE7
:1008E0007F3E1C1C08081C1C3E7F14227F22145FC4
:1008F0005F005F5F06097F017F006689956A60601F
:1009000060606094A2FFA29408047E040810207E18
:10091000201008082A1C08081C2A08081E1010109D
:10092000100C1E0C1E0C30383E3830060E3E0E06E3
:10093000000000000000005F000000070007001436
:100940007F147F14242A7F2A1223130864623649F5
:100950005620500008070300001C224100004122DD
:100960001C002A1C7F1C2A08083E080800807030E2
:100970000008080808080000606000201008040251
:100980003E5149453E00427F400072494949462157
:1009900041494D331814127F1027454545393C4ACB
:1009A00049493141211109073649494936464949E2
:1009B000291E00001400000040340000000814222A
:1009C0004114141414140041221408020159090698
:1009D0003E415D594E7C1211127C7F494949363E99
:1009E000414141227F4141413E7F494949417F097F
:1009F0000909013E414151737F0808087F00417F8A
:100A000041002040413F017F081422417F40404087
:100A1000407F021C027F7F0408107F3E4141413E1F
:100A20007F090909063E4151215E7F0919294626A1
:100A30004949493203017F01033F4040403F1F20A5
:100A400040201F3F4038403F63140814630304787C
:100A500004036159494D43007F414141020408109C
:100A600020004141417F04020102044040404040D7
:100A7000000307080020545478407F284444383845
:100A800044444428384444287F38545454180008B7
:100A90007E090218A4A49C787F0804047800447D91
:100AA00040002040403D007F1028440000417F402E
:100AB000007C047804787C08040478384444443882
:100AC000FC1824241818242418FC7C080404084862
:100AD0005454542404043F44243C4040207C1C20B3
:100AE00040201C3C4030403C44281028444C90900E
:100AF000907C4464544C4400083641000000770068
:100B000000004136080002010204023C2623263C74
:100B10001EA1A161123A4040207A385454555921FF
:100B200055557941225454784221555478402054E7
:100B30005579400C1E527212395555555939545435
:100B4000545939555454580000457C410002457DA4
:100B5000420001457C407D1211127DF0282528F0CD
:100B60007C545545002054547C547C0A097F4932FA
:100B7000494949323A4444443A324A4848303A4171
:100B800041217A3A42402078009DA0A07D3D42421A
:100B9000423D3D4040403D3C24FF2424487E4943A3
:100BA000662B2FFC2F2BFF0929F620C0887E090316
:100BB00020545479410000447D413048484A32383D
:100BC0004040227A007A0A0A727D0D19317D262969
:100BD000292F28262929292630484D402038080861
:100BE000080808080808382F10C8ACBA2F10283495
:100BF000FA00007B000008142A142222142A140888
:100C00005500550055AA55AA55AAFF55FF55FF0096
:100C10000000FF00101010FF00141414FF0010104B
:100C2000FF00FF1010F010F0141414FC001414F75F
:100C300000FF0000FF00FF1414F404FC141417104C
:100C40001F10101F101F1414141F00101010F0009C
:100C50000000001F101010101F10101010F01000D6
:100C60000000FF101010101010101010FF100000E6
:100C700000FF140000FF00FF00001F10170000FC21
:100C800004F414141710171414F404F40000FF00F3
:100C9000F714141414141414F700F714141417147C
:100CA00010101F101F141414F4141010F010F00082
:100CB000001F101F0000001F14000000FC140000A3
:100CC000F010F01010FF10FF141414FF1410101087
:100CD0001F00000000F010FFFFFFFFFFF0F0F0F03A
:100CE000F0FFFFFF0000000000FFFF0F0F0F0F0FCE
:100CF0003844443844FC4A4A4A347E02020606021A
:100D00007E027E0263554941633844443C04407E80
:100D1000201E2006027E020299A5E7A5991C2A49F9
:100D20002A1C4C7201724C304A4D4D303048784884
:100D300030BC625A463D3E494949007E0101017E70
:100D40002A2A2A2A2A44445F444440514A444040C3
:100D5000444A51400000FF0103E080FF0000080802
:100D60006B6B083612362436060F090F0600001882
:100D7000180000001010003040FF0101001F0101A9
:100D80001E00191D1712003C3C3C3C0000000000F6
:100D90000D0AFFFF050E08090D0C06070F040013CE
:100DA0000393050E08090D0C06070F04FFFFC58508
:100DB000848687C4FFFF001303931A9217FFFFFF77
:100DC0006FF07F030370037813F0800FFBD0704740
:100DD0004008FE4340A004404408FE4344A00440B1
:100DE0000018FE4300C004403000FE433090044031
:100DF0003400FE43349004401C18FE431CC00440E1
:100E00001018FE4310C004400818FE4308C00440F8
:100E10000C18FE430CC004400C10FE430CB0044000
:100E20001010FE4310B004401810FE4318B00440E8
:100E30001C10FE431CB004401410FE4314B00440C8
:100E40000418FE4304C004400010FE4300B00440F8
:100E50000008FE4300A004400408FE4304A0044030
:100E60000C08FE430CA004400808FE4308A0044000
:100E70001418FE4314C004401818FE4318C0044060
:100E80000410FE4304B004400810FE4308B00440C0
:100E90001400FE43149004404C08FE434CA0044050
:100EA0000420FE4304D004402410FE4324B0044038
:100EB0002010FE4320B004402810FE4328B0044018
:100EC0002C10FE432CB004400020FE4300D0044010
:100ED0004808FE4348A004401000FE431090044020
:100EE000090AFFFFFFFFFFFFFFFFFFFFFFFFFF0DEF
:100EF00000060807FFFF0E0FFF0CFFFFFFFFFFFFBD
:100F00000B05FFFF15191519000100003892FF1F8E
:100F100012000000000200006492FF1F7300000036
:100F200000220100D892FF1F2100000000210100D3
:100F3000C092FF1F0900000000030000FC92FF1F89
:100F400000000000010309044C92FF1F0000000094
:100F5000020309044890FF1F000000000303090476
:100F60000093FF1F000000000000000000000000D0
:100F70000000000065787000000000000000E03F05
:100F8000000000000000E0BF763C7935EF39EA3D13
:100F9000763C7935EF39EABD0000E0FE422EE63FAF
:100FA0000000E0FE422EE6BF1893FF1FF8B500BF19
:100FB000F8BC08BC9E46704709EF000035040000ED
:0C0FC000ED3B0000E5570000ED7A00005A
:040FCC00F8B500BFB5
:100FD00038B5084B1C681C6054B1074D94FAA4F353
:100FE000B3FA83F355F823309847631E1C40F5D1BC
:100FF00038BD00BFA0D004402892FF1F38B5084B71
:101000001C681C6054B1074D94FAA4F3B3FA83F33F
:1010100055F823309847631E1C40F5D138BD00BFFA
:10102000A0C004400892FF1F38B5084B1C681C6024
:1010300054B1074D94FAA4F3B3FA83F355F823306F
:101040009847631E1C40F5D138BD00BFA0B00440D6
:10105000D891FF1F38B5084B1C681C6054B1074D70
:1010600094FAA4F3B3FA83F355F823309847631E38
:101070001C40F5D138BD00BFA0A004408891FF1FDF
:1010800038B5084B1C681C6054B1074D94FAA4F3A2
:10109000B3FA83F355F823309847631E1C40F5D10B
:1010A00038BD00BFA09004405091FF1F0000000019
:1010B000002000000000F041280000000C000000AB
:1010C0005A000000F3FFFFFFDFFFFFFFA3FFFFFF5A
:1010D000AEFFFFFF7300000076000000020000007A
:1010E00004000000D8FFFFFFB5FFFFFFA2FFFFFFD6
:1010F00002000000FBFFFFFF0000000000000000F6
:1011000000000000000000000000000000000000DF
:1011100000000000000000000100000000200000AE
:101120000020000000100000AB0A000000080000D2
:10113000660600005505000092040000000400004F
:101140008E03000033030000E8020000AB02000041
:1011500000200000F3FFFFFFF4FFFFFFF5FFFFFF9C
:10116000F6FFFFFFF7FFFFFFF8FFFFFFF9FFFFFFAD
:10117000FAFFFFFFFBFFFFFFFCFFFFFFFDFFFFFF8D
:10118000FDFFFFFFFEFFFFFFFFFFFFFF000000006E
:1011900014050000000102070B0102070B4A1400AE
:1011A00002000C0024000000A8FFFFFFBCFFFFFFAF
:1011B000E1FFFFFF0D0000000400000078000000C8
:1011C00079000000BCFFFFFFABFFFFFFDEFFFFFF6A
:1011D0001700000057000000100000000A00000087
:1011E00008000000150000001800000029000000A1
:1011F0000200FFFFFFFF00004CF50000DCF50000DF
:10120000F4F50000C4F5000064F5000000000000E3
:10121000A0FE0000A0FE0000049EFF1F00001900B9
:1012200000000000000000000000000000000000BE
:101230000000000038FE000038FE0000169CFF1F72
:10124000000001000100000000000000000000009C
:10125000000000000000000044FE000044FE00000A
:10126000229DFF1F0000020001000000000000009E
:101270000000000000000000000000006CFE000004
:1012800058FE0000128AFF1F01001E00000000002F
:10129000000000000000000000000000010000004D
:1012A00000000000ACFE0000ACFE00007C9BFF1FB5
:1012B0000000040001000000000000000000000029
:1012C000000000000000000028FF000028FF0000D0
:1012D000369CFF1F00000400010000000000000019
:1012E000000000000000000000000000D8FE000028
:1012F000E4FE0000A89DFF1F0000040001000000A4
:1013000000000000000000000000000000000000DD
:10131000B8FE0000B8FE0000049CFF1F00007F0024
:1013200001000000000000000000000000000000BC
:101330000000000060FE000058FE0000608AFF1FF1
:10134000010011000000000000000000000000008B
:10135000000000000000000070FF000070FF0000AF
:101360002A9CFF1F00000100010000000000000097
:101370000000000000000000C48AFF1F5CFC0000A9
:10138000CC8FFF1FA08AFF1F2C8CFF1FE88AFF1F36
:10139000A08BFF1FC88EFF1F0000000094FF0000FD
:1013A00094FF0000709DFF1F00000A000100000074
:1013B000000000000000000000000000000000002D
:1013C00078FE000058FE0000108AFF1F01000C008C
:1013D000000000000000000000000000000000000D
:1013E000000000002C0001002C000100269CFF1FC3
:1013F00000000100010000000000000000000000EB
:10140000000000000000000050FF000050FF00003E
:10141000249CFF1F00001E000100000000000000CF
:101420000000000000000000000000007CFF000041
:101430007CFF00008C9BFF1F01000A0001000000E0
:10144000000000000000000000000000000000009C
:101450000C0001000C0001007A9DFF1F000001003C
:10146000000000000000000000000000000000007C
:10147000000000001CFF00001CFF0000D69BFF1FA7
:1014800000000C0000000000000000000000000050
:10149000000000000000000020000100200001000A
:1014A000869DFF1F000001000100000000000000F9
:1014B000000000000000000000000000F8FF000035
:1014C000F8FF00002090FF1F040050000000000003
:1014D000000000000000000000000000000000000C
:1014E0000000010000000100889EFF1F00000300B3
:1014F00000000000000000000000000000000000EC
:10150000000000004C0001004C000100909BFF1FF8
:1015100000001800000000000000000000000000B3
:10152000000000000000000044FF000044FF000035
:10153000809BFF1F00000900010000000000000068
:10154000000000000000000038FC0000B0F70000C0
:10155000D800010008F7000004F800004CF7000074
:10156000148EFF1F508CFF1F048DFF1F2490FF1F40
:10157000808EFF1FBC8CFF1F4C8DFF1F288DFF1F0F
:1015800000000000ECFE0000F8FE0000E09DFF1FE0
:101590000000060001000000000000000000000044
:1015A00000000000000000003800010038000100C9
:1015B000E89BFF1F00000100010000000000000088
:1015C000000000000000000000000000C4FE000059
:1015D000C4FE0000B29DFF1F00001E0000000000BE
:1015E00000000000000000000000000000000000FB
:1015F00010FF000010FF0000CE9BFF1F0000040042
:1016000001000000000000000000000000000000D9
:1016100000000000ECFF0000ECFF0000169DFF1F23
:1016200000000200010000000000000000000000B7
:101630000000000000000000440001004400010020
:10164000889DFF1F00000600000000000000000051
:101650000000000000000000000000004CFE000040
:1016600058FE00002C89FF1F01001E000000000032
:10167000000000000000000000000000088CFF1FB8
:101680000C8FFF1F988CFF1FC48BFF1F788FFF1FCD
:1016900008010100748CFF1F948DFF1F00000000E3
:1016A00088FF000088FF0000B69DFF1F00007F003C
:1016B0000100000000000000000000000000000029
:1016C00000000000CCFE0000CCFE0000C29DFF1F09
:1016D00000004600000000000000000000000000C4
:1016E00000000000708DFF1FA48EFF1FE0F70000B8
:1016F000A4F70000C8000100FC00010070F7000022
:101700008CF700002C0101000000000064FF0000C5
:1017100064FF0000949BFF1F00007F000100000099
:10172000000000000000000000000000348BFF1FDC
:101730005C8EFF1FFC8FFF1FF08DFF1F588BFF1F5C
:10174000D0F60000308FFF1F388EFF1F7C8BFF1FED
:101750007C8AFF1F108BFF1FE08CFF1F0000000022
:1017600084FE000058FE00006089FF1F0000040096
:101770000000000000000000000000000000000069
:101780000000000001000000000000000000000058
:1017900004FF000004FF0000C49DFF1F00007F0045
:1017A0000100000000000000000000000000000038
:1017B00004000000000000001800010018000100F3
:1017C000849DFF1F000001000000000000000000D9
:1017D000000000000000000016034E0075004500E8
:1017E0005600490020004D00490044004900000017
:1017F000EC02010000000000E8030000000000000F
:1018000000600640A402010000000000000000008B
:1018100000000000000000000000000000000000C8
:1018200000000000000000000000000000000000B8
:1018300000000000000000000000000000000000A8
:101840000000000000000000000000000000000098
:10185000000000000000000000000000EC02010099
:1018600000000000E80300000000000000700640D7
:10187000C4020100000000000000000000000000A1
:101880000000000000000000000000000000000058
:101890000000000000000000000000000000000048
:1018A0000000000000000000000000000000000038
:1018B0000000000000000000000000000000000028
:1018C000000000000000000081A1000081A10000D4
:1018D00081A1000081A100000A04000040A3FF1FB5
:1018E000BDAA0000BDAA0000BDAA0000BDAA00005C
:1018F000BDAA0000BDAA0000BDAA0000BDAA00004C
:10190000BDAA0000BDAA0000BDAA0000BDAA00003B
:10191000BDAA0000BDAA0000BDAA0000BDAA00002B
:10192000BDAA0000BDAA0000BDAA0000BDAA00001B
:10193000BDAA0000BDAA0000BDAA0000BDAA00000B
:10194000BDAA0000BDAA0000BDAA0000BDAA0000FB
:10195000BDAA0000BDAA0000BDAA0000BDAA0000EB
:10196000BDAA0000BDAA0000BDAA0000BDAA0000DB
:10197000BDAA0000BDAA0000BDAA0000BDAA0000CB
:10198000BDAA0000BDAA0000BDAA0000BDAA0000BB
:10199000BDAA0000BDAA0000BDAA0000BDAA0000AB
:1019A000BDAA0000BDAA0000BDAA0000BDAA00009B
:1019B000BDAA0000BDAA0000BDAA0000BDAA00008B
:1019C00008000000FFFFFFFF1201100100000040AF
:1019D000C0168504750201020301000018035400BB
:1019E000650065006E007300790064007500690091
:1019F0006E006F0009027300020100C0320904008A
:101A00000002010300000724010001250006240252
:101A1000010100062402020200092403010301025D
:101A20000100092403020401010100090504024028
:101A300000000000052501010109058302400000A6
:101A40000000052501010309040100020300000054
:101A50000921110100012221000705810340000135
:101A6000070502032000020006C9FF0904A15C75F6
:101A700008150026FF00954009758102952009761A
:101A8000910295040976B102C00000000403090424
:101A90000C03000000000000000000000000000037
:101AA0000000000000000100000000000496FF1F7D
:101AB0006C96FF1FD496FF1F00000000000000007E
:101AC0000000000000000000000000000000000016
:101AD0000000000000000000000000000000000006
:101AE00000000000000000000000000000000000F6
:101AF00000000000000000000000000000000000E6
:101B000000000000000000000000000000000000D5
:101B100000000000000000000000000000000000C5
:101B200000000000000000000000000000000000B5
:101B300000000000000000000000000000000000A5
:101B40000000000000000000000000000000000095
:101B500001000000000000000E33CDAB34126DE632
:101B6000ECDE05000B00000000000000000000009B
:101B70000000000000000000000000000000000065
:101B80000000000000000000000000000000000055
:101B90000000000000000000000000000000000045
:101BA0000000000000000000000000000000000035
:101ED0001893FF1F00000000000000004497FF1F40
:101EE0004497FF1F4C97FF1F4C97FF1F5497FF1FEE
:101EF0005497FF1F5C97FF1F5C97FF1F6497FF1F9E
:101F00006497FF1F6C97FF1F6C97FF1F7497FF1F4D
:101F10007497FF1F7C97FF1F7C97FF1F8497FF1FFD
